:020000040800F2
:1000000000200010B53603081D3703086D65000891
:100010001D3703081D3703081D37030800000000C3
:100020000000000000000000000000001D37030871
:100030001D370308000000001D370308E9590008B8
:100040001D3703081D3703081D3703081D37030834
:100050001D3703081D370308C10C0008B10D000847
:10006000750D0008390D0008FD0C0008A12B0008D3
:10007000912B0008812B0008712B0008612B0008D0
:100080004D2B0008392B00081D3703081D370308C6
:100090001D3703081D3703081D370308870C0008A8
:1000A0001D5100085D5100080D51000885510008E0
:1000B0004D5100083D5100082D5100081D3703081F
:1000C0001D3703081D3703081D3703081D370308B4
:1000D0001D370308155B0008995A00081D5A0008CF
:1000E000B56500081D3703081D3703081D370308D1
:1000F0001D3703081D3703081D3703081D37030884
:100100000000000000000000000000001D37030890
:100110001D3703081D3703088530010869300108C1
:10012000252B0008112B0008FD2A0008E92A0008E9
:10013000D52A00081D370308000000000000000059
:100140001D3703081D3703081D3703080000000092
:10015000000000000000000000000000000000009F
:1001600000000000000000001D3703081D370308D1
:100170001D37030800000000000000000000000020
:08018000000000001D37030818
:100188002D2343702E2303712F23C371704700283A
:1001980070B51EDB0928044620DD012303EB830329
:1001A8005B00B0FBF3F2092AF8D87BB10D4EB4FB23
:1001B800F3F00928CCBF57223022A6FB03E50244FE
:1001C80003FB1044EB0801F8012BF0D100230B705E
:1001D80070BD2D230B7040420131DBE7303001F850
:1001E800010BF3E7CDCCCCCC884230B44FF00104FE
:1001F8002ED301FB04F4B0FBF4F58D42F9D284B19F
:10020800AAB901E0B0FBF4F5092DCCBF5722302282
:100218002A4404FB150003F8012BB4FBF1F4002C6D
:10022800F0D100221A7030BC7047B0FBF4F5092DEC
:10023800CCBF372230222A4404FB150003F8012BD7
:10024800B4FBF1F4002CF0D100221A7030BC7047D6
:100258000546002AEBD1D7E72DE9F04714461D469D
:10026800064600234FF47A722046294633F04AF8AE
:10027800DFF840814B4A4C4F88FB00310144C317DB
:1002880082FB002EC3EB611188FB012887FB002746
:100298008644464AC3EBEE2EC1EB011C82FB0E29B5
:1002A800A0EB8C0C0744424A86F806C0C3EB2747EC
:1002B8004FEAEE7C08EB010ACCEBA90C82FB078223
:1002C8004FEAE1780CEB4C0CC8EB6A18AEEBCC0E9D
:1002D800C8EB0818DFF8E0C086F804E0A1EB880155
:1002E80071718CFB0010F917C1EBE21240F2B551A5
:1002F80001FB1272C3EBE050B2F5896F4FEA800739
:100308003CDA40F2DA239A4242DCB2F5B77FB4BF56
:100318004FF0000C4FF0010C4FEA4C09DFF89C80BD
:1003280009EB0C0308EBC3031FFA8CFED88A09EB10
:100338000C0108EBC10116310B2301E031F8020D65
:10034800824218DA013BF9D1CC44012338F83C0049
:10035800B37007F2B2770132121ABE44F270A6F8EF
:1003680000E0204629464FF47A72002332F0CAFF93
:100378003281BDE8F0870133DBB2E9E74FF0030EC5
:10038800F44640F29650DFF834804FF00609CEE785
:100398004FF0020EDFF82480F44640F229404FF077
:1003A8000409C4E7C5B3A29107452EC2ABAAAA2A7D
:1003B80073B06D1689888888792D0311784B0308E6
:1003C80003685A1C0260197070472DE9F047089CB1
:1003D8002578002B804689460CBF4FF0200A4FF045
:1003E800300A661C35B3002A29DD334601E002468F
:1003F80098B113F8011B501E0029F8D1971E60B15F
:100408003D46013D51464046C8476B1C002BF8DC71
:10041800257827EAE770013055B1041B2946404684
:10042800C847301916F8015B002DF7D1BDE8F087F1
:10043800BDE8F087002A04DC2846BDE8F0870020E4
:10044800EBE7571EDCE783684268D0ED037A00EBE0
:1004580083010133934281ED040A836004BF0023C2
:10046800836000EB830393ED047A036870EE277AC8
:100478009A42C0ED037A77EEC77AC0ED037A0CDAB8
:10048800013307EE103AF8EEC76AB7EE007A87EE46
:10049800A60A036030EE070A704707EE102AB8EE86
:1004A800C77A87EE870A704790ED057A90ED004A83
:1004B800D0ED066AD0ED014AD0ED047A90ED035AEA
:1004C800D0ED025AA4EE007AB0EE406AB0EE470AC8
:1004D800B0EE667AA6EE247A67EEC07AA0EE457A88
:1004E800E6EE257A80ED057AC0ED067A7047D0ED04
:1004F800057A90ED013AD0ED003AD0ED064A90ED3C
:10050800024A90ED077A90ED035A90ED086AD0ED13
:10051800045AC0ED067AF0EE406A27EE830AC0ED71
:10052800056AA3EEA60A80ED087AA4EE240AA5EED1
:10053800470AA5EEC60A80ED070A7047D0ED007A93
:1005480090ED017A30EE670AE7EE007AB0EE670ABE
:10055800C0ED007A704770470A44914214D030B415
:100568000139551E41F2210211F8014F082380EA92
:10057800042004044CBF82EA40004000013B80B2E2
:10058800F7D18D42F0D130BC7047012380F8453057
:10059800704790F8203033B1012B03D14FF400633A
:1005A8008382704770474FF4806383827047037873
:1005B800407840EA032010FB01F04FF4807190FB73
:1005C800F1F000F30F0000B27047704770474378AE
:1005D800007840EA032010FB01F04FF4807190FB93
:1005E800F1F000F30F0000B270472DE9F74F6A4CA5
:1005F800DFF8A8E123880091DEF80010B4F9048040
:10060800C3EB21125B00C3EBE103B4F902105243C0
:100618005943131308FB03F84FEAA83808EBE12104
:1006280001EB8102B1F5FA3802F180024FEAE17973
:100638004FEA222349F1FF39B4F908200193A8FBB6
:1006480008AB08FB09F30BEB430BA161D31702FBC3
:1006580009F108FB0311A2FB08230B441F0316032F
:1006680047EA1257B4F90A2002FB0BF1D3170AFB29
:1006780003130546A2FB0A011944020A42EA016271
:1006880092194FEA2123E6887B41003243F5004363
:10069800A2FB060106FB03114A10CB1752EA03011D
:1006A8006FD0B4F91060B4F90E00F71706FB0BF120
:1006B8000AFB0711A6FB0AAB8B4400FB09F6C1171E
:1006C80008FB0161A0FB08898944DEF804104FEAA1
:1006D8004846C1F5801E4FEA494747EAD8371AEB22
:1006E800060AB4F90C8076464BEB070BF717002681
:1006F8004FEACE70F90716EB0A064FEAC80741EA37
:100708005E0147EB0B0740F6354E861B61EB07078A
:10071800A6FB0E010EFB071132F0F4FDB4F916200A
:100728004E13470B47EAC14702FB06FED31707FBE8
:1007380003EEA2FB07237344564307FB0366A2FBA1
:1007480007233344560E46EAC3163218B4F9146028
:100758004FEA636747EB01037143F71700FB07177D
:10076800A6FB00013944C60C46EA413692194FEA05
:10077800E147B4F912607B41100A40EA0360320194
:1007880012180DB1120A2A60009B13B11A46019B78
:10079800136003B0BDE8F08FAC43002000230020B5
:1007A80070472DE9F041324E324F74893B89B6F9D2
:1007B8001420B6F902E0B6F90E80B6F920C01B1B6A
:1007C80034895C43E313B6F912401A44E4020A255B
:1007D80094FBF2F41C44B6F90430F4616543A4F5C3
:1007E8007A6404FB04F204FB0EFE5C43B6F90C3099
:1007F800121302FB08F85A4312144FEAEE2E02EBCA
:1008080064340EEBE828B6F900E0F388FE68023499
:10081800A41008EB8E0804F5004408FA0CF86343AA
:100828004CF2503208F10208DC0BA6EBA80642FA9B
:100838000CF3734353BF5B00B3FBF4F35B00B3FBF0
:10084800F4F31A1202FB02F440F6DE3262430A4C59
:1008580012145C4302EB2442083502F6CF622D11D4
:1008680003EB221300B1036001B10D60BDE8F08114
:10087800744300200023002043E3FFFF2DE9F04FDD
:10088800654B664EB3F80AC03469B3F8048087B084
:100898004FEA0C2A05901889B4EB0A0A4FF00002B7
:1008A8004FF0000565EB020BA0FB0A4500FB0B555A
:1008B800E00940EA45604FEA084407198E46D8889F
:1008C8004FEAE51141EB0208A0FB0A45CDE90278A1
:1008D800B3F8028000FB0B55200A40EA05604FEA96
:1008E800C83410EB04084FEA252141EB02099A8924
:1008F800A2FB0A0102FB0B11C20D42EA412212F5CA
:10090800FA604FEAE15343F10001B0F5FA6FCDE91F
:10091800000171F10001B4465EDA0524A2FB04016E
:1009280004FB031100FB03F402FB0144DDE9026749
:10093800A0FB020121444D104FEA3004361B4FEA58
:10094800900444EA817467EB05078D10B8EB04083E
:1009580069EB0509DDE9004531484FF0FF31844274
:1009680075EB0101CDE9026723DA40F6AC501218A5
:100978004FF000014B4102FB03F1A2FB022303EB02
:100988004103D900D000101A41EA527163EB01010A
:10099800341847EB0105CDE902450B24A2FB0401FD
:1009A80004FB031149104FEA3000B8EB000869EB6B
:1009B80001090AFB0BF3DDE90001AAFB0AAB0BEB0B
:1009C800430B4FEADA7242EA4B02801A4FEAEB73A2
:1009D80061EB0301CDE90001DCF81410A1FB082349
:1009E80001FB0933540D5D1544EAC324DDE90223F4
:1009F800A21A65EB03031D46D30B059A43EA454348
:100A080002B11360BEF1000F02D0009BCEF8003097
:100A180007B0BDE8F08F00BF9843002000230020F6
:100A280024FAFFFF37B504466A460D460C30032109
:100A380023F0A8FF024690B1B4F91A106846FFF7F0
:100A4800B6FD2880B4F91E100DF10200FFF7AFFDC6
:100A5800A880B4F91C1001A8FFF7A9FD688010460A
:100A680003B030BD07B5F7216A4623F08BFF9DF828
:100A780001309DF800100C4A1B0143EA01339DF830
:100A8800021043EA111353609DF804309DF80310D7
:100A98001B0143EA01339DF8051043EA1113136063
:100AA80003B05DF804FB00BF0023002070B40468A5
:100AB800037B2268022101FA03F31A4213D0426928
:100AC8000A495C2000FB02124FF6FE7650685289F4
:100AD800C5680068296831402960C168D24392B26C
:100AE8000A40C260636070BC704700BFE0710020BC
:100AF80030B40A4B1D7875B1094B002003EBC505CE
:100B08001A6899885062D4682143D160083323F861
:100B1800040CAB42F4D130BC704700BFC074002055
:100B2800C474002010B40268047B11680223A34037
:100B3800194209D00649406800240C7001684FF634
:100B4800FE742140016053605DF8044B704700BF9C
:100B580007460020002326220360027027228270A5
:100B6800012243600271837170472DE9F3410569E1
:100B780006460F467DBBD0F80080C8F30A0323B3AE
:100B88000023D6F80080019324F0FAFE042819D136
:100B9800214C236943F001032361BBB2A8F800305C
:100BA80024F0EEFE04282ED108F102030193019BE4
:100BB8003F0C1F8024F0E4FE2369042823F001037E
:100BC800236125D06FF0010505E024F0D9FE042843
:100BD80005D04FF0FF35284602B0BDE8F0810E4C35
:100BE800236943F002032361C4F81480236943F0A6
:100BF8004003236124F0C4FE2369042823F0020380
:100C08002361BDD0E5E7236923F001032361D9E718
:100C1800336804333360DEE700200240F8B5044649
:100C28000D468E180027B54201D12069F8BDE3684A
:100C3800591CE160234415F8012B1A720429F2D1DA
:100C4800A1682046FFF791FFE7602061EBE7024BC0
:100C5800186805F009B800BF7023002010B490E8A8
:100C68000600047B40690223A3404B6013685DF8CB
:100C7800044B4FF6FE710B40136004F085BF2DE95D
:100C8800F0410B4E346873691C400FD0DFF82480A4
:100C98000127B4FA84F3C3F11F0307FA03F558F8E0
:100CA800230003689847AC437561F2D1BDE8F08131
:100CB80000040140302300202DE9F0410B4E346838
:100CC80073691C400FD0DFF828800127B4FA84F339
:100CD800C3F11F0307FA03F558F823000368984780
:100CE800AC437561F2D1BDE8F08100BF000401405A
:100CF800302300202DE9F0410B4E346873691C4005
:100D08000FD0DFF828800127B4FA84F3C3F11F035A
:100D180007FA03F558F8230003689847AC43756150
:100D2800F2D1BDE8F08100BF00040140302300206B
:100D38002DE9F0410B4E346873691C400FD0DFF881
:100D480028800127B4FA84F3C3F11F0307FA03F5D7
:100D580058F8230003689847AC437561F2D1BDE8A1
:100D6800F08100BF00040140302300202DE9F0414C
:100D78000B4E346873691C400FD0DFF828800127B8
:100D8800B4FA84F3C3F11F0307FA03F558F82300F4
:100D980003689847AC437561F2D1BDE8F08100BFA4
:100DA80000040140302300202DE9F0410B4E346847
:100DB80073691C400FD0DFF828800127B4FA84F348
:100DC800C3F11F0307FA03F558F82300036898478F
:100DD800AC437561F2D1BDE8F08100BF0004014069
:100DE80030230020002878D0F0B58488B4FA84F441
:100DF800C4F11F04651C83B062D0E6B206F0FC059E
:100E080005F1804505F5803506F00306AF68DFF883
:100E1800DCC000684CF82410B6004FF00F0E0EFA34
:100E280006FE27EA0E07AF60D5F808C0DFF8C0E075
:100E38002A4FC0F38721B1400120A04041EA0C01AC
:100E4800A960CEF800003D68254EDFF8A8C0C14370
:100E58000D403D6035680D4035603D68214E0543C5
:100E68003D60DCF800500D40CCF800505EF8085C9E
:100E780034442940102B4EF8081C94F86040AEF119
:100E8800080E1FD003F1804303F58233196801432C
:100E98001960154B2344197E914211DD26449511A2
:100EA80096F870108DF804100024012101A81A7614
:100EB8008DF805508DF806408DF8071028F010FCC5
:100EC80003B0F0BDDCF800300343CCF80030DEF8A6
:100ED80000100143CEF80010DBE770470004014022
:100EE80004040140784B030800230020302300202D
:100EF80014040140080401400B490C4A0C4808B589
:100F08008B6943F001038B61136843F480531360CA
:100F18000021402233F0BDFD064B4FF0FF329A61AD
:100F2800C3F81B2008BD00BF0010024000000140AC
:100F3800302300200023002003685B6A18470368F9
:100F48001B6A184770B44E1C0568C2728672AC6979
:100F5800A44670BC60472DE9F041044618460D468A
:100F68001646984631F004FD2768E6722844A072B8
:100F780029467D69434632462046AC46BDE8F041E5
:100F88006047036810B504461B68984723682046E5
:100F98009B689847A37B0133A37310BD03681B6943
:100FA800184710B5036804469B689847FF23012239
:100FB8006373227310BD074B984202D04FF0FF3085
:100FC8007047054A538B01339BB25383508B80B2D1
:100FD800704700BF00380040B057002038B583681C
:100FE8000446154601F07F0113B11A689B881385E2
:100FF800606840F2E93300E07BB30289013B12F0FC
:10100800020F9BB2F8D0017340F2E93300E023B33A
:101018000289013B12F0010F9BB2F8D0037B606894
:1010280040F2E93300E0DBB10289013B12F0020F24
:101038009BB2F8D0057340F2E93300E083B102892E
:10104800013B12F0010F9BB2F8D0037BA36813B1E8
:101058001A689B889361012038BDFFF7ACFFDEE773
:10106800FFF7A9FFF2E7F8B584894FF6FF764FF44A
:101078007A742BB311B30F78013101E0B44217D061
:101088000589013CAD07A4B2F8D507734FF47A740B
:1010980002E0BCB2B4420BD00589ED0704F1FF377A
:1010A800F7D5057BEDB20AB115700132013BE0E7D7
:1010B800FFF781FF003018BF0120F8BDFF27DFE7E9
:1010C8000120F8BD427A02B9704710B5044603689A
:1010D800406804F10A0198470023637210BD437AFF
:1010E8005A1C0344D2B242729972037A934200D8CE
:1010F80002B9704710B504460368406804F10A0154
:1011080098470023637210BD98B10B4B012210B4AD
:1011180002FA01F103F1750402E00333A34209D096
:101128001A788242F9D15A780A42F6D001205DF83D
:10113800044B70470020FAE7F04B030830B40A4D1F
:10114800002305F1780401E0272B0AD003EB4302C2
:101158000133A15C8142F7D12A4430BC92F87A006D
:101168007047002030BC7047784B030870B544883E
:1011780006460D46C4F30B0422460021284633F0E8
:1011880088FC3369094A934209D3094A934206D233
:10119800224628461946BDE8704032F0E7BA23B126
:1011A80021462846BDE87040184770BDD8BB0308E3
:1011B800C4BC0308064B07498B4202D300231846D8
:1011C80070471A88C2F30B029042F8D01433F3E741
:1011D80050B70308D8BB0308024A136823EA000083
:1011E80010607047E03D0020F8B5174D2B78A52B0F
:1011F80028D16B78BE2B25D1022229464FF6FF70E5
:10120800FFF7AAF9114FAC1C22884AB1A618BE42B2
:1012180018D2052A16D92146FFF79EF93446F3E776
:1012280021460222FFF798F90222A118FFF794F944
:101238000634074B641B1C8041F60F53C31A5842EF
:101248005841F8BD0020F8BD00F00308000004086C
:10125800EE3500202DE9F04FDFF848914C4F8BB068
:101268000326A7EB09071822002104A833F011FC74
:10127800484BCDF8109005971A69120604D5464ACE
:101288005A6002F188325A6001228DF824203422F3
:10129800DA60424B424C1B88ADF8003002226946A6
:1012A80004A8FFF7BBFC022269464FF6FF70FFF760
:1012B80053F9DFF8F4A080464FF0000B544536D3BD
:1012C8000AAC002524F8245D0222214604A8FFF771
:1012D800A5FC022221464046FFF73EF940BAC0432A
:1012E800ADF80800022202A904A8FFF797FC0798A6
:1012F80060B106ABC0F104022946184433F0C9FBBB
:10130800069904A8FFF731FC079508909DF824304A
:10131800089A23B11F490B6943F080030B61013E12
:101328002DD0002A9FD1FFF75FFF50B32CE06588CE
:101338008DF80DB0C5F30B05AB1DADF8083023884B
:10134800C3F30B02ADF80A201B0B062202A904A85E
:101358008DF80C30FFF762FC062202A94046FFF721
:10136800FBF8616880462A4604A8FFF757FC6168C5
:1013780040462A46FFF7F0F8143480469EE7002AD4
:10138800D1D0052002F046FD0BB0BDE8F08F00BFBC
:10139800000004080020024023016745654C03084B
:1013A80050B7030800F00308D8BB03080378202BC4
:1013B800024600F10100F9D0092BF7D02D2B2CD0D3
:1013C8002B2B03BF5378B7EE000A0246B7EE000A8C
:1013D800A3F13001C8B209289FED467A10D8F2EE81
:1013E800046A07EE901AF8EEE77A12F8013FE7EE82
:1013F800267AA3F13001C8B20928B0EE677AF0D98D
:101408002E2B4CD003F0DF03452B0BD0F7EE007AE0
:1014180067EE276A20EE260A70475378BFEE000A67
:101428000246D5E710B451782D2959D02B290ABF87
:101438009178501C901C0024A1F13003092B53D83B
:10144800002303EB830301EB430310F8011FA1F111
:101458003002092AA3F13003F3D9B3F59A7F28BFE4
:101468004FF49A73072B42D9DFED236A1A46F7EE39
:10147800007A083A072A67EEA67AFAD803F0070333
:101488002BB1F2EE046A013B67EEA67AFBD124B3D6
:10149800C7EE276A5DF8044B20EE260A704753789A
:1014A800A3F13001C8B2092802F10102AAD8F2EE6C
:1014B800046AF0EE665A07EE901AF8EEE77A12F828
:1014C800013F87EEA66AA3F13001C8B2092866EE8B
:1014D800A56A37EE067AEED994E767EE276AD9E768
:1014E800901C91780124A7E7F7EE007ACFE7F7EE92
:1014F800007AC5E70000000020BCBE4CB5EEC00A6B
:10150800DFED317AF1EE10FACCBF30EE270A30EE7B
:10151800670ADFED2E7A20EE270A30B5FDEEC07A95
:1015280087B017EE904A054684EAE470002303A9C1
:10153800A0EBE47001930093029327F04BFB002C7F
:10154800ACBF20232D2303A88DF8003031F010FA0A
:10155800012803A924D002282DD0032805BF302351
:10156800684668468DF8013033F09BFA684631F0DA
:10157800FFF90338C4B222466946284633F0C8FA50
:1015880000232B55284631F0F3F92E22431C2A5408
:101598000DEB0401E81833F0A1FA284607B030BD76
:1015A800302368468DF801308DF802308DF803300D
:1015B80033F077FADAE7302368468DF801308DF892
:1015C800023033F06EFAD1E76F12033A00007A4422
:1015D8002DE9F041064615460846B6FBF2F43CB93B
:1015E80005FB1464124B1B5D00F8013BBDE8F0815C
:1015F800B4FBF2F767B90E4B05FB174705FB1464FC
:10160800DA5D00F8012B1B5D00F8013BBDE8F081B5
:10161800B7FBF2F8B8F1000F02D04046FFF7D8FF49
:1016280005FB1878024B13F8082000F8012BE3E7B4
:10163800887D0308104B2DE93048D3E9004554EA6A
:1016480005020BD1034601220020187158719871C8
:101658009A70DA7018801881BDE83088074B1A68CC
:1016680014EB020B45F1000C5A466346FEF7F4FDF5
:101678000120BDE8308800BFD82400201858002079
:10168800F0B402888578154FC37804794179A2F2BD
:10169800B27202F0030606EB4606013D05EB86052D
:1016A800013B37F815608579008940F2B5579208F3
:1016B80007FB0232931903EB430304EBC303C3EBA9
:1016C800031301EB8303C3EB031305EB830300212F
:1016D8004FF47A72C2FB0301F0BC7047784B0308E1
:1016E800FAB170B48E18044603E0101A14D1B1424E
:1016F80014D014F8012BA2F14103192B11F8013B66
:10170800A3F1410598BF2032192D03F12000ECD92F
:10171800D01A01D1002BEAD170BC7047002070BCF0
:101728007047104670474FF0FF32FFF7D9BFA0F15E
:101738006103192B98BF20387047A0F14103192B7A
:1017480098BF20307047202805D0093804288CBF5E
:1017580000200120704701207047613819288CBF8C
:10176800002001207047413819288CBF0020012033
:101778007047303809288CBF002001207047A0F13D
:101788003003092B07D920F02000413819288CBFD5
:101798000020012070470120704730B402681146CC
:1017A800531C036011F8024B0160D31C517803608D
:1017B8009378151D05601B0443EA0123D078234361
:1017C80043EA006030BC70470368591C1A46016040
:1017D80012F8021B0260587841EA0020704703683B
:1017E8005A1C02601878704738B5044600681546D8
:1017F80031F0BCFF22682A44226038BD036810B467
:101808000A0A5C1C04601A7003685A1C026019708A
:101818005DF8044B704703685A1C026010B41970D5
:1018280003680A0A5C1C04601A7003680A0C5C1CD2
:1018380004601A700368090E5A1C026019705DF87A
:10184800044B704703685A1C026019700368090A40
:101858005A1C0260197070472DE9F047002488B0BF
:1018680080460F461E46A14605AD531C03931178CA
:1018780039B3252933D1931CCDF8109003935078B0
:1018880030284ED04FF0000AA0F13003DBB2092B0C
:1018980042D96C2819D0642800F0938024D82528D0
:1018A8001CD063D9582876D063281BD1317840469C
:1018B800B847039A531C039311780436013400295E
:1018C800D7D1204608B0BDE8F087039B5A1C039285
:1018D8001B78642B7CD02AD8252B54D1252140464F
:1018E8000134B847039AC0E7732833D044D9752820
:1018F8004FD106F1040E30682B4600220A217646A5
:10190800FEF772FC049A0095534639464046FEF7A6
:101918005CFD039A0444A8E704AA03A924F046F846
:10192800B7E7D31C039390784FF0010AACE7732B09
:1019380010D05BD9752B3AD0782B96D1A3F15802E9
:10194800B2FA82F2306852092B4610210436FEF7AB
:101958004BFCD7E73368049A009339460023404686
:10196800FEF733FD04360444039A7EE70028B9D114
:10197800204608B0BDE8F0876E28B3D1039A3368D3
:1019880004361C6071E72AD9582BD7D0632B8DD029
:101998006BE77828A6D1A0F15802B2FA82F2306833
:1019A80052092B461021FEF71FFC0436AAE706F160
:1019B800040E30682B4600220A217646FEF714FCF6
:1019C800A0E7331D306829461E46FEF7E0FB99E77D
:1019D800331D306829461E46FEF7D9FB92E7002BD7
:1019E8007FF443AF204608B0BDE8F0876E2BC6D021
:1019F8003BE70EB400B584B005AB019053F8042B57
:101A08000649039301A8FFF727FF019B00221A70DC
:101A180004B05DF804EB03B0704700BFC9030008C9
:101A28002DE9F04707468CB01E469246002A6AD137
:101A3800154614460A8840F2B1739A423AD98B780F
:101A4800581E0B2836D891F803E00EF1FF301E28F7
:101A580030D891F804C0BCF1170F2BD891F8059035
:101A6800B9F13B0F26D888793B2823D8B1F80880EC
:101A7800B8F57A7F1ED24FF00108002E34D10989BB
:101A88000491002CB4BF2D212B21002CB8BF644237
:101A9800039005910795CDF80890CDF804C0CDF8CE
:101AA80000E0384606942F49FFF7A3FF40460CB0E4
:101AB800BDE8F0870023012118468E46ADF8243092
:101AC8008DF828308DF829308DF82A30ADF82C3073
:101AD80099469C461A4698468DF826108DF8271088
:101AE8000B4609A9002ECAD00390CDF80890CDF86E
:101AF80004C0CDF800E038461B49FFF77AFF40469E
:101B08000CB0BDE8F087194C84FB0234A318D41735
:101B1800C4EB6314C4EB0415A2EB85052DB2002DAC
:101B28000846B8BF6D42FFF7ABFD4FF47A72002349
:101B38008046894631F0E6FB3C230AFB030A4FF452
:101B48007A7200234046494631F0DCFB4FF47A7143
:101B580092B20023C1FB0A2309A8FEF77DFB24B239
:101B680009A967E7D07D0308B07D030889888888BC
:101B78000FB430B583B006AB0A490B4853F8042BB1
:101B8800096800680193FFF767FE084C054620685E
:101B980004F05AF80028FAD0284603B0BDE83040CF
:101BA80004B07047483200204C32002070230020D7
:101BB800DFED2B7AB4EEE70AF1EE10FA4ADDDFED3D
:101BC800296A9FED297A01E0B0EE670AB4EEC70AE8
:101BD800F1EE10FA70EE667AF6DC9FED247AF4EEF8
:101BE800C77AF1EE10FA38D5DFED1E6A9FED207A3C
:101BF80001E0F0EE407AF4EEC77AF1EE10FA37EE33
:101C0800A60AF6D4DFED1B7AB4EEE70AF1EE10FA75
:101C180014DDDFED137A37EEC00A60EE006A9FED3F
:101C2800166A9FED167ADFED167AA6EE867A20EE12
:101C3800266AE6EE877AA6EE270A7047DFED117A64
:101C4800B4EEE70AF1EE10FA44BFDFED087A37EE9A
:101C5800C00AE2E7F0EE407ABFE7B0EE670AD1E7E4
:101C6800DB0F4940DB0FC940E4CB1641DB0F49C00D
:101C7800E4CB16C1DB0FC93F92E741B99730083C66
:101C880015A82ABEDB0FC9BF09B909E0194690FBA0
:101C9800F1F301FB13030846002BF7D10846704700
:101CA8000146FBE79FED317A70EE077AFDEEE76AB1
:101CB80016EE903A2033402B02D99FED2D0A70473B
:101CC800B4EEC70AF1EE10FA0FDDB0EE677A9FEDB9
:101CD800296ADFED296A01E0B0EE677AB4EEE67AA8
:101CE800F1EE10FA77EEC67AF6DC9FED247AF4EE80
:101CF800C77AF1EE10FA0FD5B0EE677A9FED1D6A3C
:101D0800DFED1F6A01E0B0EE677AB4EEE67AF1EE35
:101D180010FA77EE867AF6D49FED147AF4EEC77A45
:101D2800F1EE10FA1DDC9FED177AF4EEC77AF1EEAA
:101D380010FA44BF9FED117A77EE677A27EEA76A0B
:101D4800DFED115ADFED116A9FED117AE6EE256A93
:101D580067EE865AA6EE267AE5EE877AB0EE670A2F
:101D680070479FED0C7A77EE677AE7E7DB0FC93F9C
:101D780000000000DB0FC940E4CB1641DB0F49C06F
:101D8800E4CB16C1DB0FC9BF92E741B99730083CD5
:101D980015A82ABEDB0F494007EE901AF8EE677ABD
:101DA8009FED837A27EE800A20EE070AFDEEC07ABF
:101DB80017EE903A2033402B00F28C80DFED7D7ACD
:101DC800B4EEE70AF1EE10FA40F3E880B0EE407A9C
:101DD8009FED796ADFED796A01E0B0EE677AB4EEDB
:101DE800E67AF1EE10FA77EE467AF6DC9FED747A31
:101DF800F4EEC77AF1EE10FA40F1CD809FED6E6AED
:101E0800DFED706A01E0F0EE477AF4EEE67AF1EE83
:101E180010FA37EE867AF6D4DFED6B7AB4EEE77A0D
:101E2800F1EE10FA51DCDFED697AB4EEE77AF1EE03
:101E380010FA44BFDFED627A37EEC77A27EE076AF9
:101E4800DFED635ADFED637ADFED636A9FED635A76
:101E5800E6EE257A67EE065AE6EE276AF7EE007A8E
:101E6800A5EEA67AF0EE675AE7EE055AE7EE457A50
:101E780087EEA55ADFED547A30EE277AFDEEC76A71
:101E880016EE903A2033402B29D99FED557AF6EE7D
:101E9800006AB7EE006AF7EE004AC4EEA57A00239E
:101EA800836143610362C36180ED045A67EEA66AE9
:101EB80027EE866A27EE877AC0ED006AC0ED026ACF
:101EC80080ED016A80ED037A7047DFED3A7A37EEEC
:101ED800C77AB3E7B7EE005AF0EE455ACAE7B4EE50
:101EE800E70AF1EE10FA5FDD9FED336ADFED336A42
:101EF80001E0B0EE677AB4EEE67AF1EE10FA77EE2A
:101F0800467AF6DC9FED2E7AF4EEC77AF1EE10FAF7
:101F180047D59FED296ADFED2B6A01E0F0EE477A9D
:101F2800F4EEE67AF1EE10FA37EE867AF6D4DFEDC3
:101F3800267AB4EEE77AF1EE10FA27DCDFED237AA1
:101F4800B4EEE77AF1EE10FA44BFDFED1D7A37EE12
:101F5800C77A27EE076ADFED1E4ADFED1E6ADFED5E
:101F68001E7AE6EE246A67EE064AE6EE267AB7EEB1
:101F7800006AA4EEA77AF6EE006A36EE476AF8EE33
:101F8800007A27EE277A66EE266A84E7DFED097A7B
:101F980037EEC77ADDE7B0EE677A3DE7F0EE407AD4
:101FA80024E7B0EE677AC2E7F0EE477AAAE700BF07
:101FB80027D4D236DB0F4940DB0FC940E4CB1641AA
:101FC800DB0F49C0E4CB16C1DB0FC93FDB0FC9BF2C
:101FD80092E741B99730083C15A82ABEF304353F6B
:101FE8000000008070B406688E4217D90139751E4A
:101FF800002311F8014F0822634013F0800F4FEAC5
:10200800430318BF83F0D503013ADBB2F5D18D4203
:10201800EFD1721C0260337070BC70470023F8E780
:1020280010B44C09012250F8243001F01F0102FAC3
:1020380001F10B4340F824305DF8044B70474B091D
:1020480001F01F0150F82320012303FA01F1114286
:1020580014BF184600207047074A084B10781B78B1
:10206800074A834296BFC31AC3F18003002012684F
:1020780018441044704700BFBC6500203865002034
:102088002C430020064A074B10781B7883428ABFEE
:10209800C3F18003C01AC018C0F17F00704700BFA9
:1020A800BC6500203865002030B5134C237883B018
:1020B8001BB90120237003B030BD1049052200234D
:1020C8000D688DF804208DF8053000BFA86804F06D
:1020D800EFF96A4601A902236868FEF7C4FFA868F9
:1020E80004F0ECF900BF9DF8013003F0010383F020
:1020F8000100237003B030BDA7560020945600207D
:1021080070B5064C0646256803E023685B1BB3429E
:1021180003D8FFF7C9FF0028F7D070BD1858002072
:10212800F0B51F4C83B0277800234FF0030E0093BF
:102138000E4615468DF804308DF800E06FB3030E97
:102148008DF801300DF10203010C020A9870197024
:1021580006205A70FFF7D4FFE8B100BF114F3B6863
:10216800986804F0A5F923783A68002B14BF052372
:102178000423694650680022FEF775FF3B68324623
:10218800002158682B46FEF76EFF3B68986804F0FC
:1021980095F900BF284603B0F0BD0DF10103D3E760
:1021A800A65600209456002038B505460C4600BFB8
:1021B800806804F07DF9686840F2E93300E0B3B163
:1021C8000289013B12F0020F9BB2F8D0047340F26F
:1021D800E93300E05BB10289013B12F0010F9BB2C9
:1021E800F8D0037BA86804F069F900BF38BDFEF792
:1021F800E2FEA86804F062F900BF38BD2DE9F04F8F
:1022080089B0B2F1000A02900491039340F3C580AB
:102218000B46002201EB8A0153F8040B8B4202445F
:10222800FAD1039B0592002B00F0AF80059B002B91
:102238007CD05E4B059A1B68DFF888910092009964
:10224800DAB25118B1F5807F8CBFC2F58072009A5E
:102258000192574A92689A4240F28280554A117810
:10226800002206928DF81C2002228DF818200029E1
:1022780060D01A0E8DF819200DF11A021C0C190ADB
:102288009370147051700620FFF73AFF0621D9F8B1
:102298000000FFF789FF484A0123137000BFD9F8EF
:1022A8000030986804F004F9424BD9F800201B78F4
:1022B8005068002B06A90CBF042305230022FEF753
:1022C800D2FE0024049D029E019FA34629684FEA7E
:1022D800840800220B46013471B1B9422DD2D9F8D5
:1022E800000031684068FEF7BEFE2A683368134470
:1022F8003360BF1AC5F800B0A24505F1040506F120
:102308000406E3D1D9F80030986804F0D7F800BF84
:10231800264B019900981B68421A0092234A0B44E5
:102328001360039A4AB3009A002A88D1059809B025
:10233800BDE8F08F0DF11902A0E7029CD9F8003032
:1023480054F80810586800223B46FEF78CFE54F8F3
:1023580008202B683A44DF1B44F808202F60D1E797
:102368000598009C1549164A001B059005980023FE
:102378000B70137009B0BDE8F08F059B009A9B1A8B
:102388000593059809B0BDE8F08FFFF78DFE00288A
:102398007FF44CAF039B0593C8E7039C1CB9FFF778
:1023A80083FE0594C2E700230593BFE72C43002072
:1023B800FC190020A6560020A7560020BC65002066
:1023C800386500209456002070B5104D104E2B78BB
:1023D80031788B4284B016D00E4A03921A44029286
:1023E8008CBF0C46CA1A04A98CBFC3F18002002412
:1023F800012341F8102D02A802220194FFF7FEFEE6
:10240800002333702B7004B070BD00BF3865002006
:10241800BC6500203C650020F0B5124B9D6885B076
:102428000DB905B0F0BDED0A14D0002704AE7C1933
:102438006410E00210226946FFF772FE0F2809DDDA
:102448006B4653F8042B01320AD1B342F9D1254621
:10245800AF42ECDBFFF7B8FF034BED021D60E0E78E
:10246800671CF5E7FC1900202C43002070B5194CB7
:10247800194D23782978994284B027D0174A0392B6
:102488001A44029234BF0E46CA1A04A934BFC3F1D3
:1024980080020026002341F8102D02A8022201968E
:1024A800FFF7ACFE23781844C0B203062B7848BF68
:1024B80080F080008342207002D0002004B070BDFC
:1024C800002301202B70237004B070BD012004B0DC
:1024D80070BD00BF38650020BC6500203C65002049
:1024E80010B50C4C45F20820FFF70AFE20680621BB
:1024F800FFF75AFE084B20680122C7211A70FFF720
:1025080053FE06480649074A002303700B70136000
:1025180010BD00BF94560020A7560020BC650020BF
:10252800386500202C430020F0B55B4B5B4A97B020
:102538001968914200AF00F0A3805949594A002315
:102548004FF47000C1F888003B607B60136843F467
:102558008033136003E03B68B3F5A04F09D01368DC
:1025680003F400337B603B6801333B607B68002BDE
:10257800F1D04C4B1B6813F4003318BF01237B6068
:102588007B68012B52D0464C464B474AE260474A8B
:10259800596A11605A6A42F080725A625A6942F462
:1025A800FC025A610025032207F10801012341F6C4
:1025B800FF764FF09040FD60BE603A73BB732BF01E
:1025C80051FC4FF6FF7307F108013948BB602BF047
:1025D80049FC07F108013748374E2BF043FC07F157
:1025E800080136482BF03EFC07F1080134482BF06F
:1025F80039FC07F1080133482BF034FC07F10800D7
:102608002BF089FCBB683049304AA1FB03133049E1
:102618009B0CF0204FF0070E5C370B60566084F877
:1026280023009560C2F800E0BD46F0BD294A1D4B65
:10263800122111605A685A605A685A605A6842F4FE
:1026480080625A605A6822F47C125A605A6842F4CE
:10265800E8125A601A6842F080721A601A68920189
:10266800FCD559680F4A21F003015960596841F0B7
:1026780002015960536803F00C03082BFAD182E772
:1026880000221A6062B6144B1B6883F30888134B48
:102698001B689847FEE700BFFC9F0020EFBEADDE39
:1026A80000ED00E0001002400005FA05045B002080
:1026B80000040048000800483F190100000C0048C9
:1026C800001000480014004883DE1B4310E000E0BF
:1026D8001C5800200020024000D8FF1F04D8FF1F0C
:1026E80070B50F4C0F4DC0EBC00004EB8004686957
:1026F80026693043686182B09209667BA160002533
:10270800012101A863618DF804608DF805208DF81A
:1027180006508DF8071026F0E3FF02B070BD00BF29
:102728000C1A002000100240074BC0EBC00030B468
:1027380003EB8000054C056963692B4363610176EF
:10274800427630BC704700BF0C1A002000100240CF
:102758002DE9F04F5E4C54F8204083B0002C71D026
:10276800A66D984691465B4B72682265A16023600E
:1027780004F15E014FF4807304F5AF726161A261E8
:10278800E36023610746307E23F084F9F068A8B13E
:10279800514B00215A68904203F11C0300F09280CB
:1027A80001310C29F6D100207A1CD2B20C21FFF796
:1027B800BBFF236DF26862632433E364B068D8B169
:1027C800454B00215A68904203F11C0378D001312F
:1027D8000C29F7D100257A1CD2B20B212846FFF725
:1027E800A3FF2346F27E3D492846FFF779FF236D74
:1027F800B268A2632833A36494F85D0002F05CFC1D
:10280800054694F85C0002F057FC18F0080F824661
:1028180096F819B01AD0CDB118F0110F4FF00B037C
:1028280007F1010714BF4E213E21EF715A46AB71E3
:10283800284602F0A1F818F0010F45D0636B5BB38E
:10284800A36B4BB3204603B0BDE8F08F18F0010F1F
:102858000CBF4FF02E084FF04E0819F0020F09D0A8
:1028680045B10B227B1CAA71EB7128465A4641469A
:1028780002F082F819F0010FE0D0BAF1000FDDD0B4
:1028880001370C238AF807705A4641468AF8063001
:10289800504602F071F8D1E7337FB27E8DF80420FC
:1028A8009B090021012201A88DF805308DF806103A
:1028B8008DF8072026F014FF204603B0BDE8F08FFE
:1028C800CDB288E7C8B26FE7284603F0F1FDB5E757
:1028D80054320020684C03080C1A0020650C0008CC
:1028E80000B97047F0B595B0054623F08FFD6E4EE0
:1028F800C368026832600446002B00F0C380284693
:1029080002F0DAFB694B186218B1292200238271A0
:10291800C371227A664D2E2102F02EF8306802F03B
:10292800ABFD23F0B7F83068624A038823F001034F
:102938001B041B0C038014A91E232B8001270F23C3
:102948000025138021F84C7D2D230293ADF80C50FF
:10295800ADF80650ADF80E5023F006FDE379ADF85A
:10296800145060229907ADF816500695ADF81C5022
:10297800ADF81E50ADF82050ADF82250049200F189
:10298800838013F0010F14BF022200224FF48073DA
:10299800ADF81470ADF81C20ADF82030002304AA5F
:1029A80061793068069301F0D9FD3068617923F0C8
:1029B800BBFC3068436C43F40043436403889BB218
:1029C80043F080030380E3799B0768D56179026A45
:1029D80004238B4022EA03020262026A1343036261
:1029E8003268354F13889BB243F001031380207C73
:1029F80000222921FFF798FE3049207C002360221D
:102A0800FFF76EFEE068386026F0D6FD3868036888
:102A18004FF6FE721340036026F0CEFD09A826F09B
:102A28009DFD33686279264938680A913433134426
:102A3800099380221023002509A940F22A3E0E920C
:102A48000B934FF400724FF400530D9510951395A6
:102A580011950F921293ADF830E026F08DFD627952
:102A680033680C2A98BF1749D86898BF31F81250B4
:102A78003A6815490543DD601368012043F00203F5
:102A88001360087015B0F0BD13F0010F14BF0822D1
:102A98002A460423ADF81E20ADF816307EE7012241
:102AA800617926F0F5FB9BE78C5600200023002077
:102AB8008256002080560020885600202D0B0008E2
:102AC80060460020607C0308845600200348D0F844
:102AD8003C3113B100F59A70184770470C1A002062
:102AE8000348D0F8203113B100F58C7018477047AF
:102AF8000C1A00200348D0F804310BB1FC301847F9
:102B0800704700BF0C1A00200348D0F8E8300BB11A
:102B1800E0301847704700BF0C1A00200348D0F86F
:102B2800CC300BB1C4301847704700BF0C1A0020D6
:102B38000348D0F8B0300BB1A8301847704700BF31
:102B48000C1A00200348D0F894300BB18C30184789
:102B5800704700BF0C1A00200248836F0BB1703019
:102B6800184770470C1A00200248C36D0BB1543047
:102B7800184770470C1A00200248036C0BB1383014
:102B8800184770470C1A00200248436A0BB11C30E2
:102B9800184770470C1A00200248836803B1184789
:102BA800704700BF0C1A0020F0B53E4C059D00EBA5
:102BB800800004EB80046468002C71D03A4E490010
:102BC8004FF42040CFB27062A169090454D4606800
:102BD800DFF8E0E047F4903100EA0E0001434FF4DB
:102BE80020406160706203E0411E002848D008461A
:102BF800A1698907F8D54FF42040A262706203E00A
:102C0800421E00283CD01046A2695206F8D5274A31
:102C18006168DFF8A0E0706242EA0342174301EA04
:102C28000E0217436760C3B1013BDBB201332B448B
:102C3800A0694FF4204210F0040002F1FF3207D1DE
:102C4800511C26D0A06910F0040002F1FF32F7D021
:102C5800626A05F8012B9D42EAD14FF42040706268
:102C680002E0431E60B11846A3699B06F9D52023EC
:102C78007062E3610120F0BD411E08B10846A3E778
:102C88000B4A138801339BB24FF0FF3113807162F6
:102C9800F0BD074972620B8801339BB20B80F0BD0F
:102CA8002046F0BD885700200023002000240002A1
:102CB800EC350020009800FCF0B50E46017801299B
:102CC80085B004464BD002294FD11D46836846F093
:102CD800800113B118689B880385606840F2E93366
:102CE80001E0002B55D00689013B16F0020F9BB27C
:102CF800F7D0017340F2E93301E0002B49D0018994
:102D0800013B11F0010F9BB2F7D0037B60684FF0D5
:102D1800000C83894FF6FF764FF47A734FF0FF0E5D
:102D2800654502D126E0B34222D00189013B8F07D5
:102D38009BB2F8D580F80CE04FF47A7302E0BBB28E
:102D4800B34215D00189C90703F1FF37F7D5017BD5
:102D5800C9B20AB1117001320CF1010CE0E790F927
:102D68000400411C01D002280CDD002005B0F0BD94
:102D7800FEF721F9A3688BB11A689B88936101203B
:102D880005B0F0BD617900923246FFF70DFF05B03E
:102D9800F0BD0392FEF70FF9039AB7E70120E5E7C4
:102DA80007B5032301AAF621FFF786FF9DF8053032
:102DB8009DF804201B0243EA02439DF806201343B2
:102DC800054AB2F92020C2F10802D340034AD36071
:102DD80003B05DF804FB00BF74430020002300200B
:102DE80007B5022301AAF621FFF766FF9DF8042024
:102DF8009DF8053043EA0223024A138103B05DF8C7
:102E080004FB00BF0023002007B5032301AA00210B
:102E1800FFF752FF9DF805309DF804001B0243EAB6
:102E280000439DF80600184303B05DF804FB08B59D
:102E3800FFF7EAFF014B586108BD00BF00230020DF
:102E480008B5FFF7E1FF014B186108BD002300201A
:102E5800F0B5037C012B85B0044663D0022B67D103
:102E6800836913B11A689B881385606940F2E93356
:102E780001E0002B6CD00289013B12F0020F9BB2DB
:102E8800F7D0C323037340F2E93301E0002B5FD08E
:102E98000289013B12F0010F9BB2F7D0037B6069F6
:102EA8004FF0060E838902AE4FF47A734FF6FF7126
:102EB800FF2703E0013B9BB28B423CD00289950778
:102EC800F8D507734FF47A7302E0ABB28B4232D075
:102ED8000289D20703F1FF35F7D5027BD2B20EB1D2
:102EE80032700136BEF1010EE8D1A36913B11A6838
:102EF8009B8893619DF80C009DF808609DF8091067
:102F08009DF80A509DF80B209DF80D3041EA0621E6
:102F180043EA002342EA0522012021876287A3872A
:102F280005B0F0BD90F91400431C01D0022805DD5E
:102F3800002005B0F0BDFEF73EF8D6E702AB617D94
:102F4800009343220623FFF72FFE0028D2D1EFE794
:102F5800FEF731F8A3E7F0B5037A012B85B00446F4
:102F680063D0022B67D1036913B11A689B88138554
:102F7800E06840F2E93301E0002B6CD00289013BA4
:102F880012F0020F9BB2F7D0BB23037340F2E93370
:102F980001E0002B5FD00289013B12F0010F9BB2C8
:102FA800F7D0037BE0684FF0060E838902AE4FF43A
:102FB8007A734FF6FF71FF2703E0013B9BB28B4208
:102FC8003CD002899507F8D507734FF47A7302E06D
:102FD800ABB28B4232D00289D20703F1FF35F7D565
:102FE800027BD2B20EB132700136BEF1010EE8D1C9
:102FF800236913B11A689B8893619DF80C009DF8AA
:1030080008609DF809109DF80A509DF80B209DF85E
:103018000D3041EA062143EA002342EA0522012055
:10302800E1822283638305B0F0BD90F90C00431C54
:1030380001D0022805DD002005B0F0BDFDF7BBFF7B
:10304800D6E702AB617B00933B220623FFF7ACFD7A
:103058000028D2D1EFE7FDF7AEFFA3E7B0F1FF3FBD
:1030680056D0022854DCF0B4324C00EB800004EB5C
:1030780080004468002C5BD02F4E49004FF420405C
:10308800CDB27062A169090444D460682B4F45F041
:103098008071384041F4903101434FF42040616021
:1030A800706203E0411E002838D00846A1698F07E6
:1030B800F8D54FF42040A262706202E0421E68B365
:1030C8001046A2691106F9D562681C4945F00075D9
:1030D80045F480350A4015434FF42040656070621E
:1030E80002E0421ED0B11046A2699207F9D54FF40A
:1030F8002040A362706202E0431E78B11846A369BB
:103108009B06F9D520237062E3610120F0BC70476B
:1031180000207047411E08B10846B3E7084A1388E3
:1031280001339BB24FF0FF3113807162F0BC7047DE
:103138002046FBE78857002000230020009800FC69
:10314800EC35002070B40578012D07D0022D02D18E
:1031580070BCFDF743BF002070BC7047134670BCBD
:103168000A46417990F9040078E72DE9F04F4FF4C9
:10317800807385B043838383C38300F10C050446C1
:10318800322002F08FFB112200212846FFF7DAFFD8
:10319800602201212846FFF7D5FF642002F082FB58
:1031A80002A920460027FDF73DFC0123B946B84691
:1031B8003E460193012E14BF1122122200212846F7
:1031C800FFF7C0FF002E0CBF4FF0010B4FF0FF3B85
:1031D8004FF00A0A012202212846FFF7B3FF142004
:1031E80002F060FB02A92046FDF71CFCBDF90A208D
:1031F800BDF90C00BDF90810304B82420BFB029957
:10320800A8BF02468A42A8BF0A469A4201FB0B8819
:103218000BFB00774FDB012002F02AFDBAF1010A0F
:10322800D8D10136022EC5D1254B93FBF8F893FB74
:10323800F9F97022A3F58423002193FBF7F7A4F88A
:103248001A80A4F81C90E7832846FFF77BFF20220A
:1032580001212846FFF776FF002231462846FFF76E
:1032680071FF642002F01EFB019B23B94FF48073A9
:103278006383A383E383607EC8B101F01DFF054625
:1032880003F08AF998B11DB12223AB710023EB71C9
:10329800284622F079FC21460A4B41F8083F284687
:1032A8000823F022FDF79EFD284621F0DDFB0120D2
:1032B80005B0BDE8F08F00230193B2E701F0FFFFEE
:1032C80000D03B00D5050008F0B500F10C0585B02D
:1032D80004460F4601230DF1070202212846FFF795
:1032E800EBFC18B90026304605B0F0BD9DF8073054
:1032F800DB07F7D502AA0321284621F043FB012367
:103308000DF1070209212846FFF7D6FC06460028DA
:10331800E8D011220A212846FFF714FF9DF807304C
:1033280013F00C0FDED1B4F91A1002A8FDF74FF90B
:1033380040423880B4F91C100DF10A00FDF747F936
:1033480040427880B4F91E1003A8FDF740F94042C6
:10335800B880C8E737B500F10C04054600220A21F9
:103368002046FFF7EFFE142002F09CFA0F220A21F4
:103378002046FFF7E7FE0A2002F094FA01AA032389
:1033880010212046FFF798FC0A2002F08BFA9DF8DE
:10339800043080336B839DF805308033AB839DF810
:1033A80006308033EB8300220A212046FFF7CAFE4D
:1033B8000A2002F077FA0DF10302012302212046C8
:1033C800FFF77AFC01230DF1030209212046FFF7DC
:1033D80073FC11220A212046FFF7B4FE012003B036
:1033E80030BD3122F421ADE6044B93F82020920140
:1033F800343202F0FC02F421A4E600BF744300203A
:103408002E22F4219EE6012248219BE60122582122
:1034180098E62DE9F04F87B090F855300290002BD0
:1034280040F0C181029A137C1032012B104603929E
:1034380000F01682022B00F0B181BD4CBD4EDFF8C2
:10344800FC92BD48DFF8F8E24FF0640A4FF0100C28
:103458004FF47A75D9F80430C3F30803002B40F011
:10346800F380EFF31183002B40F0EE80216882682F
:1034780000BF23689942F9D1376805FB07F39B1A07
:10348800B3FBF7F305FB013101270191D9F80430AB
:10349800C3F30803002B40F09D80EFF31183002B4A
:1034A80040F098802368816800BF22689342F9D170
:1034B800D6F800B005FB0BF2521AB2FBFBF205FB83
:1034C8000323019A9B1AB3F57A7FDFD3BAF1010A75
:1034D800C0D1029D297C012900F0B981022900F0A0
:1034E8004981029B012993F8503000F04F8102294D
:1034F80000F03A81DFF844928F48DFF844E24FF059
:103508000F0A4FF0100C4FF47A75D9F80430C3F352
:103518000803002B40F0B480EFF31183002B40F038
:10352800AF802168826800BF23689942F9D1376863
:1035380005FB07F39B1AB3FBF7F305FB01310127E2
:103548000191D9F80430C3F30803002B5FD1EFF3DE
:103558001183002B5BD12368816800BF22689342E6
:10356800F9D1D6F800B005FB0BF2521AB2FBFBF208
:1035780005FB0323019A9B1AB3F57A7FE1D3BAF1CD
:10358800010AC2D1029C237C94F84E20012B00F042
:103598007081022B00F0D680012B00F0DB80022B1B
:1035A80000F0B280012B00F0B980022B00F0988067
:1035B800012B00F09F80022B7ED0012B00F086802B
:1035C800022B04D1039801223821FDF707FD07B02B
:1035D800BDE8F08FEFF311888CF3128881680368D7
:1035E800DB0344BFCEF8007081682368DEF8002052
:1035F8005FFA88F888F31188D6F800801A4405FB2A
:1036080008F35B1AB3FBF8F305FB023359E7EFF352
:1036180011888CF3128881680368DB0344BFCEF8F5
:10362800007081682368DEF800205FFA88F888F364
:103638001188D6F800801A4405FB08F35B1AB3FB1F
:10364800F8F305FB023395E7EFF311828CF3128848
:1036580087680368D90303D50123CEF8003087684B
:103668002368DEF80010D2B282F311883268194458
:1036780005FB02F3DB1BB3FBF2F305FB013103E7A8
:10368800EFF311828CF3128887680368D90303D596
:103698000123CEF8003087682368DEF80010D2B224
:1036A80082F311883268194405FB02F3DB1BB3FB74
:1036B800F2F305FB013142E71A4637210398FDF77B
:1036C8008DFC029B1B7C012B7FF47AAF0298382279
:1036D800417D90F91400FFF7C1FC07B0BDE8F08FF9
:1036E80018221C210398FDF779FC029B1B7C012BF7
:1036F8007FF461AF029C02233722617D94F91400A4
:10370800FFF7ACFC237C58E718221B210398FDF730
:1037180065FC029B1B7C012B7FF447AF029C18239E
:103728001C22617D94F91400FFF798FC237C3FE785
:10373800185800201C58002010E000E000ED00E0C0
:10374800145800201A210398FDF748FC237C012B0C
:103758007FF425AF029C18231B22617D94F9140085
:10376800FFF77CFC237C1DE71A4619210398FDF717
:1037780035FCBFE66B2103220398FDF72FFC297C5B
:10378800029B012993F850307FF4B1AE02981922B8
:10379800417D90F91400FFF761FCABE680226B21B4
:1037A800FDF71CFC49E61D09013D052D03F00F033B
:1037B80068D8414A32F8150040FA03F2D40761D5B7
:1037C800012404FA03F3013B18402FF0EBFD3B4BB7
:1037D8003B4A5B5D184412EBC00553D052F83000E9
:1037E800AE88038A33407FF41DAE00F13842354974
:1037F800EB71920A8A5C02F01F0352092021022A07
:1038080004FA03F3A97152D0032A4BD0012A44D0F9
:10381800002304A9059304962AF024FB02992A4B55
:1038280041F80C3F28460823F022FDF7DBFAAB8865
:10383800B3FA83F3C3F11F03581C3FF4F3AD01221D
:1038480002FA03F321490A6813430B60EAE5697D2C
:1038580095F9140003236B22FFF700FC297C40E64E
:1038680002988023417D90F914006B22FFF7F6FB44
:10387800E3E51346617D94F914001A22FFF7EEFB85
:10388800237C89E60299104B41F80C3FF02208236B
:103898000020FDF7A7FA0123D4E70D4A51690B432D
:1038A8005361B5E70A4AD1690B43D361B0E7084AC7
:1038B80091690B439361ABE73C7C0308487C0308A0
:1038C800B86B00207C7703089305000800040140CA
:1038D800001002401749184B184A194810B4D1F87B
:1038E800884044F47004C1F888401C6844F001041E
:1038F8001C605C6822405A601A6822F0847222F4C4
:1039080080321A601A6822F480221A605A6822F4F7
:10391800FE025A60DA6A22F00F02DA621A6B002499
:1039280010404FF0006218639C608A605DF8044B99
:10393800704700BF00ED00E0001002400CC07FF8A7
:10394800CCFC00FF38B50B4C23688BB15A68821A3F
:10395800002A054604DA0CE05A68AA1A002A07DB8E
:103968009A68226018461A6890472368002BF3D19A
:1039780038BD38BDE85A00200B4B002210B4027243
:1039880003F5A074032102E0072A09DC9979890765
:1039980002D51979815401329C4203F11403F3D101
:1039A8005DF8044B704700BF847703081023037049
:1039B800704700BF30B401230225142415212222A8
:1039C800057244704171C27003700371837030BC1A
:1039D800704700BF2C22022302704370704700BF5B
:1039E800436A8269D154436A0169826B01338B420D
:1039F80028BF00234362002A2FD0EFF31181502300
:103A080083F31288836B1A68D2072CD470B45E686B
:103A18006EB9456A826A954217D084691444DC609D
:103A28000ED9AA1A5A608562002280F854201A68B2
:103A380042F00102C9B21A6081F3118870BC704764
:103A48000469A21A5A608662EEE7012380F85430AE
:103A5800C9B281F3118870BC7047026D136843F0D6
:103A6800800313607047C9B281F31188704700BFA3
:103A7800426B10B462B1436CC2684469D11A013B0D
:103A8800615C5DF8044B08BF13464364C8B27047D5
:103A9800016A4369C4685B5C0131A14228BF1146D1
:103AA80001625DF8044BD8B2704700BF836B13B155
:103AB80090F854007047836A406A181AB0FA80F088
:103AC80040097047416A836A99420AD3CB1A816BCD
:103AD800026961B14968501E0B4483420AD2C01A78
:103AE800704702691144CB1A816B0029F2D1501E2C
:103AF800C01A704700207047436B43B1426C5B6843
:103B080093422FBF981AC0689B1AC0187047C269A1
:103B1800036A9A422FBFD01AC0688018C01A70472B
:103B28000A4B30B503F1140493F900205D78072A95
:103B3800C8BF143A811804330D7313F8025C855416
:103B480013F8012C0A76A342EED130BD904C03083D
:103B580003682DE9F041DF691FB13B46BDE8F0413C
:103B68001847002A164611DD04460D460E4400E0AB
:103B780023689B68204698470028F9D0236815F8E1
:103B8800011B1B6820469847AE42F1D1BDE8F08181
:103B980000232322027043708370C370704700BFF4
:103BA8002DE9F0470569C3681D4028D00F46064631
:103BB8004FF000484FF00009B5FA85F328FA03F2F0
:103BC800D2431B3B32611540042B16D8DFE803F0C3
:103BD8003129211903007B6A002B32D003F1FF3A07
:103BE8001FFA8AFAC7F824903C6A34B12368204641
:103BF800514698476468002CF8D1002DDCD1BDE807
:103C0800F0873868716B036889B29847002DD3D163
:103C1800F5E77868B16B036889B29847002DCBD176
:103C2800EDE7B868F16B036889B29847002DC3D1F6
:103C3800E5E7F868316C036889B29847002DBBD175
:103C4800DDE7F36A1FFA83FACEE700BF30B5044612
:103C5800006D61710368A26823F00103036087B0F7
:103C6800A379009213F004023DD04FF4805213F070
:103C78000203019244D102934FF48063002203931C
:103C880011F00103059237D1049308238D07694683
:103C980048BF049325F0F2FB6079236DA17900F009
:103CA8000202002A15BF4FF440324FF480324FF41D
:103CB8000034002410F0010F586808BF2246CC07D2
:103CC8004CBF024320EA02025A609A6809074CBFB7
:103CD80042F0080222F008029A601A6842F00102D3
:103CE8001A6007B030BD13F0020301920BD04FF4F5
:103CF800005513460295C1E7042304930C23C5E736
:103D08004FF40053B7E70293B8E700BF10B5044675
:103D1800006DA160036823F001030360A37986B0F6
:103D280013F00402009141D04FF4805213F00203C3
:103D3800019244D102934FF4806362790393D107CF
:103D48004FF000030493059345BF0423049308230D
:103D58000C236946920748BF049325F08FFB6079CE
:103D6800236DA17900F00202002A15BF4FF44032FA
:103D78004FF480324FF40034002410F0010F5868DB
:103D880008BF2246CC074CBF024320EA02025A6011
:103D98009A6809074CBF42F0080222F008029A60AC
:103DA8001A6842F001021A6006B010BD13F002034F
:103DB800019207D04FF4005113460291BDE74FF42A
:103DC8000053B7E70293B8E7022828BF022010B4CF
:103DD800084C094B207000EB8002C0EBC202074977
:103DE8005DF8044B013003EB4203C0B20B6014F0E2
:103DF80091BF00BF9B490020B03C0020B84F002075
:103E080008B524F08BF9FDF725FABDE8084024F041
:103E18006DB900BF2DE9F04F013085B0C3B20393EF
:103E28008E4D8F4F8F4C904E0A2302933220DFF82D
:103E3800409220F0E7FA4FF4FA7A4FF0100C4FF462
:103E48007A70D9F80430C3F30803002B40F0C88017
:103E5800EFF31183002B40F0C3802968A26800BFEC
:103E68002B689942F9D1D7F800E000FB0EF39B1AB2
:103E7800B3FBFEF300FB01314FF0010E0191D9F8BD
:103E88000430C3F30803002B40F08E80EFF3118356
:103E9800002B40F089802B68A16800BF2A689342F4
:103EA800F9D1D7F800B000FB0BF2521AB2FBFBF2C3
:103EB80000FB0323019A9B1AB3F57A7FDFD3BAF18B
:103EC800010ABED1039B002B40F0C4804FF47A7ADC
:103ED800DFF89C9150464FF0100CD9F80430C3F32A
:103EE8000803002B40F09980EFF31183002B40F07A
:103EF80094802968A26800BF2B689942F9D1D7F845
:103F080000E000FB0EF39B1AB3FBFEF300FB01314C
:103F18004FF0010E0191D9F80430C3F308033BBBFD
:103F2800EFF3118323BB2B68A16800BF2A68934273
:103F3800F9D1D7F800B000FB0BF2521AB2FBFBF232
:103F480000FB0323019A9B1AB3F57A7FE3D3BAF1F6
:103F5800010AC2D1029B013B02937FF467AF434938
:103F6800434B4448444A0860DA6005B0BDE8F08F26
:103F7800EFF311888CF31288A1682368DB0344BF30
:103F8800C6F800E0A1682B6832685FFA88F888F301
:103F98001188D7F800801A4400FB08F35B1AB3FBBA
:103FA800F8F300FB0233CDE7EFF311888CF31288A6
:103FB800A1682368DB0344BFC6F800E0A1682B684A
:103FC80032685FFA88F888F31188D7F800801A44B5
:103FD80000FB08F35B1AB3FBF8F300FB023369E755
:103FE800EFF311828CF31288D4F808E02368D90320
:103FF80003D501233360D4F808E02B683168D2B2C6
:1040080082F311883A68194400FB02F3A3EB0E030C
:10401800B3FBF2F300FB01312EE7EFF311828CF3CF
:104028001288D4F808E02368D90303D50123336044
:10403800D4F808E02B683168D2B282F311883A6864
:10404800194400FB02F3A3EB0E03B3FBF2F300FBEE
:1040580001315DE7184622F077FA37E71858002053
:104068001C58002010E000E014580020FC9F00209D
:1040780000ED00E0EFBEADDE0400FA0538B5434BB5
:104088005A899989914224BF00225A81198ADA896A
:10409800914224BF0022DA81DA788AB3072A2FD026
:1040A8003B493C4D91F85300012400210A282C700B
:1040B8009C70D9713DD00C2865D0DFED377A8ABB6A
:1040C800364C9FED370AA278002918BFF0EE407AE7
:1040D800062A04D8334901EB820191ED050A2179BA
:1040E80059B3013A032A4DD8F7EE007A87EE800AD1
:1040F8002FF012FD2388984228BF1846208038BD2B
:10410800D97921B198780428B8BF0420987020483C
:1041180090F853000A280CD00C28CED1DFED227A73
:10412800002ACDD0072ACBD00A282CD1DFED1F7A60
:10413800C6E70A20DFED1E7AC1E79B78154A07EE2D
:10414800103A1178B8EEC77A27EE277A07EE901A58
:10415800F8EEE77A67EE877AB4EEE70AF1EE10FA3E
:1041680010DDC0EE077AFDEEE77A17EE903A102BD5
:10417800A8BF1023012BB8BF0123DBB28B4238BF85
:104188000B46137038BDDFED0B7A99E7F06C002011
:10419800046D00208C6700206F120339B87100206D
:1041A8006F120338904C03080AD7A3390F506E3AA0
:1041B8005304E9386F12833A2DE9F047A44FA54E0E
:1041C80023F0ACFFBE421ED2DFF80483DFF804936D
:1041D8004446258862197DB14A450DD2052D0BD973
:1041E80033886188C3F30B03994200F0D6801446E4
:1041F80025886219002DEFD1716830461436FCF716
:10420800B5FFBE42E4D3944A1378A3F117010229FB
:104218000FD9924911F83300002840F0EA80D800FD
:104228000144497829B18E4911F83330002B00F048
:1042380008818C4B5A78022A40F2D58000228A499C
:104248005A701A788948022A016000F2C88002EB85
:104258008201874BC2EBC10203EB4203998C5A8C53
:10426800844C9142236001D300225A84824B9A786D
:10427800042A00F0DD8032B91A88B2F5F07F84BFD5
:104288004FF4F0721A807D4DFFF7F8FE2B687C4AD8
:104298001A40002A00F0D880D80700F1C4805904D9
:1042A80000F1BC801A0700F1B4809B0400F1AA80D9
:1042B80021F03AF910B9734813F092FD8020FCF709
:1042C8008BFF4FF40010FCF787FF4FF00070FCF7EE
:1042D80083FF4FF08060FCF77FFF2CF0A5F90021E9
:1042E8003022694830F0D5FB20681EF02FF8674B64
:1042F800276803F1500102E0043399426DD01A781F
:10430800002AF9D19C78D8788442F5D26049614B6B
:104318000D79614961480A70614E624C0460C82297
:10432800642111FB0521002259609A60DA601A6144
:104338005A619A61DA6183F8202083F82120376076
:1043480017F0A6FB584B9FED595A1B88584A9FED0A
:10435800596A5079584906EE903AF8EEE66A138899
:10436800C5EE265A07EE103A53881279C1ED005A65
:1043780007EE903AB8EEC77A504BF8EEE77A187223
:104388005A7227EE067A67EE867ABDE8F04783ED23
:10439800017AC3ED007A23F0A9BE63799B077FF405
:1043A80026AF716894F804A03046FCF7DFFE338826
:1043B800BAEB133F04D01436BE42FFF409AF22E72C
:1043C80073887068AA1FC3F30B039A4204F10601AD
:1043D800A8BF1A462FF0CAF9EDE7012296E7002296
:1043E8001A70234B3AE7204902EB420201EB8201A3
:1043F80027E7D8000C186468002C7FF411AF172445
:1044080014700DE72E48FCF7E7FE4020FCF7E4FEA9
:104418004EE72C48FCF7E0FE2B6846E72A48FCF7F5
:10442800DBFE2B683EE72948FCF7D6FE2B6836E70B
:104438009A8AB2F57A7FBFF426AF4FF47A729A82DD
:1044480021E718231370F4E643F001032B6023E7F8
:10445800D8BB030850B70308444300201479030865
:10446800887203089B49002084520020BC4F00201A
:10447800B03C0020B84F0020B8710020E03D00207B
:1044880009600002D45600205C24002064690020E2
:104498006C7900203046002020210020A024002034
:1044A800902400209E67002098260020C0C9FB4861
:1044B800CC24002017B7D1389C2600204C79002046
:1044C80009400002016000020920000208600002A1
:1044D80002F003080000040808B523F01FFEFCF7EB
:1044E800B9FE23F003FEFFF767FE0120BDE8084090
:1044F80014F010BC38B50C4C0C4DAC4206D26168B7
:1045080020461434FCF732FEAC42F8D3084A094B73
:10451800094C1460002209491A705A70084808604A
:10452800BDE838401CF01EBC50B70308D8BB0308D0
:10453800B84F00209B490020B03C0020BC4F002011
:104548008452002008B5FFF7D5FF23F0E7FDFCF7FC
:1045580081FEBDE8084023F0C9BD00BFF0B50C29B5
:104568002BD8DFE801F06F2A2A2A4C2A2A2A2B2A7C
:104578002A2A0700046AB2F80CE097881668674D83
:1045880024F480540462036A4468C16923F4005324
:1045980043EA0E3321F4E641A84243EA073341EAED
:1045A800062100F0B58005F50065A84200F0B0804E
:1045B80092684460C16102640362F0BD046A96892E
:1045C8009588D2F800E0554F24F480740462036A99
:1045D8004468C16923F4007343EA062321F0730198
:1045E800B84243EA052341EA0E017ED04C4DA84269
:1045F8007BD092684460C161C2630362F0BD046A03
:1046080096899588D2F800E0444F24F0100404629B
:10461800036A4468816923F0200321F0807143EA2A
:10462800061321F4E641B84243EA051341EA0E2194
:1046380048D03B4DA84245D092684460816182636E
:104648000362F0BD046A9389B2F804E01768334E38
:1046580024F001040462056A4468816943EA0E0390
:1046680021F4803125F002059BB221F07301B0429C
:1046780043EA050341EA070114D0294DA84211D0A5
:1046880005F54065A8420DD005F58065A84209D01A
:1046980005F58065A84205D092684460816142634F
:1046A8000362F0BDD689158A578A23F0080333437D
:1046B8003D43D68824F4407423F00403ADB2334359
:1046C8002C43E9E7D589178AD68823F0800343EA83
:1046D800051324F44064558A23F0400344EA870410
:1046E80043EA061344EA8504A6E7D589178AD688DB
:1046F80023F4006343EA052324F44054558A23F441
:10470800806344EA071443EA062344EA051470E781
:10471800158A24F4804444EA851449E7002C0140B2
:10472800003401402DE9F84F4FF48C720021824883
:10473800824C834D834E844FDFF82882DFF828921D
:1047480030F0A7F981488249DFF820E2DFF820C27B
:1047580000221359834200F0C380B3F1804F00F068
:10476800D580AB4200F0D980B34200F0D880BB427C
:1047780000F0D780734500F0D680634500F0A6802E
:10478800434500F0D2804B4500F0D280DFF8E4A129
:10479800534508BF4FF4802300F09A801432B2F5D5
:1047A800AA7FD6D1654D6B4F6B4E05F5AA784FF0B1
:1047B800030A4FF0020903E01435454500F08E80E6
:1047C800AB79002BF8D02B791C09013C052C03F0A0
:1047D8000F03F1D837F8140040FA03F2D207EBD5EB
:1047E8004FF0010B0BFA03F3013B18402EF0DAFDF2
:1047F8005A4B1B5D184416EBC004DDD056F8303018
:104808005748297A03F13842920A825C02F01F0065
:104818005209022A0BFA00FB71D0032A68D0012A38
:1048280005D14B4A4A4852694BEA02024261B4F840
:1048380004E0BEFA8EF2C2F11F0292B2D00803EB76
:10484800800002F00702046A92004FF00F0C0CFA85
:1048580002FC24EA0C040462046A01FA02F222430C
:10486800002402624FF0010C224603E0102A04F1F2
:104878000204A1D00CFA02F030EA0E0102F10102A2
:10488800F4D1D3F808B00AFA04F1C9430BEA010BD2
:10489800C3F808B0D3F808B0C3F808B0B3F804B048
:1048A8001FFA8BFB2BEA00009880988880B29880CA
:1048B800186808401860D3F800B009FA04F040EA14
:1048C8000B001860D8680140D960CFE74FF4005357
:1048D800D1F818A043EA0A038B615FE7BDE8F88FB7
:1048E800D1F818A04FF4006343EA0A038B6155E737
:1048F800174A1748D2694BEA0202C26197E7144A7D
:10490800134892694BEA0202826190E70123D1F8C9
:104918001CA043EA0A03CB6140E70223F7E704231C
:10492800F5E71023F3E72023F1E74FF48033CFE7CF
:104938004FF40033CCE700BFC44A00208477030853
:10494800000400400008004000100040002C014016
:10495800001002403C7C0308B86B0020487C030828
:104968007C770308004001400044014000140040E7
:104978000034014000480140002867D003682DE951
:10498800F04F03F138445C4EA40A0125345D04F06D
:104998001F066409022C05FA06F558D0032C00F00E
:1049A800A580012C58D08088B0FA80F4C4F11F0487
:1049B800A4B2E50803EB850504F007042E6AA400F9
:1049C8000F27A74026EA07062E622E6A01F0030782
:1049D800A2407C1E3243012CC1F3810CC1F30018A4
:1049E8002A62C1F341113CD9C60700F189808507C5
:1049F80000F19580440700F1A380020700F1B1801F
:104A0800C60600F1BF80850600F1CD80440600F19E
:104A1800DB80020600F1E980C60500F1F780850514
:104A280000F10581440500F11381020500F121819F
:104A3800C60400F12F81850400F13D81440400F192
:104A48004B81020400F15981BDE8F08F70472B4C6F
:104A5800A6693543A561A6E7284C666935436561B3
:104A6800A1E7002422464FF0010E4FF0030904E0AD
:104A78000132102A04F10204E6D00EFA02F636EAF0
:104A88000005F5D1D3F808A009FA04F5ED430AEAC0
:104A9800050AC3F808A0D3F808B00CFA04FA4AEAE1
:104AA8000B0AC3F808A0B3F804A01FFA8AFA2AEA86
:104AB80006069E80B3F804A008FA02F646EA0A063B
:104AC800B6B29E801E682E401E60D3F800A007FA7A
:104AD80004F646EA0A061E60D3F80CA001FA04F6AA
:104AE80005EA0A0A46EA0A05DD60C1E7034CE669F9
:104AF8003543E56157E700BF7C77030800100240A3
:104B08001A6822F003021A601A683A431A60DA68CF
:104B180022F003020A438507DA607FF56BAF1A6853
:104B280022F00C021A601A6842EA87021A60DA68F0
:104B380022F00C0242EA81024407DA607FF55DAF99
:104B48001A6822F030021A601A6842EA07121A60DC
:104B5800DA6822F0300242EA0112DA6002077FF5D1
:104B68004FAF1A6822F0C0021A601A6842EA871228
:104B78001A60DA6822F0C00242EA8112C606DA60D8
:104B88007FF541AF1A6822F440721A601A6842EA47
:104B980007221A60DA6822F4407242EA0122850686
:104BA800DA607FF533AF1A6822F440621A601A6837
:104BB80042EA87221A60DA6822F4406242EA8122D5
:104BC8004406DA607FF525AF1A6822F440521A606D
:104BD8001A6842EA07321A60DA6822F4405242EA56
:104BE8000132DA6002067FF517AF1A6822F44042F4
:104BF8001A601A6842EA87321A60DA6822F4404278
:104C080042EA8132C605DA607FF509AF1A6822F4F4
:104C180040321A601A6842EA07421A60DA6822F4D7
:104C2800403242EA01428505DA607FF5FBAE1A6838
:104C380022F440221A601A6842EA87421A60DA6847
:104C480022F4402242EA81424405DA607FF5EDAE63
:104C58001A6822F440121A601A6842EA07521A6067
:104C6800DA6822F4401242EA0152DA6002057FF55E
:104C7800DFAE1A6822F440021A601A6842EA8752C4
:104C88001A60DA6822F4400242EA8152C604DA6005
:104C98007FF5D1AE1A6822F040721A601A6842EAAB
:104CA80007621A60DA6822F0407242EA01628504FB
:104CB800DA607FF5C3AE1A6822F040621A601A689B
:104CC80042EA87621A60DA6822F0406242EA816248
:104CD8004404DA607FF5B5AE1A6822F040521A60D3
:104CE8001A6842EA07721A60DA6822F0405242EA09
:104CF8000172DA6002047FF5A7AE1A6822F040421A
:104D08001A601A6842EA87771F60DA6822F0404220
:104D180042EA8171D960BDE8F08F00BF03682DE9D0
:104D2800F04F03F13845644EAD0A0124755D05F076
:104D38001F066D09022D04FA06F400F0A280032D67
:104D480000F0A480012D52D08088B0FA80F4C4F11C
:104D58001F04A4B2E50803EB850504F007042E6AD6
:104D6800A4000F27A74026EA07062E622E6A01F044
:104D7800030702FA04F47A1E3443012AC1F3810CB2
:104D8800C1F300182C62C1F3411135D9C60700F1EF
:104D98009780850700F1A380440700F1B1800207DE
:104DA80000F1BF80C60600F1CD80850600F1DB80EA
:104DB800440600F1E980020600F1F780C60500F11B
:104DC8000581850500F11381440500F12181020563
:104DD80000F12F81C60400F13D81850400F14B816B
:104DE800440400F15981020455D4BDE8F08F334DD5
:104DF8006E6934436C61A7E7002422464FF0010E28
:104E08004FF0030904E00132102A04F10204ECD047
:104E18000EFA02F636EA0005F5D1D3F808A009FA29
:104E280004F5ED430AEA050AC3F808A0D3F808B068
:104E38000CFA04FA4AEA0B0AC3F808A0B3F804A06B
:104E48001FFA8AFA2AEA06069E80B3F804A008FA2E
:104E580002F646EA0A06B6B29E801E682E401E601A
:104E6800D3F800A007FA04F646EA0A061E60D3F84B
:104E78000CA001FA04F605EA0A0A46EA0A05DD600A
:104E8800C1E70E4DAE693443AC615DE70B4DEE6989
:104E98003443EC6158E71A6822F040421A601A68F5
:104EA80042EA87771F60DA6822F0404242EA81715D
:104EB800D960BDE8F08F00BF7C770308001002407E
:104EC8001A6822F003021A601A683A431A60DA680C
:104ED80022F003020A438507DA607FF55DAF1A689E
:104EE80022F00C021A601A6842EA87021A60DA682D
:104EF80022F00C0242EA81024407DA607FF54FAFE4
:104F08001A6822F030021A601A6842EA07121A6018
:104F1800DA6822F0300242EA0112DA6002077FF50D
:104F280041AF1A6822F0C0021A601A6842EA871272
:104F38001A60DA6822F0C00242EA8112C606DA6014
:104F48007FF533AF1A6822F440721A601A6842EA91
:104F580007221A60DA6822F4407242EA01228506C2
:104F6800DA607FF525AF1A6822F440621A601A6881
:104F780042EA87221A60DA6822F4406242EA812211
:104F88004406DA607FF517AF1A6822F440521A60B7
:104F98001A6842EA07321A60DA6822F4405242EA92
:104FA8000132DA6002067FF509AF1A6822F440423E
:104FB8001A601A6842EA87321A60DA6822F44042B4
:104FC80042EA8132C605DA607FF5FBAE1A6822F440
:104FD80040321A601A6842EA07421A60DA6822F414
:104FE800403242EA01428505DA607FF5EDAE1A6883
:104FF80022F440221A601A6842EA87421A60DA6884
:1050080022F4402242EA81424405DA607FF5DFAEAD
:105018001A6822F440121A601A6842EA07521A60A3
:10502800DA6822F4401242EA0152DA6002057FF59A
:10503800D1AE1A6822F440021A601A6842EA87520E
:105048001A60DA6822F4400242EA8152C604DA6041
:105058007FF5C3AE1A6822F040721A601A6842EAF5
:1050680007621A60DA6822F0407242EA0162850437
:10507800DA607FF5B5AE1A6822F040621A601A68E5
:1050880042EA87621A60DA6822F0406242EA816284
:105098004404DA607FF5A7AE1A6822F040521A601D
:1050A8001A6842EA07721A60DA6822F0405242EA45
:1050B8000172DA6097E600BF10B50409013C052CBF
:1050C80017D80D4B33F8142000F00F0042FA00F304
:1050D80013F001030DD0012303FA00F0013810404A
:1050E8002EF060F9054A064B125D104403EBC00030
:1050F80010BD002010BD00BF3C7C0308487C03089D
:10510800B86B002001490248FEF74ABDB44B0020A5
:105118000048014001490248FEF742BD644B0020A7
:105128000040014001490248FEF73ABD3C4B0020CF
:105138000008004001490248FEF732BD144B002028
:105148000004004002494FF08040FEF729BD00BF2F
:10515800EC4A002010B5064C06482146FEF720FD13
:1051680004F1C8010448BDE81040FEF719BD00BFAE
:10517800C44A0020002C0140004401400149024873
:10518800FEF70EBDC44A0020002C01402DE9F04175
:105198000468514DA30AAB4200F084800AD94F4DF0
:1051A800AB4277D00135AB425FD0023DAB426DD008
:1051B800BDE8F0814A3DAB4270D00135AB4258D0D2
:1051C800B3F5801FF4D14FF0480E012647794FEA16
:1051D800970C00296AD0B000634685190227D4F8D5
:1051E8000C809F400CEB4503BFB23D4D03F1040C0E
:1051F80047EA080745F8231045F82C20E760EFF345
:105208001181502282F31288821905EBC2021369B8
:10521800002B32D013620433821905EBC20257699E
:1052280017B11F6053690433821905EBC2029769ED
:1052380017B11F6093690433821905EBC202D7695D
:1052480017B11F60D36904330027CAB21F6082F305
:105258001188304405EBC000036A8BB9E3684FF648
:10526800FE721340E360BDE8F0814FF4887E0626A5
:10527800ACE74FF0980E0326A8E705EB0E03CBE743
:10528800E36843F00103E360BDE8F0814FF0C00E2E
:1052980004269BE74FF0E80E052697E74FF0700EBF
:1052A800022693E74FF0200E00268FE7BF0802235F
:1052B80006FA03F0BB40DB43E768094D9BB23B406D
:1052C80087190CEB470CE3600CF1040345F82C102C
:1052D80045F8232093E700BF4B0010005100100051
:1052E800C44A002030B503685C4D18885C4CB4FB98
:1052F800F2F20139013AAB4294B283B089B282B278
:1053080066D05848834263D0B3F1804F60D0A0F58F
:10531800983083425CD000F58060834258D0524870
:1053280083425BD000F5806083427DD022F44072D6
:1053380000F58C3092B283421A80D9621C850ED057
:10534800484A93420BD002F54062934207D002F5D7
:105358008062934203D002F58062934201D1002219
:105368001A8601225A611A883C4992B242F0010217
:105378008B421A8062D0B3F1804F61D03B4A93428E
:1053880060D002F5806293425ED002F500629342DB
:105398005CD002F5806293425AD002F59032934273
:1053A80058D002F54062934256D002F5806293428B
:1053B8001ED002F58062934208BF092219D002A8C4
:1053C8004FF0012340F8043D24F08AF903B030BDC2
:1053D800254822F07002834292B2A3D101201A809C
:1053E800D9621C8558611A8892B202431A80C5E7AF
:1053F80008221F4B03EBC20301A893F835408DF830
:105408000440012300228DF805308DF807308DF80F
:10541800062024F065F91B2CD8D1164B019301A85E
:1054280024F05EF903B030BD01201A80D9621C85D2
:1054380058611A8892B202431A809CE70022D8E782
:105448000122D6E70222D4E70322D2E70422D0E7DA
:105458000522CEE70622CCE70722CAE7002C014046
:1054680000A24A040034014000100040000400403B
:10547800904C030819010001204B98422DD0B0F13F
:10548800804F2CD0A3F5943398422AD003F580633B
:10549800984228D003F50063984226D003F580632C
:1054A800984224D003F59033984222D003F5406304
:1054B800984220D003F58063984207D003F58063B3
:1054C800984208BF092202D00020704708220C4BDE
:1054D80003EBC20393F8340070470022F7E7012278
:1054E800F5E70222F3E70322F1E70422EFE70522BA
:1054F800EDE70622EBE70722E9E700BF002C0140B1
:10550800904C03082DE9F04F013085B0C3B20393E6
:105518000B4602918B4C8C4E002B00F09A80322067
:105528008A4D8B4FDFF82C921EF06CFF4FF4FA7AFD
:105538004FF0100C4FF47A70D9F80430C3F3080315
:10554800002B40F0DE80EFF31183002B40F0D98070
:105558002968A26800BF2B689942F9D1D7F800E002
:1055680000FB0EF39B1AB3FBFEF300FB01314FF077
:10557800010E0191D9F80430C3F30803002B40F061
:105588008780EFF31183002B40F082802B68A1689D
:1055980000BF2A689342F9D1D7F800B000FB0BF29C
:1055A800521AB2FBFBF200FB0323019A9B1AB3F5D4
:1055B8007A7FDFD3BAF1010ABED1039B002B40F0FA
:1055C800BD804FF47A7ADFF88C9150464FF0100C7A
:1055D800D9F80430C3F30803002B75D1EFF3118316
:1055E800002B71D12968A26800BF2B689942F9D1B4
:1055F800D7F800E000FB0EF39B1AB3FBFEF300FBA9
:1056080001314FF0010E0191D9F80430C3F30803BA
:1056180013BBEFF31183FBB92B68A16800BF2A689D
:105628009342F9D1D7F800B000FB0BF2521AB2FB43
:10563800FBF200FB0323019A9B1AB3F57A7FE3D3AD
:10564800BAF1010AC4D1029B013B0293002B7FF4FB
:1056580066AF05B0BDE8F08FEFF311888CF31288C0
:10566800A1682368DB0344BFC6F800E0A1682B6883
:1056780032685FFA88F888F31188D7F800801A44EE
:1056880000FB08F35B1AB3FBF8F300FB0233D2E725
:10569800EFF311888CF31288A1682368DB0344BFF9
:1056A800C6F800E0A1682B6832685FFA88F888F3CA
:1056B8001188D7F800801A4400FB08F35B1AB3FB83
:1056C800F8F300FB023370E7EFF311828CF31288D2
:1056D800D4F808E02368D90303D501233360D4F84C
:1056E80008E02B683168D2B282F311883A6819440D
:1056F80000FB02F3A3EB0E03B3FBF2F300FB013153
:105708007FE7EFF311828CF31288D4F808E023685E
:10571800D90303D501233360D4F808E02B68316836
:10572800D2B282F311883A68194400FB02F3A3EB62
:105738000E03B3FBF2F300FB013118E7184620F023
:1057480003FF3EE710E000E014580020185800203E
:105758001C58002000ED00E0204B5B68C3F30803F1
:1057680030B4BBB9EFF31183A3B91D4B1D4C1868B6
:10577800A16800BF1A689042F9D11B4B1C684FF40E
:105788007A7202FB04F3591AB1FBF4F130BC02FB44
:1057980000107047EFF31182102383F31288114928
:1057A8008C680B6813F4803F104B02D001201860FE
:1057B8008C680B49D2B20D68186882F311880A4BBD
:1057C80019684FF47A72284402FB01F31B1B30BCA2
:1057D800B3FBF1F302FB0030704700BF00ED00E0BF
:1057E8001858002010E000E01C5800201458002031
:1057F8002DE9F84F8046FFF7AFFF254E2549DFF822
:10580800A0E0254A254D844610274FF47A740120DC
:10581800DEF80430C3F30803D3B9EFF31183BBB93F
:105828000B68D2F808A000BFD1F800904B45F7D11B
:10583800D6F800B004FB0BF9A9EB0A09B9FBFBF990
:1058480004FB0393A3EB0C034345E1D3BDE8F88FB6
:10585800EFF3118A87F31288D2F808B01368DB03D4
:1058680044BF2860D2F808B00B68D5F800905FFAFA
:105878008AFA8AF31188D6F800A0994404FB0AF33F
:10588800A3EB0B03B3FBFAF304FB0933DAE700BF1E
:105898001C5800201858002010E000E01458002080
:1058A80000ED00E02DE9F04FDFF830C1474A4849E4
:1058B800484E494D8046102718F1FF38C0F08480C3
:1058C800DCF80430C3F30803002B5CD1EFF3118339
:1058D800002B58D10B68946800BF08688342F9D13F
:1058E800D6F800904FF47A7000FB09FEAEEB040E78
:1058F800BEFBF9FE00FB03EEDCF80430C3F308033B
:105908004FF47A740120FBB9EFF31183E3B90B6804
:10591800D2F808A000BFD1F800904B45F7D1D6F8CF
:1059280000B004FB0BF9A9EB0A09B9FBFBF904FB6E
:105938000393A3EB0E03B3F57A7FBDD2DCF80430F2
:10594800C3F30803002BDFD0EFF3118A87F3128823
:10595800D2F808B01368DB0344BF2860D2F808B057
:105968000B68D5F800905FFA8AFA8AF31188D6F89E
:1059780000A0994404FB0AF3A3EB0B03B3FBFAF36F
:1059880004FB0933D5E7EFF3118487F31288D2F8C3
:1059980008901368D80303D501232B60D2F8089028
:1059A8000B682868E4B284F31188D6F800A04FF495
:1059B8007A7400EB030E04FB0AF3A3EB0903B3FBB1
:1059C800FAF304FB0E3E97E7BDE8F08F10E000E025
:1059D800185800201C5800201458002000ED00E042
:1059E80030B4EFF31183102282F312880649074C72
:1059F8000A680748013200250A602560DBB20268A0
:105A080083F3118830BC70471858002014580020C0
:105A180010E000E01D4B70B59C68236D626BDD697A
:105A2800C2B1A36B2BB12B0702D5236D08221A62D2
:105A380070BD2A06F7D5A26A616A8A4220D0511C35
:105A4800A069A162825C2069266D81423285EAD311
:105A5800A362E8E7A906E4D5E26A22B1988C216B33
:105A680080B29047DDE7E1699B8C6069DBB24E1C30
:105A7800E6614354E169E368994228BFE261D0E7EF
:105A8800226D136823F080031360CCE754320020A2
:105A98001D4B70B55C68236D626BDD69C2B1A36B89
:105AA8002BB12B0702D5236D08221A6270BD2A0676
:105AB800F7D5A26A616A8A4220D0511CA069A16206
:105AC800825C2069266D81423285EAD3A362E8E7C9
:105AD800A906E4D5E26A22B1988C216B80B290477E
:105AE800DDE7E1699B8C6069DBB24E1CE6614354DB
:105AF800E169E368994228BFE261D0E7226D136843
:105B080023F080031360CCE7543200201D4B70B59E
:105B18001C68236D626BDD69C2B1A36B2BB12B07C7
:105B280002D5236D08221A6270BD2A06F7D5A26A2B
:105B3800616A8A4220D0511CA069A162825C2069F6
:105B4800266D81423285EAD3A362E8E7A906E4D547
:105B5800E26A22B1988C216B80B29047DDE7E16957
:105B68009B8C6069DBB24E1CE6614354E169E368D3
:105B7800994228BFE261D0E7226D136823F08003C1
:105B88001360CCE75432002070B4EFF31186502331
:105B980083F31288836B1A68D20720D45D686DB9C5
:105BA800446A826A944217D081691144D9600ED937
:105BB800A21A5A608462002280F854201A6842F0BF
:105BC8000102F1B21A6081F3118870BC7047016953
:105BD8008A1A5A608562EEE7012380F85430F1B2E0
:105BE80081F3118870BC704703685B6A03B118477A
:105BF800704700BF03681B6A03B11847704700BFAE
:105C080003682DE9F041DF691FB13B46BDE8F0416B
:105C18001847002A164611DD04460D460E4400E0DA
:105C280023689B68204698470028F9D0236815F810
:105C3800011B1B6820469847AE42F1D1BDE8F081B0
:105C480003689B69184700BF03685B69184700BF72
:105C58000368DB68184700BF03689B68184700BFE4
:105C680003685B68184700BF03681B68184700BFD4
:105C7800054B53F8203033B11A689B88918A0B4240
:105C880018BF1B0493617047E4570020036803F1B1
:105C980038422DE9F04F920A584DAA5C02F01F05D0
:105CA80052090124022A04FA05F400F08C80032A20
:105CB80000F08E80012A3CD001F003077A1E012AE9
:105CC800C1F3810CC1F300188088C1F3411135D9A3
:105CD800C60700F19780850700F1A380440700F10B
:105CE800B180020700F1BF80C60600F1CD808506AD
:105CF80000F1DB80440600F1E980020600F1F7803C
:105D0800C60500F10581850500F11381440500F100
:105D18002181020500F12F81C60400F13D8185042F
:105D280000F14B81440400F15981020455D4BDE8C7
:105D3800F08F334A55692C435461BDE7002422464D
:105D48004FF0010E4FF0030904E00132102A04F16C
:105D58000204ECD00EFA02F636EA0005F5D1D3F8C3
:105D680008A009FA04F5ED430AEA050AC3F808A0F1
:105D7800D3F808B00CFA04FA4AEA0B0AC3F808A0E8
:105D8800B3F804A01FFA8AFA2AEA06069E80B3F836
:105D980004A008FA02F646EA0A06B6B29E801E6811
:105DA8002E401E60D3F800A007FA04F646EA0A0659
:105DB8001E60D3F80CA001FA04F605EA0A0A46EABE
:105DC8000A05DD60C1E70E4A95692C43946173E7C3
:105DD8000B4AD5692C43D4616EE71A6822F0404219
:105DE8001A601A6842EA87771F60DA6822F0404230
:105DF80042EA8171D960BDE8F08F00BF7C77030863
:105E0800001002401A6822F003021A601A683A4326
:105E18001A60DA6822F003020A438507DA607FF520
:105E28005DAF1A6822F00C021A601A6842EA87020B
:105E38001A60DA6822F00C0242EA81024407DA604A
:105E48007FF54FAF1A6822F030021A601A6842EAEA
:105E580007121A60DA6822F0300242EA0112DA60A8
:105E680002077FF541AF1A6822F0C0021A601A686B
:105E780042EA87121A60DA6822F0C00242EA811206
:105E8800C606DA607FF533AF1A6822F440721A60EA
:105E98001A6842EA07221A60DA6822F4407242EA73
:105EA80001228506DA607FF525AF1A6822F4406280
:105EB8001A601A6842EA87221A60DA6822F4406295
:105EC80042EA81224406DA607FF517AF1A6822F4A5
:105ED80040521A601A6842EA07321A60DA6822F4F5
:105EE800405242EA0132DA6002067FF509AF1A68C9
:105EF80022F440421A601A6842EA87321A60DA6865
:105F080022F4404242EA8132C605DA607FF5FBAEF0
:105F18001A6822F440321A601A6842EA07421A6084
:105F2800DA6822F4403242EA01428505DA607FF5F8
:105F3800EDAE1A6822F440221A601A6842EA8742D3
:105F48001A60DA6822F4402242EA81424405DA60A3
:105F58007FF5DFAE1A6822F440121A601A6842EA26
:105F680007521A60DA6822F4401242EA0152DA60F3
:105F780002057FF5D1AE1A6822F440021A601A6849
:105F880042EA87521A60DA6822F4400242EA8152F1
:105F9800C604DA607FF5C3AE1A6822F040721A6050
:105FA8001A6842EA07621A60DA6822F0407242EA26
:105FB80001628504DA607FF5B5AE1A6822F04062A6
:105FC8001A601A6842EA87621A60DA6822F0406248
:105FD80042EA81624404DA607FF5A7AE1A6822F0CB
:105FE80040521A601A6842EA07721A60DA6822F0A8
:105FF800405242EA0172DA6097E600BF2DE9F04F9D
:106008004A484B4B4B4C4FF090414FF0010A4FF030
:1060180002094FF004084FF0080C4FF0100E20272B
:106028004026802530F8022B12F0010F03D01960AA
:10603800A3F804A0083312F0020F03D01960A3F8E4
:106048000490083312F0040F03D01960A3F80480F9
:10605800083312F0080F03D01960A3F804C00833FE
:1060680012F0100F03D01960A3F804E0083312F0FF
:10607800200F02D019609F80083312F0400F02D021
:1060880019609E80083312F0800F02D019609D803D
:10609800083312F4807F05D04FF4807B1960A3F891
:1060A80004B0083312F4007F05D04FF4007B196068
:1060B800A3F804B0083312F4806F05D04FF4806B56
:1060C8001960A3F804B0083312F4006F05D04FF438
:1060D800006B1960A3F804B0083312F4805F05D090
:1060E8004FF4805B1960A3F804B0083312F4005F22
:1060F80005D04FF4005B1960A3F804B0083312F41C
:10610800804F05D04FF4804B1960A3F804B00833D2
:10611800D20B04D04FF4004219609A80083301F57D
:106128008061A1427FF47EAFBDE8F08F3C7C03081C
:10613800B86B002000180048002852D0036803F10B
:1061480038422DE9F04F920A504DAA5C02F01F0523
:1061580052090124022A04FA05F443D0032A00F064
:106168009080012A43D001F003077A1E012AC1F367
:10617800810CC1F300188088C1F341113CD9C607CE
:1061880000F18880850700F19480440700F1A2801F
:10619800020700F1B080C60600F1BE80850600F156
:1061A800CC80440600F1DA80020600F1E880C605DA
:1061B80000F1F680850500F10481440500F11281A3
:1061C800020500F12081C60400F12E81850400F14A
:1061D8003C81440400F14A81020400F15881BDE881
:1061E800F08F70472A4A95692C439461BBE7284A87
:1061F80055692C435461B6E7002422464FF0010E3E
:106208004FF0030904E00132102A04F10204E6D039
:106218000EFA02F636EA0005F5D1D3F808A009FA15
:1062280004F5ED430AEA050AC3F808A0D3F808B054
:106238000CFA04FA4AEA0B0AC3F808A0B3F804A057
:106248001FFA8AFA2AEA06069E80B3F804A008FA1A
:1062580002F646EA0A06B6B29E801E682E401E6006
:10626800D3F800A007FA04F646EA0A061E60D3F837
:106278000CA001FA04F605EA0A0A46EA0A05DD60F6
:10628800C1E7034AD5692C43D4616CE77C770308DE
:10629800001002401A6822F003021A601A683A4392
:1062A8001A60DA6822F003020A438507DA607FF58C
:1062B8006CAF1A6822F00C021A601A6842EA870268
:1062C8001A60DA6822F00C0242EA81024407DA60B6
:1062D8007FF55EAF1A6822F030021A601A6842EA47
:1062E80007121A60DA6822F0300242EA0112DA6014
:1062F80002077FF550AF1A6822F0C0021A601A68C8
:1063080042EA87121A60DA6822F0C00242EA811271
:10631800C606DA607FF542AF1A6822F440721A6046
:106328001A6842EA07221A60DA6822F4407242EADE
:1063380001228506DA607FF534AF1A6822F44062DC
:106348001A601A6842EA87221A60DA6822F4406200
:1063580042EA81224406DA607FF526AF1A6822F401
:1063680040521A601A6842EA07321A60DA6822F460
:10637800405242EA0132DA6002067FF518AF1A6825
:1063880022F440421A601A6842EA87321A60DA68D0
:1063980022F4404242EA8132C605DA607FF50AAF4C
:1063A8001A6822F440321A601A6842EA07421A60F0
:1063B800DA6822F4403242EA01428505DA607FF564
:1063C800FCAE1A6822F440221A601A6842EA874230
:1063D8001A60DA6822F4402242EA81424405DA600F
:1063E8007FF5EEAE1A6822F440121A601A6842EA83
:1063F80007521A60DA6822F4401242EA0152DA605F
:1064080002057FF5E0AE1A6822F440021A601A68A5
:1064180042EA87521A60DA6822F4400242EA81525C
:10642800C604DA607FF5D2AE1A6822F040721A60AC
:106438001A6842EA07621A60DA6822F0407242EA91
:1064480001628504DA607FF5C4AE1A6822F0406202
:106458001A601A6842EA87621A60DA6822F04062B3
:1064680042EA81624404DA607FF5B6AE1A6822F027
:1064780040521A601A6842EA07721A60DA6822F013
:10648800405242EA0172DA6002047FF5A8AE1A6847
:1064980022F040421A601A6842EA87771F60DA6879
:1064A80022F0404242EA8171D960BDE8F08F00BF16
:1064B80010B1036882881A85704700BF10B103685D
:1064C80082889A61704700BF38B1002983880268C2
:1064D80014BF002110218B40936170470E4B1B881D
:1064E80001463BB90D4B0E4A1B7810680BB981F079
:1064F8000101E9E70B4B5A691AB118B91A6810601B
:1065080058747047084A18681188084A92FBF1F2D3
:106518000121026059747047F0570020F25700209B
:10652800F4570020F85700201058002020A1070039
:1065380010B40A4B0A4A1C7801238340234052F8BE
:10654800200029B9B3FA83F149095DF8044BBBE788
:10655800191C18BF01215DF8044BB5E7E05700206E
:10656800E457002008B501210220FFF7E1FF094B9D
:106578001B7803F00503052B08D000210120FFF745
:10658800D7FF00210846FFF7D3FFFEE71CF07AFA91
:10659800F3E700BF5032002030B1036882881B8ABD
:1065A8001A4214BF01200020704700BF2DE9F041B6
:1065B8000B4E346873691C400FD0DFF82880012720
:1065C800B4FA84F3C3F11F0307FA03F558F823005C
:1065D80003689847AC437561F2D1BDE8F08100BF0C
:1065E80000040140302300202DE9F04FC04B1E78F5
:1065F8008BB0002E40F0BC80BE4BBF4C1D78DFF83E
:1066080018A3DFF81893DFF8188305F00105A4F143
:106618000A0B54F80A3CBBB1CC2707FB06B718464F
:10662800FFF71EFB80B154F80A0CFFF711FB14F8B2
:10663800023C8BB9242831D0F5B154F80A3C1846ED
:10664800FFF70EFB0028EED10136032E04F1CC042F
:10665800DFD10BB0BDE8F08F012B23D0022B2BD05C
:10666800032B37D0042B67D0052B40D0062B4FD0F7
:1066780054F80A2C1346D2E754F80A3C23281A4641
:1066880000F089819D4991F82A108142C7D19C4B1D
:10669800CAF80090C3F80C801346C0E7012304F839
:1066A800023CCAE74D2854F80A2C0CBF02230023E9
:1066B80004F8023C1346B2E700233C2804F8023CE5
:1066C80045D03E28D4D10122032304F8012C04F834
:1066D800023CB2E7C02814D80022042304F8050CB1
:1066E80004F8040C04F8062C04F8023CA5E714F896
:1066F800063C14F8052C9A422FD814F8043C83421F
:1067080003D0002304F8023C97E7062304F8023C70
:1067180014F801ECBEF1000F00F08281BEF1010F08
:1067280000F0C68101360023032E04F8023C04F170
:10673800CC047FF46EAF8CE714F8043C04F8030C27
:106748005840052304F8040C04F8023C75E70322BA
:1067580004F8013C04F8022C6FE714F8042CF9182B
:106768004240013304F8042C04F8063C887264E7BC
:10677800644B186800283FF46CAFFAF7A3FCDFF805
:10678800A4A1614DDFF8A091DAF80000FFF768FADC
:1067980000283FF45EAFDAF80000FFF759FA09283D
:1067A8001BD03F2819D02B68002B67D1042800F094
:1067B800AD810C2800F0E8807F28E5D0A0F1200208
:1067C800D2B25E2AE0D80BB92028DDD05A1C09F8CD
:1067D80003002A602AF01AFBD6E72C68002C5BD14C
:1067E8004A4FA34607F59878BBF1000F08BFBB4690
:1067F80008374745F8D1BBF1000F00F07C81083F0E
:10680800DBF800003A68065D135D9E42204402EB07
:10681800040140F06E81661E4E4422460BB9FD2AE3
:106828005DD906F8013F01322A6010F8013F11F8DE
:1068380001EF9E45F2D00AB15F4512D034482AF0E4
:10684800EDFA5F4508D35BF8080B2AF0E7FA092050
:106858002AF0DCFABB45F6D92E482AF0DFFA2A6876
:106868000024944290D2661E4E4416F8010F2AF076
:10687800CDFA2B6801349C42F7D385E70C2800F049
:1068880083800A2852D00D2850D07F2800F0FD8040
:10689800FF2B3FF679AF91E71C4E002706F5987855
:1068A800BB4602E0083646450DD0224631684846C8
:1068B800FAF716FF0028F5D1B346002FF2D1374674
:1068C80008364645F1D13B465F469B46002B97D19B
:1068D800002F3FF459AF0E482AF0A0FAB3E7511C35
:1068E800202009F80200296009F801300A46A3E7C8
:1068F80068520020E57500200E500020D456002074
:1069080000ED00E06036002068370020F0550308ED
:10691800007E0308087E0308FC9F0020EFBEADDE62
:106928000400FA0564360020683600202AF0F7FAD9
:1069380023217E482EF0C4F8002800F0E580A0EB63
:106948000900286088B1431E19F80310202940F077
:10695800EB8009EB030204E012F8011D202948D15D
:106968000346581E002BF7D12B604FF4807200218C
:1069780048462EF08EF86E4B1B78002B3FF469AE1C
:106988006C482AF04BFAFFE66B482AF047FA694848
:106998002AF044FAF8E669496948C978694ADFF88B
:1069A800D8E11364003118BF0121017066495164B0
:1069B8004021936482F84C1082F84D506349644832
:1069C8000B604432CEF80020594A012313702AF094
:1069D8003BFE58482AF022FA4FF400600EF0D0FA35
:1069E8005C4B93F82A30232B00F0968014F8023C75
:1069F8003CE62B60584C002204F5987809F80320EF
:106A080002E0083444457BD02168484611F062F919
:106A18000028F6D0444573D2636898470023A3E75B
:106A28004E4BADF822E00FCB0DF1280C02AF87E8F2
:106A38000F004CF824ED14F8051C14F8033C0694D8
:106A480004EB010E624639464FF0010C06A8CDF85A
:106A58001CE0ADF820308DF824C002F0ABFFE8B997
:106A6800019F002304F8023C002F3FF4EDAD54F8D9
:106A78000A0C11F01BFB013654F80A0CB847032E18
:106A880004F1CC047FF4C5ADE3E5013B00223448B2
:106A98002B6009F803202AF0C1F975E6029A314BF8
:106AA80003923946A4F10A00029311F053FAD7E78A
:106AB80014F8053C14F8032C0694234407936E2A13
:106AC8004FF0000308930993ADF820207FF42AAE15
:106AD80006A8FAF784FE06A8FAF776FE074606A87F
:106AE800FAF772FE06A8FAF76FFE1F4B1F60586090
:106AF80018E622469FE61D48083F2AF08FF9A2E6CD
:106B08001B482AF08BF989E728681BE7074810F02B
:106B18009CF80BB0BDE8F08F164A14F8023CC2F896
:106B28000C80CAF80090A1E5034663E768360020A8
:106B380068520020087E0308107E03089B49002045
:106B4800182B002030230020593B00086436002011
:106B58003C7E0308D4560020F0550308104D030866
:106B6800387E0308F07B0020202A0020007E0308DE
:106B78001C7E030800ED00E0603600202DE9F04F90
:106B88002DED068BAB4BAC4A1C7897B000F59C41B9
:106B9800203181460B911160002C00F0E886A74A4D
:106BA8001268904240F28380A54A06921668A54969
:106BB800A54A0591013C1C70A44B049206F480562A
:106BC8000893002E40F08180A14B1B78022B01F026
:106BD8008E81042B01F07D81012B01F031819D4BC9
:106BE8009945089B9B7800F29685002B40F0978585
:106BF800994B0793069B1E6816F4805740F08586CC
:106C0800DFF894A2049BB3F90610059B5D8BA9429B
:106C1800B4BF00250125914B1B6813F080535ED04B
:106C2800079A127812F001025FD00598408C8842CA
:106C380041F3B082002D5ED1894C94F88C10002964
:106C480059D188488849006890F82D0000240C60C4
:106C58004C608C60854900284ED10870002A4FD0BE
:106C6800F1064DD5824A1278D20649D4002F47D171
:106C7800002B45D1740243D47E4B1B78002B02F0C5
:106C880033827D4B9B78002D42F0C7823BB17B4A13
:106C98007B4B12681B689B1A002BC2F2B68210202D
:106CA8006F4C11F051FF012384F88D3028E0644BBC
:106CB80006931E68644B634A049306F48056634B3C
:106CC80005920893002E3FF47FAF00216348FBF73D
:106CD800B6F900287FF478AF17F0C4F974E77002AA
:106CE8009ED4079A127802F001025D4C002184F8C4
:106CF8008C10002DA5D05D4901200870002AAFD165
:106D0800604B1A78002A79D10599049C488BB4F90C
:106D18000070898BB4F90240B842B4BF80260026BF
:106D280046F04003B942D8BF33469B0843F080067B
:106D3800A042B8BF3346049F43F04006A142C8BFF3
:106D480033469B08B7F90440B7F9066043F080075B
:106D5800A042B8BF3B4643F04007A142C8BF3B46EC
:106D68009B0843F080073E4C8642C8BF3B4643F031
:106D7800400794F88EE08E42B8BF3B469E4501F02E
:106D88006184A4F8902084F892203A4984F88E30DF
:106D98000E78002E01F058835F2B01F0D5836F2BFE
:106DA80001F01784079B1B78DA0727D494F8921010
:106DB80021BBB4F99030322B20DD94F88E200120CD
:106DC800572A84F8920001F08C87069B1B685F079E
:106DD80041F1A6825A2A41F0A38294F89430002BFC
:106DE80042F09C8194F8963083F0010384F8963041
:106DF800002B42F0FE810C2011F0A6FE224B0993D5
:106E0800224B234D0A93069B1B685C0700F1F3860F
:106E18000DF150091F4E0B950022C9F80420344685
:106E2800149240F6330B4FF0190840F28337049D53
:106E380037E000BFE45A0020EC590020E05A002057
:106E48008C6F0020A8560020EE5B00203046002002
:106E58004E5A0020404B4C00E57500207467002016
:106E6800C0230020B84F0020B04200206826002030
:106E78001C77002020210020B86700201858002027
:106E8800DC4B002017530020584F0020BC4F002037
:106E9800B44F002064690020B469002004345445CC
:106EA80020D0A178E378994218FB0170F6D2617876
:106EB800043118FB037335F911105945A8BF594619
:106EC800B1F5617FB8BF4FF461718142E6DD994247
:106ED800E4DC21782729E1D848460434FBF7A0F8F8
:106EE8005445DED1674A0B9D1378674A99E8030039
:106EF80082E80300002B40F0BC85644B1A78002A16
:106F080000F0F88501216048FBF799F8002840F067
:106F1800E682089BDB78002B40F0E1822B881FB2C9
:106F280027F001071FFA87F84345A5F8008001F00C
:106F38000D80574F4FF002090E204FF0140B4FF001
:106F4800FF0A87F8009087F801B087F802A011F0CF
:106F5800FBFD49464C48B5F80080FBF770F800285F
:106F680000F0D88228F001039BB243452B800AD059
:106F78000E2087F8009087F801B087F802A011F07A
:106F8800E3FDB5F8008018F0020F01F0B581414B20
:106F9800414A197850680C9318F0030F08BF81F024
:106FA8000201C1F340010B92FFF78EFA2421364803
:106FB800FBF745F830B9079A1378590744BF23F00F
:106FC80004031370099B1B6813F00A0F1BD00521DB
:106FD8002D48FBF734F8002801F0B2802F887B0792
:106FE80041F1478228480621FBF729F8002801F0DB
:106FF8009480780641F1358207212348FBF71FF872
:10700800002840F0B0870C211F48FBF718F82A88A1
:10701800002800F0938242F480739A422B8009D0B2
:107028001B4B022214211A700E20FF2259709A70ED
:1070380011F08AFD194B1B78082B00F08B820E2B60
:1070480000F08882069BD3F8008018F4806F5FD028
:10705800134B1B79002B00F0248214210A48FAF7FD
:10706800EEFF002840F0228228F0B6F9012011F046
:1070780079FC002849D0DFF82CA000274FF0CC0B72
:10708800A14614E0DC7100207467002068520020DB
:10709800FC350020E0570020E4570020444300203E
:1070A8007C4D002004500020DFB2022F2CD80BFBAF
:1070B80007F87B1C5AF80840002CF5D1032290F9F8
:1070C800023002940192C278E24951F822200092DB
:1070D800184622462346012111F0C6F8034607EB5D
:1070E800470000EB0010099353B121460AEB8000DA
:1070F800CC222DF0CEFC099B4AF808300137FFB2AC
:107108001EF078FC0028D0D14C46069BD3F80080AE
:10711800079B93F800A0D04B1AF0010A00F06D828B
:1071280001221A700A9B04991B68B1F906105A8942
:10713800CA4801279142077080F24582C84B4FF038
:107148007E521A60059BC74FB3F81890049B97F9B5
:107158000420B3F90030387897F801C0002AA3EB6F
:10716800090714BF01224FF0FF32002FB8BF7F423A
:10717800B7F5FA7FA8BF4FF4FA77B84280F2BB821E
:107188003F1A07EE907AF8EEE77AB74F4B45C7ED0E
:10719800007A03DAF1EE677AC7ED007A049BB3F957
:1071A80002E0AEEB0903002BB8BF5B42B3F5FA7FF0
:1071B800A8BF4FF4FA73984280F202821B1A07EEB6
:1071C800903AF8EEE77AF145C7ED017A03DDF1EE82
:1071D800677AC7ED017A049BB3F90400A0EB0903B1
:1071E800002BB8BF5B42B3F5FA7FA8BF4FF4FA7320
:1071F8006345CCBFA3EB0C03002302FB03F207EEAD
:10720800902AF8EEE77A4845C7ED027ABCBFF1EE5E
:10721800677AC7ED027A18F4805800F0AE81B1F5AC
:10722800FA6F924BA8BF4FF4FA61B1F57A7F1A78DA
:10723800B8BF4FF47A71A1F57A71002A41F05681EE
:107248008B4ADFF844E282FB0130CB17C3EB6013B3
:10725800581C6FF0630C3EF910003EF913E00CFB6C
:107268000313A0EB0E0003FB00F382FB0312DB17F2
:10727800C3EB62139E440FFA8EFE07EE90EAB8EE57
:10728800E78A87ED038AB8F1000F40F0B2832B88B4
:107298005A0640F1FB807749774A91ED018AD2ED91
:1072A800019A92ED026A91ED034A92ED030A91ED7B
:1072B800029A92ED007AD1ED005AD7ED011A97EDB6
:1072C800002A6E4A6E4938EE445A79EEC63A77EE8D
:1072D800007A65EE233A75EEC96A75EE890A37EECB
:1072E800401A66EEA76AB0EE633AA0EE813A13F050
:1072F8000303B0EE665A78EE044A79EE867AA0EE79
:10730800815AF0EE638AA4EEA73AD4EEA78AA4EED7
:10731800E75A33EE263AF0EE687AF0EE674AF6EE70
:10732800008A35EE88AAE0EEC14A28EEC33A35EE67
:10733800635A77EE293A77EEE67AAAEE233A25EEF3
:10734800285A76EE403A34EE49AAE0EE817A74EE95
:10735800A64AAAEE235A34EE094A37EE697A64EE51
:10736800A84A63EE036AE4EE074A75EEC85A36EE99
:10737800006A67EEA87AB0EE667A95EE057AE5EED1
:10738800056AE5EE867AB1EE648AF0EE665AF0EEAA
:10739800476AB1EE674AE8EE246A63EE270A67EEA9
:1073A800A43AE4EE275AB1EE450AB0EE609AB0EE80
:1073B800631AA4EE277A23EE244AE7EEA76AA5EE1D
:1073C800249AA0EE031AE8EE245AB0EE448A31EE6D
:1073D800A16AE0EE240AA5EE278A66EEA16A72EE9B
:1073E800028AE5EE033A61EE211A26EE096AA4EE56
:1073F800A47AA0EE274A0CBFD7ED022ADFED212A96
:1074080082ED005AA2EE256AE8EEA06AE2EE081ABA
:1074180073EEA33A27EE227A34EE044AF0EE005ACD
:10742800E3EEA26AA4EE226AA1EEA57AC7ED016A8C
:10743800C1ED366A81ED356A87ED006A81ED377AEC
:1074480082ED013AC2ED027AC2ED034AF3B987ED43
:10745800027A1BE0407D0308E6750020A026002084
:107468001C260020906700208C4D0020802A0020D8
:107478001F85EB5110140020D82000201021002077
:10748800C02300200000000074790020BAF1000F2A
:1074980040F0348129F0B8FA17B0BDEC068BBDE88E
:1074A800F08F079B1B78D9077FF5DEAD4FF40F707F
:1074B80021F01AFD00283FF428AE10F0BDFE4FF46D
:1074C8000F7021F0BDFC00283FF41FAE10F0B4FE91
:1074D8004FF40F7021F0B4FC0028EED115E6099B9B
:1074E8001B6898077FF51AADB5F8008018F0010FF2
:1074F80010D148F0010398452B800BD09A4B0222FB
:1075080014211A700E20FF2259709A7011F01CFB7A
:10751800B5F8008028F002039BB243452B803FF466
:1075280036AD914B02201421FF2218700E2059709D
:107538009A7011F009FBB5F8008028E522F48073F1
:107548009BB29A422B807FF46BAD884B1B78082B3B
:107558007FF475AD2A8822F040039BB29A422B80B3
:107568003FF470AD804B022214211A700E20FF22C6
:1075780059709A7011F0E8FA64E5059B5A8B9142AC
:10758800C0F2E184B1F5FA6FD4BFC2EB0101C2F5D4
:10759800FA614FF47A7303FB01F175480378C2F579
:1075A800FA62B1FBF2F1002B3FF44AAE4378714A1C
:1075B80001FB03F182FB0123C917C1EB63113FE60D
:1075C800DFED6D7AFFE5B1F5FA6F80F2B584187AD0
:1075D8008B1A03FB00F3C2F5FA6293FBF2F3C3F1D3
:1075E800640307EE903AF8EEE77A9FED647A644B0D
:1075F80067EE877AC3ED007AA4E51B780693002B23
:107608007FF490AD5F4A1268002A3FF48BAD5E4A62
:10761800079212F8030CDFF8A4B11146D71E28F020
:1076280069FF9BF80090079A002800F00C86069BDB
:10763800B9F1000F53D107F10801787928F05AFF02
:10764800002841F031855149B87A28F053FF0028C5
:1076580000F00C86B9F1020F41F02E854C49F87BF9
:1076680028F048FF002841F023854A49387D28F052
:1076780041FF002800F00C86B9F1040F41F02C8579
:107688004549787E28F036FF002841F02185434996
:10769800B87F28F02FFF002800F00C86B9F1060FFC
:1076A80041F012853E4997F8230028F023FF00286F
:1076B80041F006853B4997F8280028F01BFF002871
:1076C80000F00C86B9F1080F41F0DB84364997F8D1
:1076D8002D0028F00FFF00283FF424AD09231A4697
:1076E80002EB82021744314A7878B9788BF8003077
:1076F8001070517016E5DFED207A46E50C9B19787D
:107708000B9B01F001011868FEF7DEFE17B0BDEC17
:10771800068BBDE8F08F13B9089A01239370244BA8
:10772800089A1D7892F8214007931B2028F01AFF29
:10773800012C05F00108814600F0488705F0020594
:10774800089A1C4E92F82030DFF874A01A4F099559
:107758009346052B00F2B487DFE813F0BC00B200B3
:107768003400FA00FC00EF00FC3500204443002000
:10777800802A00201F85EB51000000000AD7233C17
:107788001C260020E8750020AE350020B835002002
:10779800BD350020C2350020C7350020CC3500207B
:1077A800D1350020D6350020DB350020EC750020CF
:1077B800E57500206C790020B04F00200000002003
:1077C80020210020012C04BF05238BF82030B8F1BC
:1077D800000F12D0059B3088B3F918100022134609
:1077E80061F30F0260F31F4261F30F03049861F322
:1077F8001F430360032342600993B14DDBF8141063
:107808002A68914280F0108647F230510322CBF863
:107818001C108BF8202002200DF0B2FB16F022FC81
:107828002968DBF81C200A440421CBF818208BF8BF
:107838002010012C40F08A872A68DBF81810914242
:1078480080F03E879AF8000020B928F08BFE0028C7
:1078580040F036873A6822F002023A602A68738854
:10786800642101FB03234FF480600022CBF8103021
:107878008BF820208BF803200DF052FB9BF820306A
:1078880067E728F075FE012807D18D4D72882B68AF
:10789800642101FB0233CBF81030B9F1000F02D09C
:1078A800B379002B4BD1012C00F00A87844DDBF80B
:1078B80010102A689142C0F0568701238BF82030B7
:1078C800012C3AD0F379012B46D028F0D1FD9BF852
:1078D80020303EE7B8F1000FD3D1099D4FF4806006
:1078E800B9F1000F00F03C830DF032FB089A002339
:1078F8001361002D3FF47EA9284611F025F9069B57
:107908001E6816F480573FF47BA91D216D48FAF7CD
:1079180096FB00287FF474A96B4B03F1500A03E02F
:1079280004339A4500F0D2861A78262AF8D1997835
:10793800DA789142F4D2FFF765B9614D8EE728F005
:1079480097FD03224FF47A738BF82020CBF81C3074
:107958005B4D60E75A4D6CE728F08AFD032240F63C
:10796800B8338BF82020CBF81C30554D53E7574FD0
:107978003B78002B01F08982554BDFF86C81DFF8EA
:107988006CB1DFF86CA1059345465E4604909946B4
:107998000EE019F804109847032C28DC88B93B78C6
:1079A8002AF8020F01349C4205F1040580F248814F
:1079B800072CE1B23046DBF80430EADD984700B224
:1079C800EDE738F824206B88801A4FF47A719B1AF7
:1079D80001FB00F040F6CA0290FBF3F00844904225
:1079E80040F2EE23A8BF10469842B8BF184600B22E
:1079F800D5E71D213348FAF722FB28B100F03ABE3B
:107A08000436B4423FF443AC31782629F8D1B27831
:107A1800F3789A42F4D2089BDB78002B7FF437ACDA
:107A28002848FAF70CFBDFED2B7A002801F03582A5
:107A380038EE678A284A2949FDEEC87ACDED047ADE
:107A4800BDF910301B0382FB0302DB17C3EBA21244
:107A5800C9F57A731BB203FB02F343F30F334B44AC
:107A680007EE903AF8EEE77A0123C7ED037A0B7038
:107A78000DE4154B03E00433A3423FF43EAA197802
:107A88002329F8D19878DA789042F4D20D48FAF799
:107A9800D6FA00283FF431AA114B1B6813F40033BF
:107AA80041F0E68200220F4B1046995C142902F13E
:107AB8000C0201F0938101301828F6D1FFF71DBAA6
:107AC800185800207467002064690020286A002084
:107AD800A856002000007A44D34D62109426002056
:107AE800B8340020A0590308406A0020B85200208A
:107AF800BE230020DFF8F092DFF8F0A2AB4F0B9224
:107B080009F15A084FF0010B494619F8010C28F001
:107B1800F1FC00B399F8040099F8023099F803E0F1
:107B280000EB400107EB8101013BD1F8A02003EBFA
:107B38004303534493420ED097F8CC20C1F8A030A9
:107B48000BFA00F022EA00000B9B81F89CE0C1F8D8
:107B5800A43087F8CC0009F10609C145D4D1944B6B
:107B6800944A1B780B930A9BDFF884A212681B685F
:107B78000C93AAF19C094FF0000B9046DAF80430F8
:107B880083B31F7877B3DAF80820A8EB0202002A3B
:107B98000CDB99F8CC20012101FA0BF122EA010251
:107BA80008F5FA7189F8CC20CAF808100B9ACAB1FE
:107BB8009AF8002059780432D2B2002940F02E8376
:107BC80005990498098B30F9122001F1C800824206
:107BD80040F38E8599F8CC109A7841FA0BF3D907BF
:107BE80040F119860BF1010BBBF1040F0AF10C0AE5
:107BF800C4D1FFF787B96D4C94F896305BB1079BF9
:107C08001B78D80707D5049BB3F90620059B5B8B27
:107C18009A4200F3F28511216748FAF710FA002812
:107C280000F0A68294F89A302BB994F8943013B9DE
:107C38003223A4F89830012384F89A30FFF7E8B883
:107C4800DDF810905D4A06925D49126842F2010A19
:107C5800A1FB091B12EA0A0A4FEA9B1B00F0858266
:107C6800584D5948524C59492E780078267008705A
:107C78001EB156490E7886F001064C4C0F2184F847
:107C88002410002B00F01284059D514BB5F826C036
:107C9800B5F824E0059D109318462D8B00784D4BC0
:107CA800129594F8255009954B4D0495A3FB005364
:107CB8005B0803EB4303C31ADBB20F90CDF834C063
:107CC80002F480520C9304F128000BF59673CDF85A
:107CD800449097F80080DDF82490DFF818C10994E3
:107CE8003D4C0E91139200210A930896CDF81CE0A2
:107CF800089B002B00F03A83099B079D33F911205C
:107D08001FFA82FEAE454FEA410303D30D9DAE45EF
:107D180040F271835CF82120934580F03183E25E64
:107D2800BAF1000F40F0468301314145E25200F1BB
:107D38000600DDDB0E9A099C284B84F824200F2AC4
:107D480049460CBF01220022DDF8449084F8251032
:107D58001A7000F0B283224B1B491C4ADFF854B05A
:107D680008931C46042001230B7013700DF008F9CA
:107D7800DBF80030A1686268E3605B1A934284BF55
:107D8800002384F82130069B3C781E68002C01F003
:107D98008080059A134DB2F824E0178B0E4916F42B
:107DA8008056284640F0B283324634E0C023002093
:107DB8000146002018580020746700208C6F0020AE
:107DC800D34D6210C85900205C1B00205D1B0020A9
:107DD80019690020ABAAAAAAEE5B0020465300202E
:107DE80030460020746A0020C5340020204D030866
:107DF8005C2400201C690020437803EB830303EB19
:107E0800830303F2EE239BB20132A24221F8023B24
:107E180000F102000ED015F81230002B00F0EF82AE
:107E2800022BE9D001320B8821F8023BA24200F173
:107E38000200F0D1109A137801331370FEF7C1BE17
:107E4800D74CD4F88830A9EB0303002BFEF6C7AE55
:107E5800D44AD54B527C059933F812308A7DDFED30
:107E6800D36A9FEDD36AC97D9BB207EE102A07EE4D
:107E7800903AB8EEC77AF8EEE77A27EE267A67EEF8
:107E8800867A0B9AC4F88820C7EE876A40F2FF32D8
:107E9800FCEEE67ACDED077ABDF81C30934228BF98
:107EA800134609B1D31A9BB2C248C34D0178C34CDB
:107EB80035F81160226825F81130921B13440131FE
:107EC800BF4D236001F00F021B0902702B80FEF7E3
:107ED80086BEFDF741FCBB4BBB4A1B68C31A9342E5
:107EE8007EF77DAEB64B00221A80FEF778BE059A63
:107EF8000499537DD27D013B31F913301AB1C3F592
:107F08003B6308331BB2A3F57A7307EE903A9FEDF3
:107F1800AF7AAB4AF8EEE77A40F2FF3167EE877A3C
:107F2800FCEEE77ACDED077ABDF81C308B4228BF0E
:107F38000B461380FEF753BE1B7AC3F1640307EEAA
:107F4800903AFFF750BB4146FFF727BB0221A048F4
:107F5800FAF775F800283FF4DDAA2F80FFF713B869
:107F68000CF0DEFFC2E49B4AB2F90030002BB8BF28
:107F78005B42B3F5E17FBFF646A8B2F90230002BA9
:107F8800B8BF5B42B3F5E17FBFF63DA8924B93EDD6
:107F9800096AD3ED076A93ED057AD3ED037A76EE95
:107FA800866A77EE877A76EEA66AB7EE007A37EEBB
:107FB800666A77EEA77AB0EEC66AF0EEE75AB4EED4
:107FC800E56AF1EE10FAB4BFB0EE655AB0EE465A63
:107FD800B5EE405AF1EE10FA40F0DF839FED7F7A5C
:107FE800B4EEE56AF1EE10FA44BF9FED7D6A36EE15
:107FF800477AB7EE006AF4EEC66AF1EE10FAC8BF27
:10800800DFED786AF5EEC07AC8BF36EEC77AF1EED2
:1080180010FA48BFB1EE477AF6EE007A27EE677A93
:10802800DFED6F7A77EE276ABDEEE66A16EE103A54
:108038002033402B40F28A86DFED6B6A6B4ADFED16
:108048006A7AC2ED006AFDEEC76AC2ED017A16EEE1
:10805800903A2033402BC2ED027A49D8DFED617A9D
:10806800B4EEE77AF1EE10FA41F34E809FED606AC4
:10807800DFED606A01E0B0EE677AB4EEE67AF1EE21
:1080880010FA77EE467AF6DC9FED5B7AF4EEC77A63
:10809800F1EE10FA41F124809FED556ADFED576A41
:1080A80001E0F0EE477AF4EEE67AF1EE10FA37EEF8
:1080B800867AF6D4DFED4A7AB4EEE77AF1EE10FA72
:1080C80040F3C486DFED477A37EEC77A27EE076AB2
:1080D800DFED4B5ADFED4B6ADFED4B7AE6EE256AB2
:1080E80067EE065AE6EE267AA5EEA77AF0EE477A0C
:1080F800464BC2ED037A1A6812F4003240F09E86AD
:10810800434B1046995C0A2902F10C0200F08E8557
:1081180001301828F6D1FEF776BF27F040039BB24E
:10812800BB422B803EF468AF3A4B022214211A70EE
:108138000E20FF2259709A7010F006FDFEF75CBF02
:108148002B8823F00407BFB2BB422F803EF44AAF0E
:10815800304B022214211A700E20FF2259709A7097
:1081680010F0F2FC2F88FEF73DBF2B490E787FE513
:1081780094F89430002B3EF44BAE079B1B7813F019
:1081880001037EF445AE012284F8943084F89520EA
:10819800FEF73EBE024C012184F88C10FEF7ABBD01
:1081A800C023002060570020805700200000C842EC
:1081B800000080444F5A0020545A0020505A002092
:1081C80024770020E024002060E316006F12833F2C
:1081D80074670020644F0020E8200020A7DFA8343F
:1081E800DB0FC93FDB0F49400000000010140020DE
:1081F800DB0FC940E4CB1641DB0F49C0E4CB16C105
:1082080092E741B99730083C15A82ABEB834002037
:10821800A0590308FC35002001460020012900F080
:10822800238599F8CC20012303FA0BF30BF1010BFA
:108238001343BBF1040F89F8CC300AF10C0A7FF420
:108248009DACFEF75FBE511D787928F053F90028E0
:108258003FF4F9A9B9F1010F40F0268707F10D01A4
:10826800B87A28F047F9002840F02687C149F87BFA
:1082780028F040F900283FF4F8A9B9F1030F40F0BD
:108288001787BD49387D28F035F9002840F0248744
:10829800BA49787E28F02EF900283FF4F8A9B9F1F8
:1082A800050F40F01587B649B87F28F023F9002854
:1082B80040F00A87B34997F8230028F01BF90028F3
:1082C8003FF4F8A9B9F1070F40F0FA86AE4997F8DC
:1082D800280028F00FF9002840F0D386AB4997F81A
:1082E8002D0028F007F900283EF41CAFB9F1090F5A
:1082F8003EF418AFFFF7F2B948F0020343452B806C
:108308003EF445AEA24B022214211A700E20FF2221
:1083180059709A7010F018FCB5F80080FEF737BE57
:108328005D2A00F07D825B2A00F0D8855E2A00F085
:108338006B86562A00F06C86972A00F0A686A72A34
:1083480000F05686934D2B889E0740F01586A2F1C3
:10835800B703072B00F29E82DFE813F08E029C021F
:108368009C029C0280029C0272027202079B002BF4
:108378003FD05CF8212093454FEA4103FFF4CFAC8E
:10838800854A854DD25C05EB030E002A00F0B180CA
:10839800022A47D19EF8012002EB820202EB8202F8
:1083A80002F2EE2292B2032933DD12B2BAF1000FC3
:1083B8003FF4BAAC0C9D20F81520B9F1000F03D199
:1083C8000F9D022D7FF6B0ACB0F802900288B0F88D
:1083D80004E04A449644714A0FFA8EFE82FB0E521C
:1083E8006F4DA2EBEE7225F803E012B24FF00109CF
:1083F8009AE41A464B000A9D4CF8215090E4D3B2F7
:10840800022B04D9032B7FF40DAD7346FCE43B46E5
:10841800FAE4012505FA01FE0E9D25EA0E0512B2C1
:108428000E957DE4E25ABEE75E4A1278002A7FF490
:10843800EBA9B8F1000F3FF4E7A9012C40F0408107
:108448009BF82030FFF785B931465748F9F7F7FD13
:10845800002800F0D38084F8936016F02FFAFEF716
:10846800A1BC47F04003BB422B807FF45DAEFEF712
:10847800C3BD47F004039F422B800AD0444B02221D
:1084880014211A700E20FF2259709A7010F05CFBAC
:108498002F88464B464AB3F90430464982FB03020B
:1084A800DB17C3EBA2030B80FEF79CBD424B434A8C
:1084B800109201221A70424B04931B213A48F9F793
:1084C800BEFD00287FF447AC3E4BDFF8FCB00893B4
:1084D8001946DBF80030CA688B609B1AC82B00F27B
:1084E8000185069B1E6806F48056A3E45B78FFF7B7
:1084F8005EB8CAB2022A40F2B483032A92D1129A11
:10850800139D079E002D08BF32464CE700220FE05E
:10851800437803EB830303EB830303F2EE239BB25D
:108528000132A24221F8023B00F102003FF482AC82
:1085380015F812301BB1022BEAD00B88F0E7D3B242
:10854800032BFAD83B46EBE7B2F5FA7FFEF656ACBA
:1085580094F89230002B7EF451AC079B1B780121D4
:108568000B4084F8921000F0D98315F07BFDFEF7DC
:1085780045BC00BFBD350020C2350020C7350020EE
:10858800CC350020D1350020D6350020DB35002041
:10859800FC350020B44F0020746A0020565555550C
:1085A800302400205826002074670020644F0020E3
:1085B80067666666962600204653002019690020E3
:1085C800EE5B002030460020185800200025FFF7F9
:1085D800B7B8B2F5FA7FFEF611AC94F89230002BDA
:1085E8007EF40CAC079A1278012184F89210D10716
:1085F80000F1428416F062F9FEF700BC079BBA4A04
:108608001B781060D8077EF5D1ABB84B1B78002BD0
:108618003EF4F4AB089BDB78002B7EF4EFAB94F8C8
:1086280093300133DBB2032B84F893307EF6E6AB4C
:10863800AF4B5B7813B9002D7EF4E0AB15F012FD5B
:10864800FEF7B0BBAB4AAC491068B4F99020C669D4
:1086580081FB06018911F617701A00F5FF407F307B
:1086680082423EF792AB891B0A4412B2A4F89020CA
:10867800FEF78BBB089BDB78002B7FF4C5A9DFEDE9
:108688009F7A9D4938EE678AC9F5FA63FDEEC87A84
:108698001BB2CDED047ABDF91020120381FB020153
:1086A800D217C2EBA11203FB02F343F30F334B447F
:1086B80007EE903AB8EEE78A87ED038AFFF7A4B988
:1086C800099D002D3EF496AAFFF716B98C4A059B22
:1086D800D588049A1B8BB2F906105A1B914240F3B5
:1086E80089802B449942B4BF00250125FEF793BA2F
:1086F800C8398A4242DA99F8CC109A7841FA0BF3D1
:10870800DB073FF56FAA524201200D9210F002FBE1
:108718007B1E0D9A162B00F25181DFE813F023021D
:1087280037020A025C024B027002F501E001CB013C
:10873800B601A1014F015C028E017002F501E00152
:108748007A01660152013F0129011501AB460899DA
:10875800DBF80020CB69099D13448B61002D3EF4A2
:1087680049AAFFF7C9B827F083FE032140F6B832BB
:108778008BF82010CBF81C20FFF74DB899F8CC30B7
:10878800012202FA0BF223EA020308F5FA7289F8C9
:10879800CC30CAF80820FFF725BAB4EEE56AF1EE46
:1087A80010FA8CBFB0EE654AB0EE464AC4EE054AF0
:1087B8009FED542A9FED545ADFED541ADFED542AE9
:1087C8009FED543ADFED543A9FED544AA4EE825A95
:1087D800E4EEE12AA4EE857AA4EEA23AB0EE475A76
:1087E800B0EE637AA4EE837AA4EE874A84EE057A23
:1087F800FFF7F6BB0125FEF70EBA00214848F9F746
:108808001EFC00287FF407AA322384F89600A4F8F7
:108818009830FFF700BA002A0CBF0120022074E745
:10882800404B002201204049404C0B60404B0993CB
:10883800404B2270404D0A9310F06CFAFEF7E3BAF1
:108848003C4A3A4B0A9211463C4A0A6002225A7044
:10885800374B099327F0E8FEFEF7D5BA354A334B74
:108868000A921146364A0A6000225A70304B099320
:1088780027F0DAFEFEF7C7BA2E4A2C4B0A921146A9
:10888800304A0A6001225A70294B099327F0CCFE1E
:10889800FEF7B9BA792A00F08C847A2A00F07E842F
:1088A8009E2A00F073849D2A00F06884AE2A00F0A6
:1088B8005D84AD2A00F05284EF2A00F04C84FD2A32
:1088C80000F03784FB2A00F09D84FE2A00F097848C
:1088D800F72A00F091847B2A00F07684144B0993E0
:1088E800144B0A93FEF78FBAE04B00200146002094
:1088F800B867002000790020D34D621000007A4448
:10890800D855002099FB243F69A2163E39094E3DEF
:10891800E3B59E3E88FA163E45FE7F3FA7DFA834A2
:1089280074670020B03C0020B84F00209B4900200D
:10893800584F0020BC4F0020B44F00209C5200200C
:108948008452002090520020D9F8D000B64B90F8FD
:1089580036109B7811446429A8BF642121EAE1718B
:1089680080F83610002B40F0918419F047FE58E447
:10897800D9F8D000AC4B90F837109B781144FE29F9
:10898800A8BFFE2121EAE17180F83710002BECD056
:10899800162027F02FFED9F8D000E6E70C98A24B56
:1089A80041781144B1F5967FA8BF4FF4967121EA3A
:1089B800E17141709B78002B40F06184D9F8D000B8
:1089C800D3E7D9F8D000984B81781144C829A8BFBB
:1089D800C82121EAE17181709B78002BC5D0142051
:1089E80027F008FED9F8D000BFE7D9F8D0008E4BA1
:1089F80041781144C829A8BFC82121EAE171417012
:108A08009B78002BB1D0132027F0F4FDD9F8D000C3
:108A1800ABE7D9F8D000844B01781144C829A8BF26
:108A2800C82121EAE17101709B78002B9DD01220AA
:108A380027F0E0FDD9F8D00097E77B4B0C989B789E
:108A4800417911446429A8BF642121EAE171417187
:108A5800002BB3D00E2027F0CDFDD9F8D00084E745
:108A6800D9F8D000704B017A9B781144C829A8BF67
:108A7800C82121EAE1710172002B3FF476AF0B2087
:108A880027F0B8FDD9F8D0006FE7D9F8D000664BC9
:108A9800C1799B781144C829A8BFC82121EAE1718E
:108AA800C171002B3FF461AF0A2027F0A3FDD9F86C
:108AB800D0005AE7D9F8D0005B4B81799B781144F4
:108AC800C829A8BFC82121EAE1718171002B3FF4B0
:108AD8004CAF092027F08EFDD9F8D00045E7D9F82A
:108AE800D000514B417993F802E01144C829A8BF3E
:108AF800C82121EAE1714171BEF1000F40F0AD8358
:108B0800112F7FF461AF30E7D9F8D000464B0179D7
:108B180093F802E01144C829A8BFC82121EAE171ED
:108B28000171BEF1000F40F08E83102F7FF460AF0B
:108B38001BE70C993C4B0F790D931744642FA8BF82
:108B4800642727EAE7770F7127F06EFD0D9B9B7866
:108B5800002B3FF433AF0320394627F04BFDD9F8FB
:108B6800D00002E70C98304B01781144FA29A8BFCD
:108B7800FA2121EAE17101709B78002B3FF41EAFC6
:108B8800012027F037FDD9F8D000EEE60C98264BE7
:108B9800817811446429A8BF642121EAE1718170B8
:108BA8009B78002B3FF40AAF022027F023FDD9F869
:108BB800D000DAE60C981C4BC1799B78114481F3FC
:108BC8000801C171002B3FF4F9AE052027F012FD12
:108BD800D9F8D000C9E60C98134B817993F802E0D4
:108BE80011446429A8BF642121EAE1718171BEF1B1
:108BF800000F40F03C830D2F7FF420AFDEE6D9F85C
:108C0800D000094BC17893F802E01144C829A8BFE5
:108C1800C82121EAE171C170BEF1000F40F009835B
:108C28000F2F7FF4F9AEA0E61E770020B549D1F8E2
:108C380000E04200BEF1000F08D0171803EB8707C9
:108C48009EF801E07F787745BEF4DDA91044AE4F69
:108C5800AE4A03EB800300200B6038801060FEF7FB
:108C6800D2B9129AFFF79FBB04999B7831F9122069
:108C7800B2F5617F4FF4966191FBF3F3C0F2F38094
:108C880040F633019142A8BF11460C2FA1F561713E
:108C980091FBF3F100F0CB81182F7FF4C2AAC9B27F
:108CA800C8290B46A8BFC823D9F8D020D77DD8B289
:108CB800B8423FF4B6AADF1B954BD07548BF0737BB
:108CC800FF109B780137FFB23BB9002F3FF4A9AAE8
:108CD800384610F01FF8FFF7A4BA182027F08AFCCE
:108CE800F3E78C4A8C4B099210461A688B494FF46B
:108CF8007A73B3FBF2F3C3EB431203EB820302680C
:108D0800DB00A1F8A83053077EF57AA8844B854D7F
:108D18000A221A80844B0A93FEF775B883490968BA
:108D280011F4003140F09D81814B08465D5C0F2DA8
:108D380001F10C016DD001301828F7D1FA3A00235F
:108D4800A4F8902084F89230FEF758B8B4EEE77A89
:108D5800F1EE10FA40F3DF81DFED765A9FED766A87
:108D680001E0F0EE676AF4EEC66AF1EE10FA76EE0C
:108D7800E57AF6DCDFED716AF4EEE67AF1EE10FAE8
:108D880040F1C681DFED6B5A9FED6D6A01E0F0EEB0
:108D9800667AF4EEC67AF1EE10FA77EEA56AF6D4A2
:108DA800DFED687AF4EEE76AF1EE10FA40F3148129
:108DB800DFED657A77EEE66A66EEA65A9FED635AAE
:108DC8009FED636ADFED637AA5EE856A26EEA55A04
:108DD800E5EE867AE5EE276AFFF730B94949D1F81A
:108DE80000E04200BEF1000F08D0171803EB870718
:108DF8009EF801E07F787745BEF47FA80244424F91
:108E0800424803EB820300220B603A800260FEF7BF
:108E180074B83C490F68450037B12E1803EB860635
:108E28007F787678BE4289D20544374E374803EBBF
:108E3800850300250B60358005607FE7464B1B786E
:108E4800032B00F02D810022FFF75AB9DFED437A9A
:108E5800B4EEE77AF1EE10FA44BFDFED387A37EE78
:108E6800C77AFFF733B90C2F00F0F880182F7FF47A
:108E7800D8A900210B4617E7394A264913602A4B1F
:108E88000991284D0A93FDF7BEBF364A0592FEF7B1
:108E9800D9BE06F48056FEF7CDBF38EE678A324B4E
:108EA80032491870FDEEC87AC9F5FA63CDED047A37
:108EB800BDF91020120381FB0201D217C2EBA112E7
:108EC8001BB203FB02F343F30F334B4407EE903A14
:108ED800F8EEE77AC7ED037AFEF7D9B9244B0122F9
:108EE8000220A0E4234A069B1E68136823F00403AB
:108EF8001360089A012306F4805682F82130FEF7A1
:108F080099BF00BF14260020002700200427002056
:108F18001E770020584F00207C6F0020046D002031
:108F28008E790020B44F0020BC4F0020B8340020B8
:108F3800A0590308DB0FC940E4CB1641DB0F49C039
:108F4800E4CB16C1DB0FC93FDB0F494092E741B9BB
:108F58009730083C15A82ABE3C770020DB0FC9BF14
:108F6800E04B0020A856002094260020D34D621024
:108F7800FE3C0020B04F00200023BB2A149300F0D1
:108F88002E81B72A00F02781BE2A00F02B81BD2A46
:108F98007FF480AC4FF6FE71BF4AC048D68909906D
:108FA800908933440144D38191811FF0B7F8F8F7D1
:108FB80051F91FF09BF8FBF7FFF801200FF0AAFE0C
:108FC800B4F89030B64A0A92FA3B0022A4F89030DE
:108FD80084F89220FDF717BFDFEDB27AF4EEE76A66
:108FE800F1EE10FA44BFDFEDB07A77EEE66AE3E619
:108FF800AE4AAA4B09931378AD4D43F0040313709E
:10900800A74B0A93FDF7FFBEAA4B022203200AE4EE
:109018001FF084F8F8F71EF91FF068F8FBF7CCF892
:1090280001200FF077FE94F88E20FFF785B9CFB2B4
:10903800A14B0E915B78BB423FF4F3A89F4B0D9375
:1090480038460AF045F80D9B0E999B781BB1C9B2BA
:109058000C2027F0CFFA0137FFB236E60027394651
:10906800E6E797490978032900F0BE8019465BE6D0
:10907800934B1B78032B7EF415AD0FF049FDFDF7DC
:109088003CBF08231A46FEF72BBB8E4B834A099236
:109098004FF4C8721A80824B854D0A93FDF7B3BE10
:1090A8000FF036FDFDF7AFBF01231A46FEF718BBD8
:1090B80003231A46FEF714BB02231A46FEF710BB19
:1090C80007231A46FEF70CBB06231A46FEF708BB11
:1090D80005231A46FEF704BB04231A46FEF700BB15
:1090E800B0EE677AFEF7E6BF002D3DF4D8AD764CBA
:1090F80094F88D30002B3DF403AE0FF009FD0023EA
:1091080084F88D30FDF7FCBDF0EE477AFEF7BCBF62
:10911800F0EE676A44E6F0EE667A2BE65F4B099359
:109128005F4B84F8941084F89500614D0A93FEF71C
:1091380063BD0021012009F0E9FEB4F89030574AD8
:109148000992963B564AA4F8903000230A9284F874
:109158009230FDF758BE00210846ECE7FF210020B9
:1091680025F0CAF894F88E20FFF7A6BB012100204D
:1091780025F0C2F894F88E20FFF79BBB0021FF2052
:1091880025F0BAF894F88E20FFF790BB0021012053
:1091980025F0B2F894F88E20FFF785BB4B4A3F4B79
:1091A8000993137A43F0010313723D4B0A93FDF7B9
:1091B8002ABE464A394B0993137A23F001031372E6
:1091C800374B0A93FDF71FBE4FF4FA61022009F0EE
:1091D8009DFEFFF783BB19464FF6FE73DCE6194682
:1091E8000223D9E60221D7E60FF092FCB4F99020C9
:1091F800A4E50B20FDF700BE002104209BE7002119
:10920800032098E70021022095E72F4C14F02AFF4D
:10921800002384F88D30FDF773BD002B3FF467AF52
:109228002B492C4A09684FF47A7000FB031313602A
:109238005DE70F200E930D9227F0DCF9D9F8D000E6
:109248000E9B0D9AECE410200E930D9227F0D2F9A4
:10925800D9F8D0000E9B0D9A67E411200E930D9259
:1092680027F0C8F9D9F8D0000E9B0D9A48E40D20D4
:109278000E930D9227F0BEF90E9B0D9ABBE41520B4
:1092880027F0B8F9D9F8D000FFF76FBB172027F0FF
:10929800B1F9FFF793BB00BF98670020584F002033
:1092A800BC4F0020DB0FC9BFDB0F49C01C77002073
:1092B800B44F00204C3D00209B4900201E77002021
:1092C8003C77002090790020C02300202C530020F8
:1092D80018580020DC4B00202DE9F047C74C636884
:1092E80020469847002800F0C380C54B1B78012210
:1092F800042B84F83C2000F0BD80B4F91610B4F9B2
:109308001820B4F91A3021636263A363BD4B1B882C
:10931800002B69D0BC4DD4ED0C7AD5ED004A95ED03
:10932800050A95ED015A95ED067AD5ED035A95EDA6
:10933800026AF8EEE76AD5ED047AA4EEA60AA5EE6D
:10934800267A67EEC07AA5EEC07AE6EE267A85ED33
:10935800057AC5ED067A2AF0DFFBD4ED0D6AD5ED66
:10936800094A95ED0E0A95ED0A5A95ED0F7AD5ED55
:109378000D7AD5ED0C5A95ED0B6A2063F8EEE66A86
:10938800A4EEA60AA5EE267A67EEC07AA5EEC07A04
:10939800E6EE267A85ED0E7AC5ED0F7A2AF0BCFB4B
:1093A800D4ED0E6AD5ED124A95ED170A95ED135ACC
:1093B80095ED187AD5ED167AD5ED155A95ED146A0E
:1093C8006063F8EEE66AA6EEA40AA6EE857A67EE72
:1093D800C07AA0EE657AE6EE867A85ED177AC5ED55
:1093E800187A2AF099FBA063884FA17F884812F069
:1093F800D1FA3B88002B40F08480864ED6F8E050A6
:10940800854B1B685B0743D4B5F90070216B636B10
:10941800A06B824A824E92ED026AD2ED006AD2EDCA
:10942800015AC91B2163B5F90270DB1B6363B5F9E7
:1094380004703568C01B07EE900AB8EEE75A07EECD
:10944800901AB8EEE77A07EE903AF8EEE77A36EE39
:10945800056A36EE877A77EEA57A0135A06382ED44
:10946800026A82ED007AC2ED017A3560BDE8F087C4
:10947800BDE8F0876B4BB4F91600B4F91810B4F9CD
:109488001A2018802063598061639A80A2633DE79F
:10949800B6F89820322A00F08880002A66D196F81B
:1094A8009530002BB0D06048D6F8FC205F4980FB8F
:1094B8000273D217C2EB23122A80D6F8002180FB50
:1094C8000273D217C2EB23126A80D6F80431A78A36
:1094D80080FB0302DB17C3EB2213DB1BAB800023EB
:1094E800CB6086F895301EF019FEF7F7B3FE1EF034
:1094F800FDFDFAF761FE01200FF00CFCD6F8E050F4
:1095080082E7444E226BD6F8E050B3F5C87F4FF09F
:10951800000323632B80398818BFD6F8E400B7F816
:10952800008008BF0020B1F5C87F18BFD6F8E83022
:10953800616B02440B440020B8F5C87F6063C6F82D
:10954800E420C6F8E830688052D0D4F838E0D6F87D
:10955800EC10A0637144B8F1010FA880C6F8EC10B4
:1095680068D008F1FF38A7F8008049E7D6F8FC0072
:10957800236B00210344C6F8FC3021632980D6F808
:109588000001636B61630344C6F800316980A36B13
:10959800D6F80401A1630344012AC6F80431A9805E
:1095A80075D0013AA6F8982079E72B8820491F48FA
:1095B800276BA6F8F0300023B5F802E0B5F804C030
:1095C800C0684B608B602363C6F8FC702B80616BAE
:1095D800C6F8001163636B80A16BC6F80411A3631E
:1095E800A6F8F2E0A6F8F4C0C6F8F800AB80D8E711
:1095F800A36BC6F8EC30A063A880B2E76C4F0020DC
:10960800044C0020044400200844002090790020E5
:109618009C4F0020C02300208C6F00204079002040
:109628003C790020084C00201F85EB5198670020EA
:10963800BC240020DFF804C1DFF8F0E0C8328CFB5E
:1096480002A9C833D217C2EBE9128CFB03A9DB17B6
:10965800C3EBE913C8316B802A808CFB013CA28ADA
:10966800CB17C3EBEC139B1AAB80CEF80C001EF0A3
:1096780055FDF7F7EFFD1EF039FDFAF79DFD404661
:109688000FF048FBB7F80080D6F8E05069E7254BA3
:1096980086F89A101B6886F8942013F4003334D1A6
:1096A80019462148475C0B2F01F10C0110D00133FA
:1096B800182BF7D1B6F8F0101C4B2980B6F8F270C9
:1096C800B6F8F400D6F8F8106F80A880D96068E77B
:1096D800174FD7F800C05900BCF1000F09D001EBB3
:1096E800030E00EB8E0E9CF801C09EF801E0E645E3
:1096F800E0D20B44DFF848E00E4900EB830000237A
:109708003860AEF800300B60D4E70B4B1B78032BA6
:1097180001D00B46C5E70FF0FBF9D6F8E050B6F8D4
:109728009820C7E7B8340020A0590308986700209C
:1097380014260020042700203C7700201F85EB51C9
:10974800002700202DE9F0478C4B1B78DB070746E4
:1097580044D58B4B8B4D1C788B4E012C59D01CD388
:10976800022C07D189498A4A09881288914201D96D
:1097780001241C70EB7AE3B12B89D3B1854B1B789C
:10978800BBB109F0C7FC002800F09B802B7B83420B
:109798002CBF0121002131700CE07C497E4A0988E8
:1097A80010886A7B801A8842E2DAEB7A0024002B60
:1097B800E2D131782A79632A06D8022C774E00F054
:1097C800BA803378002B5DD1754AAB7A8C4238BFAA
:1097D8000C461470002B4CD1BDE8F0876B4B694DDB
:1097E80019885B88E878CB1A83EAE3728142A2EB96
:1097F800E3721DD32B788B421AD3614B1C78E01E81
:10980800012861D96749097802294FD0012C5E4E99
:10981800A5D15F4A5D491288687B0988121A91426E
:1098280039DD5D4A12888A42A4D200241C70A1E75F
:10983800B1EB400FE1DC524B1C78E11E012940F2EC
:109848009480022ADEDC57494F4E0878DFF84481BD
:10985800DFF844C1DFF838E100210324022834701E
:109868001C7088F80010ACF80010AEF8001081D118
:109878001FE0012C71D0022C0BD10720BDE8F04766
:109888000FF062B97068381A474B984258DD727009
:109898009AE7BDE8F08702241C706BE7022AD2DD44
:1098A8004049097802294FF0040464D13949364EF9
:1098B80009783E48022ACCBF00220122C28081805A
:1098C8004BE70221317075E7022A9BDC95F800C04E
:1098D80091FBFCFC0CF1010CBCF1080FDFF8B4A003
:1098E800304EA87895F801E096F800802A4CDFF809
:1098F800A090254EA8BF4FF0080C8AF800C01FFAA8
:109908008CFA10FB0AF01EFB0AFE80B2DFF88CA06E
:109918002080A9F800E000244FF0640EB8F1020F8F
:1099280034701C70CAF804408AF801E07FF439AF3B
:109938000FFA8CF1BDE73078A0B901237760337056
:10994800C2F164021A4B00FB02F083FB0023C0172C
:10995800A0EBA3506430707036E70820BDE8F047EC
:109968000FF0F2B87368F81A8EE7032C96D10D49F8
:10997800097802299AD0044EFCE600BFE57500205C
:10998800782A0020484F0020882A0020244D0020F3
:109998007C2A00208A4D00207A2A0020802A002074
:1099A8003C770020044C00207F969800084C00204B
:1099B8006BCA5F6B2DE9F04F95B0B0F908500D8177
:1099C800EDB2442D00AF0C46904600F0D182064619
:1099D80043D9812D00F0068200F29980542D00F0C1
:1099E800CE8040F228816E2D00F09082802D40F0CC
:1099F8002581C44B93F800A00AF1020A1AF0FF0A65
:109A080000F09980C04BDFF83483C04EDFF830B3E4
:109A18009A4403F101090A2516E0322D00F09583D6
:109A2800A5F13C00C0B2132840F2958300232268B8
:109A3800511C216015702268CA4502F1010121609C
:109A4800137078D019F8015B0A2DE6D1BBF8003005
:109A5800FF2BA8BFFF23DBB2E9E7052D00F07682D4
:109A680020D8022D00F0838040F29B81032D00F066
:109A78004482042D40F0E280A54920462A46F7F7A3
:109A8800B3FE00212046F7F7DDFE22680021531CB3
:109A98000125236028462B46543711706381BD4643
:109AA800BDE8F08F242D60D040F20D81282D00F004
:109AB800E681382D40F0C2800A68964B0125511C7A
:109AC80021601570226805215019206011702268E4
:109AD8000A21501920601170226800215019206055
:109AE800117022681978501920601170226859780D
:109AF80050192060117022689978531923602B46F9
:109B08001170284654376381BD46BDE8F08FA02DFB
:109B180019D040F21B81B82D00F0ED81FE2D40F0E8
:109B28008D807D4D05F1080635F8021B2046F7F7B4
:109B380089FEAE42F8D101252B4628465437638169
:109B4800BD46BDE8F08F754B08461968F7F763FE08
:109B5800734B20461968F7F75EFE724B196820466A
:109B68000125F7F758FE2B46E7E76F4BF6E7042287
:109B78006E4920460125F7F737FE2B46C1E70B68EB
:109B8800DFF8C081591C012221601A702368002562
:109B98009A1822601D70236898F85520591C216076
:109BA8001A70236898F85420591C21601A70B8F864
:109BB80050102046F7F746FE23685A1C22601D7095
:109BC80023682822591C21601A70B8F852102046C0
:109BD800F7F738FEA8F1020508F14E0635F8021F1E
:109BE8002046F7F72FFEAE42F8D12268504B0D21E0
:109BF800501C20605D181170226813F8011F501C5A
:109C08009D4220601170F7D123680222591C2160FF
:109C18001A70B8F856102046F7F714FEB8F858101E
:109C28002046F7F70FFE0125B8F85A102046F7F737
:109C380009FE2B4665E7522D3FF427AF21462846FB
:109C48000AF06CF9034600287FF475AF742D00F014
:109C5800BB80772D0DD13268716891421EBF531CAD
:109C680033601178334A08BF194620460FF00CF9C3
:109C780061E7F52D01F00383472D00F0A581392D0B
:109C8800326800F0AA8200F2A082212D01F0B6828B
:109C9800292D40F0E382531C336013780A2B01F01E
:109CA8007A83502B41F0C7813046F7F78DFDDFF8F6
:109CB8009880A8F800003046F7F786FD0125A8F837
:109CC80002002B461DE7202DB8D10B681A4D591CF0
:109CD8006A7821601A7023682A78591C21601A70E2
:109CE8002368AA78591C21601A7029892046F7F739
:109CF800A9FD23686A79591C21601A702268A9791C
:109D0800C5E600BFE54B0020684D0308282A00205F
:109D1800A14900209B3C0020084C0020ACF7FF1F05
:109D2800B0F7FF1FB4F7FF1FE03D0020447E030893
:109D38000D770020DD7D0108484F002067666666C4
:109D4800502A0020B0760020042A0020822D7FF4BB
:109D580075AF0B688A4A8B4D11788B4A581C206066
:109D6800197011892046F7F76DFD884B22681B880A
:109D7800FF2B02F10101A8BFFF2321601370A9681E
:109D880081F3100189B22046F7F75CFD296801F3D9
:109D98000F0189B22046F7F755FD7D4B22681978E7
:109DA80075E6012D7FF44AAF0B680022591C21602B
:109DB8001A7023685A1C22601D7022682521531CC2
:109DC80023602B4611709CE63268716891421EBF71
:109DD800531C336011786F4A08BF194620460FF0AC
:109DE80053F8A8E66C4B1E78043616F0FF063FF4CD
:109DF800A2AE6A4BDFF8C8811E4403F1010A4FF096
:109E08000A0924E0B9F1500F00F09D81B9F15A0F09
:109E180000F0B681B9F1320F00F0B681A9F13C002B
:109E2800C0B2132840F2B3810025294623685A1C82
:109E38002260204683F80090F7F704FD2946204663
:109E4800F7F700FDB2453FF476AE1AF8019BB9F179
:109E58000A0FD7D1524B9D68196805EB85054FF657
:109E6800FF736D009D42A8BF1D469942A8BF1946C1
:109E780025EAE57521EAE171ADB289B2D6E70B684A
:109E8800DFF84091474E591C022221601A7023685E
:109E98004FF006085A1C226083F8008023680A22C3
:109EA800591C21601A70236801255A1922601D70F7
:109EB800B9F800102046F7F7C5FCB9F8021020469B
:109EC800F7F7C0FC23685A19226083F800802368DA
:109ED8005022591921601A702368002259192160EB
:109EE8001A7031882046F7F7ADFC71882046F7F7DD
:109EF800A9FC2B4605E62C4B30E60B685A1C0A6079
:109F08001D700B685A1C0A601D70BEE51F4B0A685D
:109F18001B881C4DFF2BA8BFFF23511C2160137009
:109F2800A96881F3100189B22046F7F78BFC1F4B13
:109F380020461988F7F786FC296801F30F0189B2D2
:109F480020460125F7F77EFC2B46DAE50B22184957
:109F58002046F7F749FC082216492046F7F744FC43
:109F68000125072214492046F7F73EFC2B46C8E591
:109F7800002A3FF4E0AD114B136001252B46C0E5E4
:109F88008A4D0020104D0020484F0020244D00200D
:109F98003C770020357E0108E54B0020784D03080A
:109FA800D0290020042A0020B8340020247700207B
:109FB8004C7E0308587E0308647E0308F93E0108B6
:109FC800142A002088670020726835687B62304652
:109FD800551BF7F7E2FB052D38627B6A01F2CE814B
:109FE8008026B346012594E80600521A103AB24278
:109FF800B8BF1FFA82FB944A396A92683A61521ACA
:10A008009345396A7B622046FA6088BF1FFA82FB53
:10A01800F7F701FC7B6A002B01F08E81002D41F0DF
:10A028000D812368C7F800D05D71C0B00533C7F84B
:10A0380004D0FB61BBF1000F01F013833B6A3A695E
:10A04800934281F00A833E6A7D62AA46A846BC60B4
:10A058008025FB68A3EB08087B4BB8F5807F9B68DD
:10A0680028BF4FF4807806EB08029A4288BFA3EB1A
:10A078000608F8F7A9F97C68424621463046F8F701
:10A088004FF8F969B86104EB000C0B787B61644503
:10A098002ED2DFF8C4910CF1FF3C04F1FF3E1EF80C
:10A0A800013F09EB830219F823405688ECB10023DD
:10A0B8004FF4004204F1FF3832424FEA520202D014
:10A0C8000878284308706D0806D10AF1010A4D7016
:10A0D8001FFA8AFA01318025D34503D8E6456CD3A7
:10A0E80043456ADB01339C42E6D1F445D7D1F96197
:10A0F8007B6ABA6913449BB2D3457B6206D97B6AF3
:10A108003A6A9846D6183B699E42A2D3BC68802D0D
:10A118001CBF0AF101031FFA83FA0AF1020189B28E
:10A128002046F7F78FFB2368796A01255A192260C0
:10A1380020461D70F7F786FB2368534423602B469F
:10A14800D7F800D0DDE4414B85E63388FF2BA8BF64
:10A15800FF23DBB26BE415F0FBFA00283FF466AC92
:10A1680003780A2B2FD8B0F9023088FB0312DB17CB
:10A17800C3EBA2039BB2FF2BA8BFFF23DBB256E4BD
:10A18800334A92E8220068E698E8220065E615F06E
:10A19800DFFA00283FF448AE03780A2B3FF644AEB6
:10A1A800B0F90430B0F9061003EB830383F35005CC
:10A1B80021EAE171ADB289B238E6FB69BC681A469A
:10A1C8003B7D1370A3E70023D8E7552D17D0572DF3
:10A1D80044D14FF0FF352B4693E4531C336013787A
:10A1E8000A2B01F0DF803046F7F7F9FA3046F7F727
:10A1F800F6FA01253046F7F7F2FA2B4681E4531CAC
:10A20800336092F80080B8F1FF0F01F06381B8F174
:10A21800FE0F01F0D6803046F7F7D6FA96E80C0024
:10A228009B1A002B07DD531C336013781BB9B8F158
:10A238000C0F41F28D81B8F1270FCAD8054B0125C3
:10A2480023F818002B465CE4FC190020082A00209B
:10A25800202A0020B0760020884D030870680B3D46
:10A26800811AEF2DB5D80FF2080E5EF825F000BF61
:10A278005BB10008DBA10008DBA10008DBA1000836
:10A28800DBA10008DBA10008DBA10008DBA10008B6
:10A29800DBA10008DBA10008DBA10008DBA10008A6
:10A2A800DBA10008DBA10008DBA10008DBA1000896
:10A2B800DBA10008DBA10008DBA10008DBA1000886
:10A2C800DBA10008DBA10008DBA10008DBA1000876
:10A2D80091B10008DBA1000805AE0008DBA1000869
:10A2E800BFAF0008DBA10008DBA10008DBA1000864
:10A2F80097AF0008DBA100083DAF0008DBA100080C
:10A308000BAF0008DBA10008E5AE0008DBA10008E0
:10A31800D3AE0008DBA100087BAE0008DBA1000873
:10A3280027AE0008DBA10008DBA10008DBA10008BC
:10A33800DBA100083F9B0008DBA1000869B000080A
:10A34800DBA10008DBA100084FB00008DBA1000872
:10A35800F5AF0008DBA10008DBA10008DBA10008BD
:10A36800DBA10008E9AF0008DBA10008DBA10008B9
:10A37800DBA100081BB10008DBA10008CDB0000874
:10A38800DBA10008DBA10008C3AD0008DBA10008C1
:10A39800DBA10008DBA10008DBA10008DBA10008A5
:10A3A800DBA10008DBA1000855AD0008DBA100080F
:10A3B80039AC0008DBA10008C7AB0008DBA1000826
:10A3C8002FAB0008DBA1000807AB0008F3AC0008BE
:10A3D800ADAC0008DBA10008DBA10008DBA1000888
:10A3E800DBA10008DBA10008DBA10008DBA1000855
:10A3F800DBA10008DBA10008DBA10008DBA1000845
:10A40800DBA10008DBA10008DBA10008DBA1000834
:10A41800DBA10008DBA10008DBA10008DBA1000824
:10A42800DBA10008DBA10008DBA10008DBA1000814
:10A43800DBA10008DBA10008DBA10008DBA1000804
:10A44800DBA10008DBA10008DBA10008DBA10008F4
:10A45800DBA10008DBA10008DBA10008DBA10008E4
:10A46800DBA10008DBA10008DBA10008DBA10008D4
:10A47800DBA10008DBA10008DBA10008DBA10008C4
:10A48800DBA10008DBA10008DBA10008DBA10008B4
:10A49800DBA10008DBA10008DBA10008DBA10008A4
:10A4A800DBA10008DBA10008DBA10008DBA1000894
:10A4B800DBA10008DBA10008DBA10008DBA1000884
:10A4C800DBA10008DBA10008DBA10008DBA1000874
:10A4D800DBA10008DBA10008DBA10008DBA1000864
:10A4E800DBA10008DBA10008DBA10008DBA1000854
:10A4F800DBA10008DBA10008DBA10008DBA1000844
:10A50800DBA10008DBA10008DBA10008DBA1000833
:10A51800DBA10008DBA10008DBA10008DBA1000823
:10A52800C9AC0008DBA10008EBAA0008C1AA000812
:10A53800DBA10008DBA10008DBA10008DBA1000803
:10A54800DBA10008DBA10008DBA10008DBA10008F3
:10A55800DBA10008DBA10008DBA10008DBA10008E3
:10A56800DBA1000863AA0008DBA100082BAA0008E9
:10A57800DBA1000889A9000827A900080BA9000881
:10A58800DBA10008F1A80008DBA10008C9A80008A1
:10A59800B7A8000857A80008DBA1000827A80008EA
:10A5A800DBA10008DBA10008FDA70008CFA7000871
:10A5B800BBA7000893A7000873A7000849A70008CD
:10A5C800DBA1000831A70008DBA10008DBA1000817
:10A5D800DBA10008DBA10008DBA10008DBA1000863
:10A5E800DBA10008DBA10008DBA10008DBA1000853
:10A5F800DBA10008DBA10008DBA10008DBA1000843
:10A6080011A70008DBA10008DBA10008B7A6000815
:10A61800DBA10008DBA10008DBA1000853A60008A5
:10A62800DBA10008DBA10008DBA1000839A60008AF
:10A63800C14B1B78DB073FF5CCAD0125F9F7E0FBF3
:10A64800F9F7BAFD2B46FFF75CBA3046F7F7BCF8C6
:10A658003368B8851A46591C316012F8021B3260FB
:10A6680087F82E105A7887F82F20DA1C32609A78EB
:10A6780087F830201A1D3260DA7887F831205A1DA1
:10A6880032601B7987F8323007F12C000023BB8633
:10A69800F6F7F6FFA94AAA4B1268801A4FF001058F
:10A6A80061F10001C3E904012B46FFF72ABA531CE4
:10A6B800336013780F2B3FF68CAD911C3160C3EBE0
:10A6C800C303A0495078C854D01C30600B4491781B
:10A6D8005970111D3160D1789970511D316011790F
:10A6E800D970911D316051791971D11D31609179FD
:10A6F800597102F108013160D2799A71012517F078
:10A7080059FB2B46FFF7FDB93046F7F75DF8DFF840
:10A718004082A8F80E003046F7F756F80125A8F849
:10A728000C002B46FFF7EDB93046F7F74DF8864A8F
:10A7380000EB80004300012513802B46FFF7E1B9A9
:10A748003046F7F741F8DFF82882A8F810003046BD
:10A75800F7F73AF8A8F812003046F7F735F8012568
:10A76800A8F814002B46FFF7CCB91346511C3160EA
:10A7780013F8020B3360D31C51783360927812F0CF
:10A78800BFFA00287FF4D7A923E51346511C31608E
:10A798006E4913F8020B087033606D4953788B705B
:10A7A800D31C3360684B92789A7001252B46FFF7CB
:10A7B800A8B9684B684918684E22012528F0D6FFC9
:10A7C8002B46FFF79EB91146531C3360634B11F8B3
:10A7D800020B1870316051785970D11C3160927831
:10A7E8009A703046F6F7F0FF5D4B0125D8802B466E
:10A7F800FFF787B93046F6F7E7FFDFF86481A8F876
:10A8080000003046F6F7E0FFA8F802003046F6F7F9
:10A81800DBFF0125A8F804002B46FFF772B9DFF823
:10A82800549199F80030002B3FF485A9DFF848814E
:10A8380000253046F6F7C8FF18F010F899F80030F0
:10A84800A8EC010A01359D42F3DBFFF774B90D2925
:10A858007FF4BFAC531C33601578072D3FF6B9ACB5
:10A86800DFF8189130464FF00C08F6F7ADFF08FBFB
:10A8780005F809EB0805A8803046F6F7A5FFE8803B
:10A888003046F6F7A1FF336828811A46591C316013
:10A8980012F8021BA97232605B78EB723046F6F749
:10A8A8007CFF012549F808002B46FFF72AB93046F6
:10A8B800F6F78AFF2B4B012518802B46FFF721B9A5
:10A8C800531C33601078060600F189861A4B1B78F2
:10A8D800DD073FF530A9032828BF00200125F9F737
:10A8E80073FA2B46FFF70DB9134B1B78D8073FF5C2
:10A8F80022A90125F9F726FEF9F75EFC2B46FFF79A
:10A9080000B90D4B1B78DA073FF515A9164A1378DD
:10A91800012543F0040313702B46FFF7F2B8064BEA
:10A928001B78D9073FF507A9104B4FF4C8720125CA
:10A938001A802B46FFF7E5B8E57500201858002067
:10A94800C8240020CC330020A8670020F06C002029
:10A9580098670020B84F00203872030890670020DD
:10A96800D8550020962600201C77002090790020DA
:10A97800B8710020E54B0020403600200C33002041
:10A9880009297FF726ACDFF8B8831346511CD8F89D
:10A998000050316013F8021B297033605378AB7094
:10A9A800D31C33609378642B02F10401A8BF64239D
:10A9B8006B713160D378642B02F10501A8BF642361
:10A9C800AB7131601379EB71931D33605379642B4C
:10A9D80002F10701A8BF64232B7231609379EB70F1
:10A9E80002F108033360D3792B713046F6F7ECFE99
:10A9F800726833686881D11A00290CDD591CD8F8AF
:10AA080000003160521A002A1978417203DD9A1C3D
:10AA180032605B784370012525F006FE2B46FFF770
:10AA280070B8B94B1868D31C014621329D1E356099
:10AA380013F8035C0D705D1E356013F8025C4D70F1
:10AA4800336013F8015C8D7003339A4201F10301FE
:10AA5800ECD117F0D3FDFFF76EB8C1F34705122DFF
:10AA68003FF6B7ABC5B107F1500307F12A0A03EB6C
:10AA78004508D146A8F126083046F6F7A5FE29F87C
:10AA8800020FC145F8D1A14B3AF8022F23F8022F43
:10AA9800D145F9D1112D09D89D4A6B00023B1344C9
:10AAA8000021223223F8021F9A42FBD1994A01233E
:10AAB8001D461370FFF725B8531C9748336001787B
:10AAC8001378002940F0518504220270934A9B00B4
:10AAD8001380FAF741FE924B012598612B46FFF748
:10AAE80010B8DFF8608200233046C8F80030F6F767
:10AAF80054FE0125C8F800002B46FFF702B813469C
:10AB0800511C3160874913F8020BC87033608649BD
:10AB180053784B71D31C3360844B9278DA700125DB
:10AB28002B46FEF7EEBF3046F6F74EFE3046F6F7F8
:10AB38004BFE3046F6F748FE3046F6F750FE3368CF
:10AB4800714D1946581C2A68306011F8020B82F8BA
:10AB58002C003160597882F83610D91C31609B7806
:10AB680082F837303046F6F73AFE3046F6F737FEC9
:10AB78003046F6F734FE3046D5F80080F6F724FE66
:10AB8800A8F83A003046D5F80080F6F71DFE33687D
:10AB98007268A8F83800D11A01290ADD591C2A68F8
:10ABA80031601B7882F82E303046F6F718FE33688D
:10ABB8007268D31A032B00F31D85286849E7531CD4
:10ABC8003360514DDFF88081137888F805303046BE
:10ABD800D5F80090F6F7F8FDA9F820003046D5F82A
:10ABE8000090F6F7F1FD72683368A9F81E00D11AD3
:10ABF800072900F3D884D11A032900F36685D21AED
:10AC0800002A05DD591C2A6831601B7882F8263035
:10AC1800F9F734FA21F0DAFC454B1B68002B00F0F9
:10AC2800F7842868012517F051F92B46FEF769BF0C
:10AC38001346511C3160DFF8108113F8021B88F8A5
:10AC4800021033603B4953780B70D31C33603A4D84
:10AC580093782B71131D3360D378092BA8BF092370
:10AC68003046AB70F6F7B0FD336872682880D11AA9
:10AC7800012905DD3046F6F7A7FD33687268E881DB
:10AC88009A4240F08084F9F7F9F9336872689A4279
:10AC98003EF451AF5A1C32601B78EB7001252B46ED
:10ACA800FEF72FBF531C33601378002B00F062842B
:10ACB8004FF4004001250AF063F92B46FEF721BF47
:10ACC8001346511C316013F8025B3360D31C507873
:10ACD80033609178002D00F06084012D7EF42BAF55
:10ACE80008F0DAF92B46FEF70CBF144B1B7813F06B
:10ACF80001017FF46EAA531C33601078012508F017
:10AD080005F92B46FEF7FDBEB84F0020EE67002080
:10AD1800F0670020146800204E5A00202477002095
:10AD2800C824002098670020F0780020A867002039
:10AD3800284300208C670020B8710020E5750020AA
:10AD4800BC4F0020B8340020F06C0020CF4B1B68AB
:10AD5800002B3EF4F0AE18F055FFFF283EF4EBAEA2
:10AD68003046F6F731FD3F2840F2BD84DFF84883CE
:10AD7800002588F8005033687268A8F80400D21AD1
:10AD8800012A7EF7D8AE1A46591C316012F8021B08
:10AD980088F8021007F15000326000225D7800F850
:10ADA800242D18F001FF97F82C30AB423EF4C3AEC7
:10ADB800284618F01DFFFEF7BEBEB54B1B78012BC9
:10ADC8003EF6B9AE1146531C3360DFF8F08211F835
:10ADD800023B88F802303160D31C92F801E03360FE
:10ADE800C31A012B917840F31E843046F6F7ECFC29
:10ADF8000125A8F800002B46FEF783BEDFF8C082C5
:10AE08000023C8F800303046F6F7C7FCD8F8003001
:10AE180001250343C8F800302B46FEF772BE07230E
:10AE2800B1FBF3F3C3EBC305491B7FF4D2A9DBB233
:10AE380003F1FF395FFA89F9002B3EF47CAEDFF8A5
:10AE480054A209F101090D46531C336092F9002000
:10AE5800904B4FF0000893F90210914203F1080358
:10AE680000F0138308F10108B8F1050FF3D1FFF7DB
:10AE7800B0B9531C336013780E2B3FF6AAA9911C66
:10AE880031605578032D3FF6A4A98348062101FBBC
:10AE980003F1431802F1030E5D71C6F800E09578DE
:10AEA8004554111D3160D1785970511D31601179A7
:10AEB8009970911D31605179D970D11D31609279A5
:10AEC8001A7101252B46FEF71CBE531C3360734BC9
:10AED80012785A7501252B46FEF713BE531C3360B2
:10AEE80015781F2D3FF675A905297FF472A93046FC
:10AEF800F6F753FC6A4B43F8250015F033FFFEF7CD
:10AF08001ABE674D05F140083046F6F75DFC336818
:10AF1800A5F88000591C1A46316012F8021B85F802
:10AF2800821032605B7885F883300435A845EBD110
:10AF3800FEF701BE531C594D336013782B7230460F
:10AF4800F6F742FCA8833046F6F73EFC28833046E5
:10AF5800F6F73AFC32686883531C33601278EA7457
:10AF68007268D31A032B00F391833368D11A052929
:10AF780000F37C83D21A002A7EF7DDAD5A1C3260BA
:10AF88001B7885F8213001252B46FEF7BABD531CE6
:10AF98003360444915780D70C01A00287EF7CBAD90
:10AFA800931C33605378003318BF012301254B707D
:10AFB8002B46FEF7A6BD3046F6F706FCDFF8E8801C
:10AFC800C8F800003046F6F7FFFBC8F80400304622
:10AFD800F6F7FAFB0125C8F808002B46FEF791BDE5
:10AFE8000125F7F77DFA2B46FEF78BBD531C33601E
:10AFF8002C4B1278DFF8C8801A700023C8F800308C
:10B008003046F6F7CAFB3368D8F800202349264DA6
:10B0180010435A1CC8F8000032601B780B72304687
:10B02800F6F7D2FB28603046F6F7CEFB686030466C
:10B03800F6F7CAFBA8603046F6F7C6FB3046F6F7C7
:10B04800C3FBFEF778BD194B02F1080101323260EB
:10B0580012F8010C03F8010F9142F7D1FEF76BBD0E
:10B068001346511C3160124913F8025B8D7033602E
:10B0780055784D7083423EF45EADD31C33600D4B62
:10B0880092781A7201252B46FEF73BBDE875002021
:10B09800CE3D0020D4560020C4340020A8560020FD
:10B0A800844400204443002080320020A75600201A
:10B0B800B8670020C8240020EC7500201E77002007
:10B0C800E03D0020531C336092F80080B8F1110F66
:10B0D8003FF67FA8931C3360C34D537805F81830AA
:10B0E8003046F6F771FB40F6CA039842A8BF1846E7
:10B0F80040F2EE23984205EB4801B8BF18460125F7
:10B10800A0F2EE222B46192092FBF0F24A70FEF7CD
:10B11800F8BC1346511CB54D316013F8021B297158
:10B12800336053786B713046F6F74EFB33682880EE
:10B138005A1C32601B78AB713046F6F745FB336812
:10B1480068805A1C32601B78EB7101252B46FEF78C
:10B15800D8BCA74B10294FF0000228BF10211A6055
:10B168005A609A60DA601A7400293EF4E4AC3268D6
:10B17800013B11440132326012F8010C03F8010F4F
:10B188008A42F7D1FEF7D7BC511C316015783B6273
:10B19800132D3FF61EA8911C316050787A620DF08D
:10B1A800ADFE00283FF415A87A6A9249007801F8A4
:10B1B8002500D01C306001EB850590786870101D63
:10B1C8003060D078A870501D30601279EA703B6A00
:10B1D80001F1500202E004318A4207D008780028C1
:10B1E800F9D18D78C8788542F5D20123824A83F057
:10B1F8000103012513702B46FEF783BC1346511C2F
:10B2080031607E4D13F8021B6970336053782B70E0
:10B21800D31C33609378AB703046F6F7D5FA3368B1
:10B228002881591C1A46316012F8021B6971326074
:10B238005B78AB7101252B46FEF763BC704B3A6A0D
:10B248009B68D4F800905A449A4200F27081F7F74C
:10B25800BBF85A464946386AF6F762FF2368034442
:10B26800236086427EF767AC002100E02368013046
:10B278005A1CB04222601970F8D1FEF75CBC3368E2
:10B2880072689A4240F0CE805E4BFF221A704FF0EF
:10B29800000A5D4D12F0AAFE514620225B4885F84F
:10B2A80000A029F0F6FB87F82CA097F82C30072B84
:10B2B80000F25981DFF86491544E524697F82C30C9
:10B2C80003EB430309EBC3035B7CE3B197F82C3032
:10B2D80003EB430309EBC30320215B699BB197F898
:10B2E8002C3003EB430309EBC303586946F82200EB
:10B2F800FAF722FF2B7856F82300FBF7DFF82A78B5
:10B308000132D2B22A7097F82C300133DBB287F8B9
:10B318002C3097F82C30072BD0D92368591C216082
:10B328001A70B8F1000F3EF406AC394BC8F800307B
:10B3380001252B46FEF7E5BB002D7FF47FAF59466C
:10B348002046F6F77FFA23685A1C22601D702C4BA2
:10B3580026689D683B6A0BEB0302AA4240F26F81A4
:10B368003B6AED1AF7F730F82A463146386AF6F79D
:10B37800D7FE236803442360FEF7DDBB3046F6F7AB
:10B3880023FA326871687B6A9142834673D1064614
:10B398001D46FEF728BE3046F6F716FADFF880801D
:10B3A800FEF787BC931C33601A4B51781970D11C77
:10B3B800316091785970111D3160D2789A70FEF71A
:10B3C800BABB931C33605578022D3EF602AF304667
:10B3D800F6F7FAF9104B03EB45034FF0FF35A3F8E6
:10B3E80056002B46FEF78DBB746A00206C7900204E
:10B3F8008A4900206469002020210020484F00204D
:10B40800FC190020C8240020F9350020EC68002031
:10B418001D5D01089B3C0020B0760020F8700020DC
:10B42800886700205A1C19463260B74811F8022B69
:10B43800027031605B784370042A03D9FF2A7EF4D6
:10B4480024AB24E7B1490978994205D8022A7EF449
:10B458001CABFF2B7EF419AB236801255A19226017
:10B468001D70B8F1000F3EF466ABA94BC8F8003068
:10B478002B46FEF746BB511C316012781D46131C43
:10B48800064618BF0123FEF7AEBD0AEBC80B3046CF
:10B498008BF80220F6F798F933682AF838001A462C
:10B4A800591C316012F8021B8BF8031032605A786D
:10B4B8008BF80420DA1C32609A788BF806201A1D63
:10B4C80032600135DB788BF80530A9457FF4BCACD8
:10B4D800FEF731BB3046F6F782F93368DFF834827D
:10B4E8001A46591C316012F8021B88F85510326050
:10B4F8005B7888F854303046F6F766F9A8F85000BB
:10B508003046F6F761F93046F6F75EF996E80C0032
:10B518009B1A012BA8F852007EF70DAB3046F6F7C0
:10B5280053F90125A8F85A002B46FEF7EABA3A6AF9
:10B53800A3EB0208F6F748FF42464946386AF6F791
:10B54800EFFD236803442360002D3EF4F4AA88E647
:10B55800704B0030984418BF0120012588F85E0020
:10B568002B46FEF7CEBA5246D7E604297EF4E3AA64
:10B57800FFF7ACBA684A1368012523F40043136047
:10B588002B46FEF7BEBA5A1C32601B78003318BF30
:10B59800012388F80730FFF776BB012516F0BAFEBD
:10B5A8002B46FEF7AEBA3046F6F70EF9A8F80A00B1
:10B5B8003046F6F709F9A8F80C003046D5F800909F
:10B5C800F6F702F9A9F822003046D5F80090F6F708
:10B5D800FBF833687268A9F82400FFF70CBB00F089
:10B5E8007F00032828BF0020012507F071FD2B46A6
:10B5F800FEF787BA3046D5F80080F6F7E5F8A8F8E0
:10B60800320030462E68F6F7DFF8B086FFF7D5BA75
:10B6180042484349434A444B036001250B60136089
:10B628002B46FEF76EBA414B1A88012512FB0EF223
:10B638002B4692FBF1F2A8F80020FEF762BAF6F763
:10B64800C3FE5A463146386AF6F76AFD2368012573
:10B65800034423602B46FEF754BA7D62AA46FEF7E0
:10B668005CBDDA46C7F824B0FEF757BD5A1C3260F5
:10B678001B78EB723046F6F790F83368E8605A1C8E
:10B6880032601B782B743368726873E43046F6F7BF
:10B698009BF8A8843046F6F797F833687268E88410
:10B6A800D11A03297FF762AC1A46591C316012F887
:10B6B800021BA97732605B7885F820303046F6F7B0
:10B6C80083F833687268688450E43046F6F77CF88B
:10B6D800A8F80E003046F6F777F833687268A8F8CD
:10B6E8001000FFF78CBAC50800F0070301350133D5
:10B6F800EDB2DFF83C802846194688F8013013F08F
:10B70800CDFFFFF736BB00BFC8240020E54B002063
:10B71800113F0108B0760020B04F002014540020DB
:10B7280068540020D05400205F050008D065002030
:10B73800EC7500202DE9F04F2DED0E8BDFF8F4B0FD
:10B7480097B0DBF80420079058469047002800F08F
:10B758008E82BBF8A87000218BF85110002F6DD194
:10B76800BBF93A00DBF82450DBF82810BBF9386045
:10B77800DBF82040BBF93C20DFF8BCA0401B521A84
:10B78800CBF830009BF85210CBF83420341B0BF167
:10B798002C00CBF82C4010F0FDF8DAF800209100CE
:10B7A80041F1F587DBED0C5A1F4CDBED0B7A1F4995
:10B7B80094ED406AD4ED416A94ED427AD4F80C21B4
:10B7C80009681B4B0593B8EEE58ADBED0D5AF8EED8
:10B7D800E77AF8EEE58A013277EE867A38EE268A3D
:10B7E80078EE878A8A42C4ED407A84ED418AC4EDB6
:10B7F800428AC4F80C2101F0508393F800E0BEF1AE
:10B80800140F03F005800023D4F814510693062D75
:10B8180001F29D84DFE815F0801656168D15421743
:10B82800080CAB17EF1500BFF02400208C3F002058
:10B83800044C0020046D00208C6F0020DE4BDF4894
:10B848001A6808934FF47A76B6FBF2F2C2EB421606
:10B8580002EB8602D600DA4BDFF8C88344780593FA
:10B86800B6B2B7421D78B8F9060003F0F380DBF8EA
:10B878007C30BBF93810DBF8602003F1010E07EECD
:10B88800901A0A44BEF1010FCBF87CE0CBF8602097
:10B89800F8EEE77A03F0EB80DBED1B5ADBED1D6A6F
:10B8A80007EE10EA37EEE56AB8EEC75A012F86EEC2
:10B8B800057A37EE257A77EEC77A8BED1C7AE7EEB4
:10B8C800866A8BED1B7AF0EE667ACBED1E6ACBEDBD
:10B8D8001D6A03F06E84DBF89030BBF93A10DBF890
:10B8E800642003F1010E07EE901A0A44BEF1010F1D
:10B8F800CBF890E0CBF86420F8EEE77A03F0D2803A
:10B90800DBED205ADBED226A07EE10EA37EEE56A36
:10B91800B8EEC75A012F86EE057A37EE257A77EE0C
:10B92800C77A8BED217AE7EE866A8BED207AF0EE06
:10B93800667ACBED236ACBED226A03F06F84DBF8DD
:10B94800A430BBF93C10DBF8682003F1010E07EEC8
:10B95800901A0A44BEF1010FCBF8A4E0CBF8682096
:10B96800F8EEE77A03F0B980DBED255ADBED276ABC
:10B9780007EE10EA37EEE56AB8EEC75A012F86EEF1
:10B98800057A37EE257A77EEC77A8BED267AE6EEDA
:10B99800276A8BED257AF0EE667ACBED286ACBED37
:10B9A800276A03F02E84874CA8F80600BBF8A82065
:10B9B800059B013A1D78ABF8A82008990022072DAD
:10B9C8004A608A60CA6040F05981F9F7C5FE059B54
:10B9D800DFF850821D78079BC01A94F82831A8F820
:10B9E80000000993002B40F04F81744A5279002AD5
:10B9F80001F08081744A1278013AD2B2072D84F896
:10BA0800282102F0688200230A93704BD4F834216D
:10BA1800D3F800A0684B0893079B9FED6D6AD4ED9F
:10BA28004C9A6C49C4F834319A1A07EE902AF8EE09
:10BA3800677AB7EE007AC6EE278A0025664BDFF8EC
:10BA4800E891DFF8E881654F06932E46D1ED006A4C
:10BA580094ED4BDA9FED629ADFED62AA9FED62CA20
:10BA68009FED62AADFED62BA9FED62BA77EE69CA0E
:10BA78006CEEA6CAF4EEC7CAF1EE10FA88BFF0EE73
:10BA880047CA5D4B99ED008A2B44D3ED007AF5EE59
:10BA9800407AF1EE10FA17D0584B2B4493ED007A08
:10BAA80078EE476AB0EEE66AF4EEC67AF1EE10FA7E
:10BAB80008D5F5EEC06AF1EE10FACCBF37EE878AEA
:10BAC80037EE678A83ED008A4D4B1A88930739D081
:10BAD800022E37D09AF82E104A4B07EE901A2B44B4
:10BAE80093ED007A4B42F8EEE76A07EE903A26EEBD
:10BAF800877AF8EEE77AB4EEE77AF1EE10FA0AD42C
:10BB080007EE901AF8EE677AF4EEC77AF1EE10FABB
:10BB180088BFF0EE477A3C4B3C4903EB460331F9CA
:10BB28001600B3F90C30C31A07EE103AB8EEC77A0C
:10BB3800D007E7EE497A41F17980354B93ED008AD9
:10BB480027EE888A089B94F868212B4493ED01EA34
:10BB580078EE4EDA002A00F0F7802E4BD4F86C21EC
:10BB680007991B688A1A9A4240F3EE809AF848307F
:10BB7800022B02F0EF81022E04F0C684264B1B68CC
:10BB8800990700F19780254B87ED00CA1B689342FF
:10BB9800C0F2CA80F7EE007AF4EEE79AF1EE10FAF6
:10BBA80040F1D28008991E4BD1ED017A93ED007ACD
:10BBB800F0EEE77A3CE000BF7C6F0020F06C0020DC
:10BBC800044C0020F02400208C670020B84F00208F
:10BBD8000024744924550020A4420020B0420020CB
:10BBE800CDCCCC3DAE47813F000000000000C842EC
:10BBF80000003443610BB63B185500203426002062
:10BC0800B44F00204026002098670020644F002091
:10BC1800005500202C550020584F002028550020A2
:10BC280034550020084C002028260020BC42002063
:10BC3800F4EEC77AF1EE10FA40F18680D1ED027A7F
:10BC4800F0EEE77AB4EEE77AF1EE10FA7CDDD1EDAA
:10BC5800037AF0EEE77AB4EEE77AF1EE10FA73DDE4
:10BC68000F4B1B689B075FD50E490F4B43E00F4BEB
:10BC78000F4C1D780593072D3FF4A7AE94F8283193
:10BC88000993002B3FF4B1AE013B84F82831012D14
:10BC980001F0AF8217B0BDEC0E8BBDE8F08F00BF8E
:10BCA800584F0020644F002098670020044C002063
:10BCB800F0240020D34BD449DFF8C8E331F916C08B
:10BCC8009EED008ADFF8C0E387ED00CA03EB46006B
:10BCD80028EE098AB0F90C00A0EB0C0007EE900AD8
:10BCE800F8EEE77ADEF8000027EE888A904278EED0
:10BCF8004EDABFF64FAFB3F90C20B1F900E0C348F4
:10BD0800AEEB020E00688EEAEE72A2EBEE72824291
:10BD18001ADAB3F90E30B1F90220D21A82EAE273C4
:10BD2800A3EBE27398420FDDB94B1A88002384F81D
:10BD38006831002A43F00886B64AB74B117818686C
:10BD480081F00101FAF7C0FBB44B2B4493ED000AD4
:10BD5800069B2DEE000A022E20EE2D0AA3EC010A06
:10BD6800069304F0F983AE4BD7ED006A93ED007AA1
:10BD7800AC4BD3ED007AAC4B93ED006AAB4B67EE5E
:10BD8800277A2B4427EEAC7AD3ED007A67EE277A30
:10BD9800F0EE665AEDEEA75AB1EE467AB4EEE57AC1
:10BDA800F1EE10FA08DCB4EEE56AF1EE10FA8CBF99
:10BDB800B0EE657AB0EE467A94ED4C6AF7EE007A0A
:10BDC800B4EEE76AF1EE10FAACBF0123002343B1E9
:10BDD800F0EEE66AF0EEC77AF4EEE67AF1EE10FAE3
:10BDE80001D587ED007A022E04F01683904A914B14
:10BDF80052F826001B68B0EE4E0A98478E4A8F4BC1
:10BE080052F826001B6898479AF8373023B18C4BB4
:10BE18001B88002B00F07187B0EE4C8A894B38EEF6
:10BE2800400A2B4493ED008A83ED000A9AF84830C3
:10BE380030EE480A20EE288A002B33D0824B1B783C
:10BE480013F0010300F0BE86F7EE007AF4EEE79AED
:10BE5800F1EE10FA94F86831C1F23D85002B00F03C
:10BE6800F187D4F86C31079AD31A784A12689A4243
:10BE780018DD774BD3ED007AF0EEEDDAF4EEE7DA81
:10BE8800F1EE10FA42F17780614B1A88002384F8AA
:10BE98006831002A00F0A2866E494A6912B10A6820
:10BEA80013604B746C4B94F878212B4493ED000A83
:10BEB8002DEE000A20EE088A88ED008A32B9069B2A
:10BEC80087ED00CA03ED01CA88ED00CA0136032ECA
:10BED80009F1040908F1040807F1040705F104054C
:10BEE8007FF4CFAD059B1A78072A01F00A85012A4D
:10BEF80001F0DE870023069394F88021002A41F0A0
:10BF08008581DFF888A1554BDAF800201968D50437
:10BF180091F82C0000F10C87DFF87491504AB9F8B9
:10BF28001A3092ED006A4F4A4F4DD2ED005AD5EDC6
:10BF3800036A4E4A84ED646A07EE103A4C4B92ED60
:10BF4800005AD3ED007AD3ED013AD3ED024A84EDDD
:10BF5800626AB8EEC77A35EEC64A012236EEC77A6B
:10BF680084ED614AC4ED655A84F89821C7EE055AF4
:10BF78000A8D534206EE103A3E4BDFED3F6A93EDD1
:10BF8800005A3E4B93ED004AB7EE007AF4EEC75ADA
:10BF980035EE045AF1EE10FA88BFF0EE475A35EE46
:10BFA800275AB8EEC66AF4EEE65AF1EE10FA07EE32
:10BFB800902AB4EEC65AB8BFF0EE665AF1EE10FAFF
:10BFC800C4ED685AB8EE677A01F10983B4EEC75A2E
:10BFD800F1EE10FA88BFB0EE475A264BDFED286A1B
:10BFE800D3ED017A254B93ED014A77EE847A25EE5D
:10BFF800265A77EEA37AB4EEE76AF1EE10FA52DC2D
:10C0080048E000BF98670020644F002030550020AA
:10C01800F0570020F2570020F4570020D454002095
:10C02800105400200400002048550020E05400204F
:10C0380018540020145400206C5400206854002028
:10C04800B44F002060260020E57500202C55002004
:10C0580038550020F8570020EC540020B84F002035
:10C06800EC6500207C6700208C4D0020E055002006
:10C07800B0420020A442002000000000BC42002082
:10C088006F12833A00550020285500208C6F00203D
:10C09800A8560020B4EEE77AF1EE10FA8CBFB0EEA5
:10C0A800676AB0EE476AEC4B4A8DD3ED027A9FED92
:10C0B800EB7A534204EE103A74EEA77AB8EEC44A0B
:10C0C80026EE076AF4EEC47AF1EE10FA0AD407EE07
:10C0D800102AB8EE474AB4EEE74AF1EE10FA88BFE4
:10C0E800B0EE674ADE4ADFEDDD7A527824EE274A61
:10C0F8000AB9B1EE444A002841F04286B7EE003A48
:10C10800D84E3278002A02F0BF86D749DFEDD77AB9
:10C11800D1ED024AD1ED016A91ED037A66EE244A27
:10C12800E5EE264AE4EE074A63EE244AF4EEE74ACF
:10C13800F1EE10FAB4BFF0EE673AF0EE643A98BF49
:10C14800F0EE647A012ACDED0E4A02F0F28691ED06
:10C15800067AD1ED052AD1ED076A26EE077AA5EE13
:10C16800227AA4EE267A23EE077AB4EEE77AF1EE85
:10C1780010FAB4EEE37A8CBFF0EE676AF0EE476A25
:10C18800F1EE10FA88BFF0EE676AB4BFF0EE637A9A
:10C19800F0EE477A022A8DED0F7A00F0DE8091EDFD
:10C1A8000A7AD1ED092AD1ED0B3A26EE077AA5EEE7
:10C1B800227AA4EE237A23EE077AB4EEE67AF1EE39
:10C1C80010FAB4EEE77A8CBFF0EE663AF0EE473A32
:10C1D800F1EE10FA98BFF0EE636AA8BFF0EE477A66
:10C1E800032A8DED107A00F0B88091ED0E7AD1ED2A
:10C1F8000D2AD1ED0F3A26EE077AA5EE227AA4EEA3
:10C20800237A23EE077AB4EEE67AF1EE10FAB4EE6A
:10C21800E77A8CBFF0EE663AF0EE473AF1EE10FAA4
:10C2280098BFF0EE636AA8BFF0EE477A042A8DED56
:10C23800117A00F09280D1ED123AD1ED112A91EDE8
:10C24800137A66EE233AE5EE223AE4EE073A63EE15
:10C25800233AF4EEE63AF1EE10FAF4EEE73A8CBF40
:10C26800B0EE667AB0EE637AF1EE10FA98BFF0EEAF
:10C27800476AA8BFF0EE637A052ACDED123A6CD072
:10C28800D1ED163AD1ED152A91ED177A66EE233ADB
:10C29800E5EE223AE4EE073A63EE233AF4EEE63AA4
:10C2A800F1EE10FAF4EEE73A8CBFB0EE667AB0EE33
:10C2B800637AF1EE10FA98BFF0EE476AA8BFF0EE85
:10C2C800637A062ACDED133A47D0D1ED1A3AD1ED6B
:10C2D800192A91ED1B7A66EE233AE5EE223AE4EE4E
:10C2E800073A63EE233AF4EEE63AF1EE10FAF4EE8A
:10C2F800E73A8CBFB0EE667AB0EE637AF1EE10FAE8
:10C3080098BFF0EE476AA8BFF0EE637A072ACDED32
:10C31800143A22D091ED1E7AD1ED1D2AD1ED1F3AA3
:10C3280026EE077AA5EE227AA3EE847A27EE037A20
:10C33800B4EEE67AF1EE10FAB4EEE77A8CBFB0EE1E
:10C34800666AB0EE476AF1EE10FA8DED157A98BF7D
:10C35800F0EE466AA8BFF0EE477A77EEE67AF7EE97
:10C36800006AF4EEE67AF1EE10FAC4ED4C7A43F383
:10C37800668686EEA77A022ADDED0F7A67EE244AF2
:10C3880067EE877ACDED0E4ACDED0F7A2DD0DDED33
:10C39800107A67EE877A032ACDED107A25D0DDED85
:10C3A800117A67EE877A042ACDED117A1DD0DDED7A
:10C3B800127A67EE877A052ACDED127A15D0DDED6F
:10C3C800137A67EE877A062ACDED137A0DD0DDED64
:10C3D800147A67EE877A072ACDED147A05D0DDED59
:10C3E800157A27EE877A8DED157A2149096811F0BB
:10C3F80080530A9301F02282F6EE005AC4ED685A7F
:10C40800002A02F0908594F998311A4994ED656AEA
:10C41800C87894ED645ADAF80010DFF868E0164F2F
:10C42800DEED004AB7F906E0B9F81A700B9707EE87
:10C43800103A124BD4ED616A1D78114BD4ED627A33
:10C448001B780893BDEEC66A01F4805316EE10CA35
:10C45800BDEEC56A0D9317E0A44200206F12833A1F
:10C4680044430020E54B0020505500200000000008
:10C478007467002030460020EE5B0020E575002040
:10C48800DC7100204C55002001F4800301F01007F6
:10C49800B8EEC77A0C9305F0010816EE101A0028BA
:10C4A80040F00487002F41F03A83D54D9DED0E5A98
:10C4B80095ED006AD34825EE866AA5EE076AB0EEC8
:10C4C800675AA6EE265ABDEEC56A16EE10EA16EEB3
:10C4D800107AE645A8BF67467145C8BF0F4606EE05
:10C4E800107AB8EEC66A012A80ED006A00F0DC8096
:10C4F80095ED046A9DED0F5A25EE866AA5EE076A4A
:10C50800B0EE675AA6EE265ABDEEC56A16EE10EAD8
:10C5180016EE107AE645A8BF67467145C8BF0F46B4
:10C5280006EE107AB8EEC66A022A80ED016A00F0BB
:10C53800BB8095ED086A9DED105A25EE866AA5EE3A
:10C54800076AB0EE675AA6EE265ABDEEC56A16EE21
:10C5580010EA16EE107AE645A8BF67467145C8BFCF
:10C568000F4606EE107AB8EEC66A032A80ED026A14
:10C5780000F09A8095ED0C6A9DED115A25EE866AB9
:10C58800A5EE076AB0EE675AA6EE265ABDEEC56A52
:10C5980016EE10EA16EE107AE645A8BF6746714512
:10C5A800C8BF0F4606EE107AB8EEC66A042A80EDB8
:10C5B800036A79D095ED106A9DED125A25EE866AC8
:10C5C800A5EE076AB0EE675AA6EE265ABDEEC56A12
:10C5D80016EE10EA16EE107AE645A8BF67467145D2
:10C5E800C8BF0F4606EE107AB8EEC66A052A80ED77
:10C5F800046A59D095ED146A9DED135A25EE866AA2
:10C60800A5EE076AB0EE675AA6EE265ABDEEC56AD1
:10C6180016EE10EA16EE107AE645A8BF6746714591
:10C62800C8BF0F4606EE107AB8EEC66A062A80ED35
:10C63800056A39D095ED186A9DED145A25EE866A7B
:10C64800A5EE076AB0EE675AA6EE265ABDEEC56A91
:10C6580016EE10EA16EE107AE645A8BF6746714551
:10C66800C8BF0F4606EE107AB8EEC66A072A80EDF4
:10C67800066A19D095ED1C6A9DED155A65EE865A25
:10C68800E7EE055AE6EEA57AFDEEE77A17EE905A40
:10C69800AC45A8BFAC46A942D8BF614607EE901A80
:10C6A800F8EEE77AC0ED077AB8F1000F00F00C87D2
:10C6B800554A1268002A40F01487544A127892B1F9
:10C6C800307868B14F4FDFF868810025E8B2D8F8B4
:10C6D8000030B7EC010A9847307801358542F5DB20
:10C6E8004B4A12689047059B1A78072A01F0F88090
:10C6F8000026DAF80020570500F1E187454B1B6852
:10C708001D0700F18187444B1B78BBB1434AB9F838
:10C718001A30B2F906209A4210DC414B1B78012BE3
:10C7280001F0DE83192B01F0DB830E2B06D0082BDA
:10C7380004D03C4D0023AB60C4F8403194F8AA51B2
:10C7480025B1394B1B889F0741F09C8394F8B02191
:10C75800002A40F0BF8799F81E70002F00F02A8445
:10C76800022F01F04283032F41F03B8399F82030D8
:10C77800C3EB431103EB8101C90089B299F81F305B
:10C788000233DBB2002A00F05785002900F05485F7
:10C7980026480768B1FBF7F10FB2A4F8E071002B47
:10C7A80003F0E28007EE907AF8EEE77AF7EE006A97
:10C7B80086EEA77A1B4D012BD4ED7D6AD5ED007A64
:10C7C80077EEE67A67EE877AC4ED797A3CD0D5EDD4
:10C7D800017AD4ED7E6A77EEE67A022B67EE877AE5
:10C7E800C4ED7A7A30D0D5ED027AD4ED7F6A77EE4F
:10C7F800E67A032B67EE877AC4ED7B7A24D019E0BA
:10C8080050550020044300200C54002004750020DB
:10C81800D8710020584F002020210020EE5B002016
:10C82800444300208C4D0020B44F002028430020B2
:10C83800D0710020D5ED037AD4ED806A77EEE67AE0
:10C8480067EE877AC4ED7C7A05990978092903F09F
:10C858001682002F40F3B4839BB394ED7D7AD4ED18
:10C86800797A77EE877A012BC4ED7D7AC5ED007A67
:10C8780021D094ED7E7AD4ED7A7A77EE877A022BFE
:10C88800C4ED7E7AC5ED017A15D094ED7F7AD4EDAA
:10C898007B7A77EE877A032BC4ED7F7AC5ED027A2F
:10C8A80009D0D4ED807A94ED7C7A77EE877AC4ED5E
:10C8B800807AC5ED037A013B022BB8BF0223DBB2B5
:10C8C8000993099B002A18BF02239E46C84BDFED37
:10C8D800C96A1A68059B91781878137807EE903A18
:10C8E800F8EEE77AB0EE007A67EEA67AF4EEC77A49
:10C8F800F1EE10FA40F35E86DFEDBF6A37EEC77AD5
:10C90800B0EE676AA7EE266AF0EE466A95ED007A01
:10C918009FEDBA6A27EE066AF0EEC65A84ED546AAD
:10C92800C4ED575A99B107EE101AB8EEC75A9FEDE1
:10C93800B17A66EE064A25EE075AB7EE007A37EE68
:10C94800457A64EEA54AA4EE857A26EE076A9FED3D
:10C95800AC7A537926EE877A27EE067ACBB1DFEDEB
:10C96800A56A9FEDA86A65EEA65A06EE903AF8EE1B
:10C97800E66A65EEA65AF4EEC65AF1EE10FA01F32D
:10C98800D781B7EE006A76EE655AC6EE256A27EEBD
:10C99800267A0C289FED9C8ADFED9C6A00F055876B
:10C9A800B4EEC87AF1EE10FA98BFB0EE478AB4EE4A
:10C9B800E68AF1EE10FAB8BFB0EE668A84ED4E8AC8
:10C9C800BEF1000F00F0DD80B0EE007AF4EEC77A19
:10C9D800F1EE10FA05DD37EEC77ADFED876AE7EE8C
:10C9E800267A95ED017ADFED856A27EE267AF0EE54
:10C9F800C75A84ED557AC4ED585A99B106EE901A83
:10CA08009FED7C6AF8EEE66A27EE075A66EE866ABC
:10CA1800B7EE006A36EE666A25EE255AA5EE266A56
:10CA280027EE067ADFED766A937967EEA67A67EEE7
:10CA3800877AABB107EE103AB8EEC77A9FED6D6A08
:10CA4800DFED706A27EE257A27EE067AB4EEE67AED
:10CA5800F1EE10FA41F37481DFED6D6A67EEA67AA4
:10CA68000C2800F01087DFED686A9FED687AF4EE15
:10CA7800E67AF1EE10FA88BFF0EE667AF4EEC77A3D
:10CA8800F1EE10FAB8BFF0EE477ABEF1010FC4ED2F
:10CA98004F7A76DD5378DFED576A07EE903AF8EE75
:10CAA800E77AB0EE007A67EEA67A537AF4EEC77AA0
:10CAB800F1EE10FA05DD37EEC77ADFED4F6AE7EEE3
:10CAC800267A95ED027ADFED4D6A27EE267AF0EEAA
:10CAD800C75A84ED567AC4ED595A9BB106EE903A7E
:10CAE8009FED446AF8EEE66A27EE075A66EE866A14
:10CAF800B7EE006A36EE666A25EE255AA5EE266A76
:10CB080027EE067ADFED3E6AD37967EEA67A67EEFE
:10CB1800877AFBB107EE103AB8EEC77A9FED356A0F
:10CB2800DFED386A27EE257A27EE067AB4EEE67A44
:10CB3800F1EE10FA01F30081B5EEC07AF1EE10FAC9
:10CB480002F19483B7EE006A36EE477AC6EE076ABA
:10CB580067EEA67A0C2800F0B686DFED2B6A9FED0B
:10CB68002B7AF4EEE67AF1EE10FA88BFF0EE667AE8
:10CB7800F4EEC77AF1EE10FAB8BFF0EE477AC4EDDA
:10CB8800507A092800F04D8699F82150002D40F080
:10CB98000286002384F8B0311E4B1B7823B91E4D42
:10CBA800AA78002A41F02D81059B1D78072D7FF476
:10CBB8006EA8F8F7D1FD194B059A801B1578D88017
:10CBC800FFF765B894F86821002A3FF46BA9144A66
:10CBD80084F868311288002A7FF45EA9114A124B42
:10CBE8001178186881F00101F9F76EFCFFF75AB95E
:10CBF800BC4F00200AD7233CD7A368416F12033BE0
:10CC080000004843A4707D3F00C0F94400C0F9C447
:10CC18000000C842685200201E770020084C0020FF
:10CC2800F0570020F2570020F457002094ED577A6F
:10CC3800B1F90000D4ED586AB1F902E0E24AF4EE25
:10CC4800C76A80EAE0738EEAEE71A3EBE073F1EE57
:10CC580010FAA1EBEE71B8BFF0EE476A8B42B8BF8D
:10CC68000B4607EE103A1378B8EEC77A27EE097A22
:10CC7800002B40F0B880D54B93ED006AB4EEEA6A19
:10CC8800F1EE10FA41F1B880F7EE005A75EEC65A87
:10CC98003BEEC77A65EE8B5ACD4BA7EE256A93ED2E
:10CCA800007A26EE076AB5EEC06AF1EE10FA40F295
:10CCB800C185CAEE065AB7EE007AB0EE476AA6EE0C
:10CCC800E56AF0EE466AF4EEC76AF1EE10FA88BF3C
:10CCD800F0EE476AF5EEC06AF1EE10FAB8BFF0EE72
:10CCE8004C6ABC4B93ED007A67EE877AA7EEA68A6A
:10CCF800FEF728BF0122FEF781BEB74BB74A2B4487
:10CD080093ED007AD2ED007AB54B67EE277AF7EE0D
:10CD1800006AF4EEE67AF1EE10FA93ED007A88BF35
:10CD2800F0EE667A67EE877A27EE888AFFF776B89C
:10CD3800AC4BDFF8EC921A78AB4DD2075CBFB9F870
:10CD48001820A4F88C21A94AD5ED037A128807EE99
:10CD5800102AB8EEC77AF4EEC77AF1EE10FA42F26A
:10CD68006380A34D2B8807EE103AB8EEC77AF4EE2D
:10CD7800C77AF1EE10FAC1F2BF809E4A9E4D92ED3D
:10CD8800006AD5ED006A94F99821C4ED646A76EEDC
:10CD9800665A012AC4ED626AC4ED615A84ED656A77
:10CDA80001F05286079BC4F89C31002537EEC77AFC
:10CDB800FCEEE77A914E84ED687A17EE902AA4F893
:10CDC8008C21012296ED005A84F898218C4A9542CC
:10CDD80042F217808B4BD3ED007AD3ED013AD3EDB5
:10CDE800024AFFF7C3B87A4B93ED005AB5EEC05A22
:10CDF800F1EE10FA40F31E85834BD3ED004AF5EEB1
:10CE0800C04AF1EE10FA40F3158534EEC77A66EEA3
:10CE1800CA5A87EE246AC5EE856AB7EE007AB4EE80
:10CE2800C76AF1EE10FA88BFB0EE476AB5EEC06A7D
:10CE3800F1EE10FA76EE876AB8BFB0EE4C6A66EE8D
:10CE4800266A40E7714AD2ED007AB0EEC87AB4EEAD
:10CE5800E77AF1EE10FA7FF725A86D4AD2ED007A4D
:10CE6800B0EEED7AB4EEE77AF1EE10FA7FF71AA891
:10CE7800684AD9ED007A92ED007AF0EEE77AF4EE9E
:10CE8800C77AF1EE10FA7FF50DA801220799C4F8C8
:10CE98006C1184F86821FEF7E8BF07EE102A1978AC
:10CEA800DFF88081C4F80C71B8EEC77AF7EE006A33
:10CEB800132986EE879AB8F90400B4F810619BED3F
:10CEC800070A01F04D85544A544992ED001AD2EDF3
:10CED800053A92ED122A92ED173AD2ED091AD2EDDF
:10CEE8000E4A92ED016A92ED064A92ED0A7AD2ED67
:10CEF8000F5AD2ED132AD2ED186A92ED045AD2EDE8
:10CF0800030A67EE897A69EE288A29EE088AE1EE33
:10CF1800273A01EB86070025A2EE283AC4F800510B
:10CF2800C4F80451E1EE884AA6EE274AE7EE085A0B
:10CF380092ED167A92ED0D6A92ED021AD2ED0C1A64
:10CF4800C7ED003AE2EEA86A25EE635A27EE437A67
:10CF580092ED0B2AD2ED152AC7ED204AA0EEE34A3E
:10CF680026EE646AD2ED143A82ED054AA1EE275AFC
:10CF7800F0EE477AE1EEE45AA2EE086AE2EEC36AFE
:10CF8800E3EEA87A82ED065AC2ED0E5A82ED0F6AD8
:10CF980087ED403AC2ED176AC2ED187AC4F8085115
:10CFA800721C02F01F02A4F81021A8F80400059BC7
:10CFB800FEF723BCA4F8E071002A3FF4EDAD0A4D5A
:10CFC8004FF0020E82E400BF0C55002014550020DB
:10CFD80008550020045500204C260020FC54002051
:10CFE800F8540020E57500208C4D0020E455002001
:10CFF800E65500207C670020D0550020EC55002025
:10D008008FD00300B0420020105500203C5500206E
:10D0180038550020405500201C420020B03F002019
:10D02800A8560020084C0020894A1178D4F81871B5
:10D03800884B9FED897AFE009A1982ED007A0029C3
:10D0480079D08648B0EE476AF0EE476A0022F0ECE5
:10D05800017A013267EEA77A05EE902AB4EEE77AF4
:10D06800F1EE10FAF8EEE55AB8BFB0EE677A8A42E8
:10D0780076EEA76AA7EEA56AE9D1F5EEC06A9A1915
:10D08800F1EE10FA82ED007A55DDC6EE265A744AA2
:10D0980074490988F7EE007A75EEE75AD2ED007AFE
:10D0A80065EEA77AFDEEE77A17EE902A812A42F319
:10D0B800ED808A42A8BF0A4607EE902AF8EEE77A82
:10D0C800694AF01902EB800292ED057AD2ED003A36
:10D0D80092ED066A92ED014AD2ED046AD2ED034A56
:10D0E80092ED025AA3EEA77AA4EE276A66EEC76A03
:10D0F800A7EE646ABDEEC77AE5EE276A17EE100A56
:10D10800812882ED056AC2ED066A42F3BC8081423D
:10D11800A8BF014607EE901AF8EEE77AFCEEE77A28
:10D12800CDED087ABDF8202099198A801FB9BEF183
:10D13800130F02F08D87BEF1150F41F04C811E448C
:10D14800DFF84481B28828F81720D4F81451474AE8
:10D15800013582FB05325119EA17C2EBA102C2EB75
:10D16800C202AD1AC4F814514148D4F81C11079BE7
:10D17800404D02682D78C4F81C31591A0A440260DF
:10D18800002D40F0B28107EE901A3B4EDFF8109167
:10D198003A4FB8EEE78A06F5F07506F51378F6EC1F
:10D1A800017A9BED070ADBF80832F8EEE77A2846A1
:10D1B80027EE800A9847A5F1E000DBF82831984768
:10D1C800A5F17000DBF898319847D6F8EC00DBF849
:10D1D800AC309847D7ED007AA9EC010AE0EE087A5E
:10D1E8002435A845E7EC017AD9D1059B1D78FEF7CF
:10D1F80042BD234B234A19681288234BC9691980F9
:10D208005A8017B0BDEC0E8BBDE8F08F1F4B204E37
:10D218001A7812F0010F327840F0B083002A00F03B
:10D22800A98592001B491C48DFF878A0DFF87890A0
:10D2380026F09CFAFFF73CBAB4F8E071013F3FB220
:10D24800002FA4F8E0717FF7B7AE144DFFF704BBC9
:10D25800923F00208842002000000000F0240020B7
:10D26800943F0020903F0020B04100209324499231
:10D278002C790020883F0020306D00203079002074
:10D2880000790020F0350020084C0020E5750020CA
:10D29800E54B002040360020044300208C4D002040
:10D2A800806F00208C6F0020A8560020002F00F00F
:10D2B8005687B8F1000F42F0A783089BCA4D002B90
:10D2C80042F0F48195ED006A9DED0E5AC74825EEAF
:10D2D800866AFDEEE44AA5EE076AB0EE675AA6EE46
:10D2E800265A14EE901ABDEEC56A16EE10EA16EE2E
:10D2F800107AE645A8BF67467145C8BF0F4606EED7
:10D30800107AB8EEC66A012A80ED006A00F0DF8064
:10D3180095ED046A9DED0F5A25EE866AA5EE076A1B
:10D32800B0EE675AA6EE265ABDEEC56A16EE10EAAA
:10D3380016EE107AE645A8BF67468E45B8BF0F4679
:10D3480006EE107AB8EEC66A022A80ED016A00F08D
:10D35800BE8095ED086A9DED105A25EE866AA5EE09
:10D36800076AB0EE675AA6EE265ABDEEC56A16EEF3
:10D3780010EA16EE107AE645A8BF67468E45B8BF94
:10D388000F4606EE107AB8EEC66A032A80ED026AE6
:10D3980000F09D8095ED0C6A9DED115A25EE866A88
:10D3A800A5EE076AB0EE675AA6EE265ABDEEC56A24
:10D3B80016EE10EA16EE107AE645A8BF67468E45C7
:10D3C800B8BF0F4606EE107AB8EEC66A042A80ED9A
:10D3D800036A7CD095ED106A9DED125A25EE866A97
:10D3E800A5EE076AB0EE675AA6EE265ABDEEC56AE4
:10D3F80016EE10EA16EE107AE645A8BF67468E4587
:10D40800B8BF0F4606EE107AB8EEC66A052A80ED58
:10D41800046A5CD095ED146A9DED135A25EE866A70
:10D42800A5EE076AB0EE675AA6EE265ABDEEC56AA3
:10D4380016EE10EA16EE107AE645A8BF67468E4546
:10D44800B8BF0F4606EE107AB8EEC66A062A80ED17
:10D45800056A3CD095ED186A9DED145A25EE866A4A
:10D46800A5EE076AB0EE675AA6EE265ABDEEC56A63
:10D4780016EE10EA16EE107AE645A8BF67468E4506
:10D48800B8BF0F4606EE107AB8EEC66A072A80EDD6
:10D49800066A1CD095ED1C6A9DED155A65EE865AF4
:10D4A800E7EE055AE6EEA57AFDEEE77A17EE905A12
:10D4B800AC45A8BFAC46A942D8BF614607EE901A52
:10D4C800F8EEE77AC0ED077A002A3FF4F1A8920057
:10D4D8004749464826F04AF9464A1268002A3FF466
:10D4E800ECA814F09BF8FFF7E8B807EE901A424D45
:10D4F800424BDFF80C81DFF80C910694F8EEE78ACE
:10D5080005F5B8760027CDF824801C46059BDBED91
:10D51800077A1B78172B51D095ED007AB8EEC78A99
:10D52800082B28EE278A07D1B0EE480A089326F080
:10D53800F3FA089BA8F80000DAF8002092000BD54F
:10D54800002F02F0C687B0EE480ADBF8083206F171
:10D5580070009847B0EE408AB0EE480ADBF82831F0
:10D56800A6F170009847DBF8983130469847059B3C
:10D578001B78032BB0EE408A2CD0D5F8F000DBF8EE
:10D58800AC30B0EE480A9847D9ED007AA4EC010A0D
:10D59800E0EE287A0137032F06F1240608F1020885
:10D5A80005F10405E9EC017AB0D1059B069C1D78CC
:10D5B800FEF761BBF0EE676AFFF7A8B995ED007A50
:10D5C8000BEB4702B8EEC78A128FA8F8002028EEA6
:10D5D800278AB1E726F0A0FAA8F80000CDE7B0EE58
:10D5E800465AFEF7FABC00BF5055002004430020FD
:10D5F800403600200C540020306D0020806F002041
:10D60800084C002030790020C94DD5ED027AB2EEE1
:10D618000E7AF0EEE76AF4EEC76AF1EE10FA41D539
:10D62800C44B1B8858073DD5C34BC44AB3F90430D3
:10D63800B4F8A61182FB0302DB17C3EBA2035B1A43
:10D648009BB21AB212F1B30FBCBF03F5B4731AB28E
:10D65800B32AC4BFA2F5B4731AB2B94BB9491B793E
:10D668000978002B4FF6FF7318BF012309077FF5D0
:10D678004AA8B549096812FB03F30A7EB3499BB26D
:10D6880012FB03F381FB03121A44DB17C3EB2213CB
:10D6980007EE103AB8EEC77A77EEC77AC5ED027A88
:10D6A800FFF731B8A44BA54AB3F9043082FB031243
:10D6B800DB17C3EBA203A4F8A631FFF724B8DBF805
:10D6C8000830002B3FF41AA8A149A1F14C00984753
:10D6D800FFF714B89F49A04BD1F8EC101B6844F62B
:10D6E80020608142A8BF0146B1F57A7FB8BF4FF4E8
:10D6F8007A7189B213F0100FA4F8B211DAF8003079
:10D7080000F0F583DB0441F1C5858F4BD3F800E0C9
:10D71800BEF832707F08864D9048D4F8B431D5ED04
:10D72800037AA0FB01018809642191FBF0F1142917
:10D73800BDEEE77A04EB4305A8BF142101338B4201
:10D74800C4F8B43117EE10CAA4BF0023C4F8B4312A
:10D7580004EB4303A5F8B8C1B3F9B83107EE103AA2
:10D76800B8EEC77A77EEC77AFDEEE77ACDED067A9E
:10D77800BDF9181081EAE173A3EBE173BB4201F331
:10D78800FE8677494FF07E530B60FEF7E4BF754B7A
:10D798000593754CE8E41E216F48F4F750FC002807
:10D7A8003FF4F7A9634B1B8858063FF5F2A994F894
:10D7B8000432AB4242F08582694BD4ED827AD3EDD4
:10D7C800016A94ED505ADFED695A9FED696A27EEB8
:10D7D800C57A68EE277AA8EE267AE5EE267AB4EEC0
:10D7E800E57AF1EE10FA88BFB0EE657AB4EEC67A43
:10D7F800F1EE10FAF4EEE57AB8BFB0EE467AF1EE43
:10D8080010FA88BFF0EE657AF4EEC67AF1EE10FAF7
:10D81800B8BFF0EE467A84ED4E7AC4ED507AFFF741
:10D82800B8B9FDEEC87A534A17EE903A9780D3807C
:10D83800FFF7AAB9DFED506AFFF753BADAF800101C
:10D848004B023EF5D9ADFEF7DBBDB4EEC87AF1EE7A
:10D8580010FA98BFB0EE478ABDEEC77AB4EEE68AF2
:10D86800DFF810C1F1EE10FA17EE103AB8BFB0EEBB
:10D87800668A84ED4E8AACF80030BEF1000F7FF462
:10D88800A3A8FFF781B99FED397ADFED396A3949E5
:10D89800F4EEC77AF1EE10FA98BFB0EE677AFDEEB3
:10D8A800E77AB4EEE67AF1EE10FA17EE903AB8BFDE
:10D8B800B0EE667ABEF1010F84ED4F7A4B803FF7E8
:10D8C800E9A8FFF761B9BDEEE77A2A4B17EE102AEF
:10D8D8009A80FFF742B9002B3EF4E4AAFEF7C1BADA
:10D8E800F7F73AFF059B23491A78069B072AA0EB0E
:10D8F800030088807EF4FCAEF7F72EFF0646FEF79D
:10D90800F8BEF7F729FF059BDFF868801A780A9BAD
:10D91800012AA0EB0300A8F8020000F0CB82072A36
:10D928007EF4E8AAF7F718FF0690FEF7E5BA00BFFD
:10D938008C4D0020B44F0020644F00206766666657
:10D94800906700201C770020B84F002089888888BD
:10D95800506D0020F41B002074670020D34D621026
:10D9680004000020044C0020F024002000C0F944EA
:10D9780000C0F9C4084C002000000000002A00F094
:10D98800F981D4ED583A94ED574AD4ED627AF349C7
:10D9980094ED617A91ED005AD4ED555A94ED546A9C
:10D9A800EF4DF048F4EEC43AF3EE046AF1EE10FAE3
:10D9B80077EEA64A00F1208395ED026A26EE656AA5
:10D9C800B0EE674AA6EE074AB4EEE44A34EE666A59
:10D9D800F1EE10FA48BFB0EE456A012A80ED006A00
:10D9E80000F0C88195ED066A26EE656AB0EE674AD2
:10D9F800A6EE074AB4EEE44A34EE666AF1EE10FA8F
:10DA080048BFB0EE456A022A80ED016A00F0B28193
:10DA180095ED0A6A26EE656AB0EE674AA6EE074AF1
:10DA2800B4EEE44A34EE666AF1EE10FA48BFB0EE9E
:10DA3800456A032A80ED026A00F09C8195ED0E6A22
:10DA480026EE656AB0EE674AA6EE074AB4EEE44AE7
:10DA580034EE666AF1EE10FA48BFB0EE456A042A61
:10DA680080ED036A00F0868195ED126A26EE656AFC
:10DA7800B0EE674AA6EE074AB4EEE44A34EE666AA8
:10DA8800F1EE10FA48BFB0EE456A052A80ED046A47
:10DA980000F0708195ED166A26EE656AB0EE674A69
:10DAA800A6EE074AB4EEE44A74EE666AF1EE10FA9E
:10DAB80048BFF0EE456A062AC0ED056A00F05A81B3
:10DAC800D5ED1A6A66EEE56AB0EE674AA6EE874AB1
:10DAD800B3EE046AB4EEE44A74EE466AF1EE10FA64
:10DAE80048BFF0EE456A072AC0ED066A00F0428199
:10DAF800D5ED1E6ADFF874A2DFF8749266EEE55A77
:10DB0800E5EE877AF4EEE47A77EEC67AF1EE10FA6B
:10DB180048BFF0EE457AC0ED077AFEF7C9BDB8F107
:10DB2800000F41F03D828E4D9DED0E5A95ED006A35
:10DB38008C4825EE866AA5EE076AB0EE675AA6EE0F
:10DB4800265ABDEEC56A16EE10EA16EE107AE645BC
:10DB5800A8BF67467145C8BF0F4606EE107AB8EEF3
:10DB6800C66A012A80ED006A3FF4B1AC95ED046AFB
:10DB78009DED0F5A25EE866AA5EE076AB0EE675A44
:10DB8800A6EE265ABDEEC56A16EE10EA16EE107A13
:10DB9800E645A8BF67467145C8BF0F4606EE107A2E
:10DBA800B8EEC66A022A80ED016A3FF490AC95EDA2
:10DBB800086A9DED105A25EE866AA5EE076AB0EE52
:10DBC800675AA6EE265ABDEEC56A16EE10EA16EE9C
:10DBD800107AE645A8BF67467145C8BF0F4606EEEE
:10DBE800107AB8EEC66A032A80ED026A3FF46FAC79
:10DBF80095ED0C6A9DED115A25EE866AA5EE076A29
:10DC0800B0EE675AA6EE265ABDEEC56A16EE10EAC1
:10DC180016EE107AE645A8BF67467145C8BF0F469D
:10DC280006EE107AB8EEC66A042A80ED036A3FF45D
:10DC38004EAC95ED106A9DED125A25EE866AA5EE5A
:10DC4800076AB0EE675AA6EE265ABDEEC56A16EE0A
:10DC580010EA16EE107AE645A8BF67467145C8BFB8
:10DC68000F4606EE107AB8EEC66A052A80ED046AF9
:10DC78003FF42DAC95ED146A9DED135A25EE866A96
:10DC8800A5EE076AB0EE675AA6EE265ABDEEC56A3B
:10DC980016EE10EA16EE107AE645A8BF67467145FB
:10DCA800C8BF0F4606EE107AB8EEC66A062A80ED9F
:10DCB800056A3FF40CAC95ED186A9DED145A25EEF3
:10DCC800866AA5EE076AB0EE675AA6EE265ABDEE3A
:10DCD800C56A16EE10EA16EE107AE645A8BF674642
:10DCE8007145C8BF0F4606EE107AB8EEC66A072A15
:10DCF80080ED066A3FF4EBAB95ED1C6A9DED155A75
:10DD080065EE865AE7EE055AE6EEA57AFDEEE77A65
:10DD180017EE905AAC45A8BFAC46A942C8BF8C467E
:10DD280007EE90CAF8EEE77AC0ED077AFFF7CCBBAA
:10DD3800DFED0D6AFEF72BBEDFED0B6AFEF708BFBD
:10DD4800B5EEC07AF1EE10FA01F19482B7EE006AEE
:10DD580036EE477AC6EE076AFEF780BE4C550020BD
:10DD680050550020044300200000C8428C6F00205A
:10DD7800A8560020DFF874A2DFF87492FEF798BC6A
:10DD880084494A79002A3EF4B9A9834A1278002ABC
:10DD98003EF4B4A90B788149DFED814A07EE903A49
:10DDA8000B88B8EE677A07EE902A06EE903AF8EEFE
:10DDB800E77AF8EE666A67EE277AB7EE007A87EEBA
:10DDC800A63AB4EEE43AF1EE10FA88BFB0EE643A3F
:10DDD800B4EEC73AF1EE10FAB8BFB0EE473AFEF724
:10DDE8008FB9704B5988FEF7C9BCB4F8B21101F568
:10DDF8007A7189B2FEF7C2BC6B4B93ED006AFEF7ED
:10DE080052BF6A4F3B78013B0D2B24D8DFE813F053
:10DE1800DF07ED07A3077107230023005A078E07C2
:10DE280005070E00E606DA06CF06C306604B1B7828
:10DE3800002B02F020811A2022F094FB002842F0E7
:10DE48001A815C4B1B78002B42F0158109233B702B
:10DE58001CF0ACF9AA78012A00F05B852B79012B1C
:10DE680001F08585022B7EF49FAE3B78012B7EF472
:10DE78009BAE504B1B78002B7EF496AE1BF00AFE2F
:10DE8800FEF792BE4C4B9FED4D7AD3ED087AF4EE37
:10DE9800C77AF1EE10FA00F2F1849FED497A494D04
:10DEA800D5ED037A77EE877AC5ED037AFEF74EBC97
:10DEB800DFF84081F7F750FC4349D4F87C21096822
:10DEC8000690821A511AC4F87C01A8F80420A8F810
:10DED8000610FEF711B8F7F73FFC0A90FDF795BD5D
:10DEE8003A4B9B7B002B3EF424ACFEF727BCDD00AD
:10DEF8003FF508ACFEF72FBCB4F88C51954240F2C0
:10DF08001E8594F8A451002D40F0E387304A314E25
:10DF180092ED007AD6ED007A94F99821C4ED647AEE
:10DF280077EE676A012AC4ED627AC4ED616A84ED0E
:10DF3800657A02F07E80079BC4F89C31264A9FEDE3
:10DF4800207A92ED005A84ED687A012284F89821AB
:10DF5800FEF73CBF214B1B88002B40F00486204A6B
:10DF6800204B11781868F8F7AFFAD4F86C21079BA2
:10DF78009A1AFDF700BE1C4BD9ED007A93ED007A92
:10DF8800F0EEE77AF4EEC77AF1EE10FA7DF78AAF91
:10DF9800FDF77ABF484F00208A4D0020244D00200D
:10DFA800713DAA3FB852002008550020CE3D002000
:10DFB80046430020BD650020047900208FC2753CCF
:10DFC800000000008C4D002028430020E86A002053
:10DFD8007C670020D0550020EC550020F057002029
:10DFE800F2570020F4570020405500208C6F002085
:10DFF800A8560020084C0020D5ED015A65EEC65AF7
:10E00800B0EE674AA5EE874AB4EEE44A74EE665A63
:10E01800F1EE10FA48BFF0EE455A012AC0ED005A59
:10E028003FF4A8AED5ED055A65EEC65AB0EE674A7C
:10E03800A5EE874AB4EEE44A74EE665AF1EE10FA99
:10E0480048BFF0EE455A022AC0ED015A3FF492AE9D
:10E05800D5ED095A65EEC65AB0EE674AA5EE874A6D
:10E06800B4EEE44A74EE665AF1EE10FA48BFF0EEE8
:10E07800455A032AC0ED025A3FF47CAED5ED0D5A3D
:10E0880065EEC65AB0EE674AA5EE874AB4EEE44A92
:10E0980074EE665AF1EE10FA48BFF0EE455A042ABB
:10E0A800C0ED035A3FF466AED5ED115A65EEC65A77
:10E0B800B0EE674AA5EE874AB4EEE44A74EE665AB3
:10E0C800F1EE10FA48BFF0EE455A052AC0ED045AA1
:10E0D8003FF450AED5ED155A65EEC65AB0EE674A14
:10E0E800A5EE874AB4EEE44A74EE666AF1EE10FAD9
:10E0F80048BFF0EE456A062AC0ED056A3FF43AAE1D
:10E10800D5ED196A66EEC66AB0EE674AA6EE874A8A
:10E11800F3EE045AB4EEE44A74EE656AF1EE10FACE
:10E1280048BFF0EE456A072AC0ED066A3FF422AE02
:10E13800D5ED1D6ADFF8D4A3DFF8D49326EEC66ABE
:10E14800E6EE077AF4EEE47A77EEE57AF1EE10FA85
:10E15800B8BFF0EE457AC0ED077AFEF7A9BA089B7A
:10E16800E24D002B41F0B08095ED006A9DED0E5A0E
:10E17800DF4825EE866AFDEEE44AA5EE076AB0EEB2
:10E18800675AA6EE265A14EE901ABDEEC56A16EE28
:10E1980010EA16EE107AE645A8BF67467145C8BF73
:10E1A8000F4606EE107AB8EEC66A012A80ED006ABC
:10E1B8003EF47AAA95ED046A9DED0F5A25EE866A1B
:10E1C800A5EE076AB0EE675AA6EE265ABDEEC56AF6
:10E1D80016EE10EA16EE107AE645A8BF67468E4599
:10E1E800B8BF0F4606EE107AB8EEC66A022A80ED6E
:10E1F800016A3EF459AA95ED086A9DED105A25EE7C
:10E20800866AA5EE076AB0EE675AA6EE265ABDEEF4
:10E21800C56A16EE10EA16EE107AE645A8BF6746FC
:10E228008E45B8BF0F4606EE107AB8EEC66A032AC6
:10E2380080ED026A3EF438AA95ED0C6A9DED115AFC
:10E2480025EE866AA5EE076AB0EE675AA6EE265A4C
:10E25800BDEEC56A16EE10EA16EE107AE645A8BFBE
:10E2680067468E45B8BF0F4606EE107AB8EEC66A06
:10E27800042A80ED036A3EF417AA95ED106A9DED15
:10E28800125A25EE866AA5EE076AB0EE675AA6EE20
:10E29800265ABDEEC56A16EE10EA16EE107AE64565
:10E2A800A8BF67468E45B8BF0F4606EE107AB8EE8F
:10E2B800C66A052A80ED046A3EF4F6A995ED146A4B
:10E2C8009DED135A25EE866AA5EE076AB0EE675AE9
:10E2D800A6EE265ABDEEC56A16EE10EA16EE107ABC
:10E2E800E645A8BF67468E45B8BF0F4606EE107ACA
:10E2F800B8EEC66A062A80ED056A3EF4D5A995ED02
:10E30800186A9DED145A25EE866AA5EE076AB0EEE6
:10E31800675AA6EE265ABDEEC56A16EE10EA16EE44
:10E32800107AE645A8BF67468E45B8BF0F46FEF788
:10E3380099B9704ED4ED017A94ED006A318872690A
:10E3480077EEA77AF0EE006AB0EE677AA6EE267A44
:10E358004E1E04EBC601D6EE267A08391032F6EEC8
:10E36800003A27EE237A67EEA37A84ED207AC4ED8B
:10E37800217A614C274604F1800091ED027A91EDF3
:10E38800036AD7ED036AD7ED027A52ED014A12ED1E
:10E39800025A37EE674A76EEC65A77EE277AE4EEE7
:10E3A800845A013EA1F10801E5EE047A07F1080755
:10E3B80002F1080236EE267A00F10800E4EE877AC8
:10E3C800E5EE475A67EEA37A25EEA37AC0ED007A08
:10E3D80080ED017AD1D1BEF1140F7EF4B8AEF7F713
:10E3E800BBF9069BDFF82C81C01AA8F80200D4F804
:10E3F8001451FEF7ACBED4F818C1B4F81031C3F10B
:10E4080020025FFA82F93D4A03EB4C1702EB8707BB
:10E418005FEA990201F02A86013216013848394923
:10E4280007EB060807F1100212ED024A12ED035A33
:10E4380012ED016A12ED047A50ED024A50ED035ACA
:10E4480050ED016A50ED047A64EE244A65EE255ACF
:10E4580066EE266A67EE277A1032904541ED024A49
:10E4680041ED035A41ED016A41ED047A00F11000D3
:10E4780001F11001D8D12448A6F110010F4400EB96
:10E488000108214419F0030209D0B7EC017AF8EC2D
:10E49800017A67EE277A013AE1EC017AF5D1002B8F
:10E4A80041F07C80BEF1140F7EF451AEF7F754F9B9
:10E4B800069BDFF86080D4F81451C01AA8F802004F
:10E4C800FEF745BE0B4E0C48B268B18924F0F0F94E
:10E4D800059B93F800E0BEF1140F01F0E085D4F835
:10E4E80014510135C4F8145124E700BF50550020D9
:10E4F80004430020983F0020F0240020B03F002073
:10E508004041002000250020304100208C6F002071
:10E51800A8560020084C0020C74E318873684FEA7F
:10E5280051094FEA89005FEAD10C04EB000204EBC1
:10E53800810500F0A18000F110010CF1010CBF4F22
:10E5480002EB0C1C2944103203F1100E05F11000E7
:10E5580050ED032A50ED043A17ED043A17ED032A5B
:10E5680050ED026A10ED016A17ED021A57ED010A23
:10E5780011ED044A11ED035A52ED044A52ED035AC3
:10E5880012ED027A52ED017A51ED021A11ED010AEB
:10E5980073EE238A32EE228A47ED048A07ED038A56
:10E5A80071EE268A30EE868A47ED028A07ED018AE7
:10E5B80074EE848A35EE858A42ED048A02ED038A78
:10E5C80077EE218A37EE808A42ED028A02ED018ACF
:10E5D80073EE633A75EE655A1EED035A32EE623AEF
:10E5E80074EE644A25EE638A1EED044A23EE052A7A
:10E5F80064EE652AA3EE048A1032944524EE843A28
:10E60800A3EE842A07F110070EF1100EA5EE853A45
:10E6180000F1100001F11001E4EE852A00ED078AEF
:10E6280000ED082A01ED073A41ED082A5EED055A8A
:10E638001EED065A71EE666A30EEC66A31EEC77A8A
:10E6480070EE677A26EE253A65EEE63A25EE674AD9
:10E6580067EE054AE6EE053AA6EE853AA7EE254AA4
:10E66800E7EEA54A00ED063A40ED053A01ED064A07
:10E6780041ED054A7FF46CAF1FFA89F91A464946FD
:10E688006F4816F005FA72684946284616F000FAEF
:10E69800059B1A78142A7FF4AAAEA0E6694E317851
:10E6A8005FEA910C01F02386674F0CF101094FEAEC
:10E6B800491907EB090807F12002A7F1700012EDCC
:10E6C800076A52ED056A12ED037A52ED017A52EDAE
:10E6D800025A12ED084A52ED064A12ED045A26EE85
:10E6E800066A66EEA66A27EE077A67EEA77AA4EEB0
:10E6F800046A20329045E4EEA46A00F11000A5EE09
:10E70800057AE5EEA57AF1EEC65AB1EEE66AF1EEC3
:10E71800C76AB1EEE77A40ED085A00ED076A40EDA6
:10E72800066A00ED057ACAD1A9F120023A4404EB41
:10E738000C1711F0030018BF08320FD052ED017A00
:10E7480012ED027A67EEA77A0138E7EE077A02F14E
:10E758000802B1EEE77AA7EC017AEFD1BEF1140F07
:10E7680001F0AA840135C4F81451FEF75FBCD4F84F
:10E77800185136493648374BEA00114415448A88FF
:10E78800196800EE102A643AC82AA8BFC822782A55
:10E79800B8BF782207EE902AB8EEC07AF8EEE77A8A
:10E7A80000EB850577EE670A77EE876A67EE877A6A
:10E7B80020EEA67AB8EE400AC7EE870A2846D5F8B2
:10E7C8001490D5F81880EF692E6A16F09BFD059B0A
:10E7D800C5F8149093F800E0C5F81880BEF1140F3E
:10E7E800EF612E6201F04E84D4F818211A49D4F84A
:10E7F8001451013281FB0213A3EBE27C0CEB4C03B6
:10E80800A2EB030C0135C4F818C1C4F81451F4E59F
:10E81800F6F7A2FF059B069093F800E0BEF1140FEF
:10E8280005BFDFF83880D4F81451D4F81451A8F88B
:10E838000050FCF7ECBF00BF983F002000250020E7
:10E84800F0240020923F00207025002088420020FC
:10E85800106F00207C6F002056555555084C00203D
:10E86800306E99BC2716983DA40DC93F843459BE13
:10E87800DB0F4940D06D393A00000000F0EEE76A3E
:10E88800B7EE005A35EE665A1FED0B4A5FED0B5A8C
:10E898001FED0A6A1FED0C7A94ED6B0AF1EEC54A7A
:10E8A800E6EE845AF5EEC07AA6EEA56AF1EE10FA05
:10E8B800A6EE867A48BF5FED127A27EE247A48BF23
:10E8C80037EEC77A27EE000A25F026F9B0F5617F02
:10E8D80000F3C18607EE900AF8EEE76A5FED1B7A4F
:10E8E80066EEA76A07EE905ABDEEE67AF8EEE77A8A
:10E8F80017EE103A2033402B41F2B3841FED220A61
:10E9080025F00AF900B207EE900AB8EEE77AFFF7A9
:10E91800C6BAD549D54B89681B6899423FF69EAA65
:10E928003B780C3B022B7EF63FA9D14C3A702378FA
:10E93800002B3EF439A900232370FEF735B9CD4AE0
:10E9480002F1500503E00432954200F0C2821378C8
:10E95800262BF8D19678D3789E42F4D2FFF7D1BA15
:10E96800C54DC64F95ED004A95ED057AD5ED014A9E
:10E9780095ED066AD5ED046A95ED035AD5ED025A70
:10E9880067EE897A07EB8602A4EE277AA4EEA76AD7
:10E9980066EEC76AA5EE476AE5EEA76A20EE070AA3
:10E9A80085ED056AC5ED066A82ED007A29EE088ACA
:10E9B80025F0B2F869EE288AD5ED0E5AD5ED176A1A
:10E9C80095ED091AD5ED121A95ED0F5A95ED187AAD
:10E9D80095ED0A2AD5ED132A95ED0D6AD5ED167A2F
:10E9E80095ED0C3AD5ED0B3A95ED154AD5ED144A4F
:10E9F800E1EE085A002207EB8601E8EEA16A00B2B0
:10EA0800C4F80021A2EE085AC4F80421C4F8082169
:10EA1800A8EEA27A26EE656A67EEE67AA3EE655A54
:10EA2800A3EE886AA6EEC47AE8EEA47A85ED0E5ABB
:10EA3800C1ED205A85ED0F6AC1ED406A85ED177A60
:10EA4800C5ED187AFEF7ACBAD4F89C51079B5D1B4C
:10EA5800FEF7ACB9BBF93820CBF8201007EE902AA6
:10EA68000121F8EEE77ACBF86020CBF87C10002281
:10EA7800012FCBED1C7ACBED1B7ACBF8742001F07B
:10EA8800D082B7427CF427AFBBF93A20CBF8642098
:10EA980007EE902A00210122F8EEE77ACBF824103D
:10EAA800CBF890200022012FCBED217ACBED207AF4
:10EAB800CBF8882001F0B982B7427CF440AFBBF9AB
:10EAC8003C20CBF8682007EE902A00210122F8EEBE
:10EAD800E77ACBF82810CBF8A4200022012FCBED41
:10EAE800267ACBED257ACBF89C207CF45CAF9FEDA1
:10EAF800648A032D49D04CB107EE904AF8EEE77AC4
:10EB0800F4EEC87AF1EE10FA01F102845D4A5E4C27
:10EB18001168DBF86820A8F8060094F8200102EBD9
:10EB2800560292FBF6F60022CBF828608A620A6346
:10EB3800CA6228B1554A126832F480637CF436AF51
:10EB4800534A126812F4003241F063825148114668
:10EB5800835C012B02F10C0200F0F48401311829C6
:10EB6800F6D1FCF723BF4C494B69002B3DF403A8B1
:10EB78004A484B4B008893FBF0F00B684FF0010EAE
:10EB8800186081F811E0FCF7F6BFB0EE480A24F0EF
:10EB9800C3FF00B2AFE71F20069221F0E3FC069AFC
:10EBA80000287FF458A901233B70FFF754B9012AC4
:10EBB80001F0B5830E2313203B7009F0C5FFAA7836
:10EBC800FFF749B9012A01D1F3F78AFC0D23132075
:10EBD8003B7009F0B9FFAA78FFF73DB9314B3249CC
:10EBE8005B680968C8338B4205D30BF081FCAA78AF
:10EBF80000283FF430A9032AD5D1DFF8C480D8F81B
:10EC0800000009F0F1FA294B1B780022022BC8F802
:10EC1800002001F03984AA78C5E71A2021F0A2FC67
:10EC280000283FF415A9224B1B88002B7FF410A95C
:10EC3800204B4520D3F800801AF000FE0E201AF071
:10EC4800FDFD40461AF0F0FEDDF81C8040461AF043
:10EC5800EBFE194A194B12681A6040460A233B70AA
:10EC68001AF08CFFFFF7F4B8FC1900202C430020A1
:10EC7800BD650020646900201C420020B03F0020D0
:10EC88000000000000790020F0240020B04F002090
:10EC9800B8340020A0590308F85700201058002065
:10ECA80020A1070080670020185800202443002076
:10ECB800C4650020C0650020D4650020CC65002014
:10ECC8008C3E00200BF0EEFBA34B002105208DE8C5
:10ECD8000300A3F10802029153200BF049FF00281A
:10ECE8007FF46DAF9D4BAA78186008233B70FFF73F
:10ECF800B2B80BF0D7FB9A4A0292A2F10C032A2170
:10ED080001930091A2F10A035021163A49200BF011
:10ED18002FFF00287FF453AF904BAA7818604FF06C
:10ED2800FF31596007233B70FFF795B80BF0BAFB2A
:10ED38001BF072FA00283FF442AF0BF0D9FB002811
:10ED48003FF43DAF874A884B12681A600A233B702C
:10ED5800AA78FFF780B8DFF804820BF0A3FB834A98
:10ED6800D8F80430126864339342BFF428AF4020C7
:10ED78000BF06EFB00287FF422AFD8F80030DFF8E4
:10ED88001CA2DFF8F0B14FF040090FE01AF056FD71
:10ED9800DBF80020D8F80030013A0133B9F1010955
:10EDA800CBF80020C8F8003001F02C831AF80330A3
:10EDB8001846002BEAD100234FF0FF32C8F8003084
:10EDC8000423C8F804203B70AA78FFF744B8684BBE
:10EDD8001B78D90701F1AA821F2021F0C3FB002864
:10EDE8003FF4EDAE0C233B70E9E6604B5B491B68D2
:10EDF8004B60604800230B60032103603970FFF704
:10EE08002AB8DFED5D7A5D4B94ED687AC3ED007A40
:10EE1800C3ED017AC3ED027A594BF0EE674AF0EE82
:10EE2800673A1968FDF7A2B8564A574DD2ED006AFD
:10EE3800564A95ED006A1278C4ED646A84ED656AF5
:10EE4800002A00F01B8276EE665A94F99821C4EDE8
:10EE5800615A0132C4ED626A00F08085079BC4F8EC
:10EE68009C31002537EE677AFCEEE77A484E84ED50
:10EE7800687A17EE902AA4F88C21FF2296ED005AA2
:10EE880084F89821FDF7A2BF4249DFED437A09686B
:10EE9800C4ED4C7A11F080530A9340F0D083DAF82D
:10EEA800001011F480030A9300F0FB8100230A93F9
:10EEB800B6EE007A67EE877AF4EEE57AF1EE10FAAC
:10EEC800C8BFF0EE675A40F3BA83C4ED685AFDF73D
:10EED80097BA2C4A2C4DD2ED007A2C4A95ED007A3F
:10EEE8001278C4ED647A84ED657A002A00F04283D2
:10EEF80077EE676A94F99821C4ED616A0132C4ED2E
:10EF0800627A00F0B686079BC4F89C3100259FED15
:10EF18001A7A1F4E84ED687AFF2296ED005A84F81B
:10EF28009821FDF753BF124B1D7805F00108FDF736
:10EF3800BBBB73EEE77AB7EE007AF4EEC77AF1EE70
:10EF480010FAC4ED4C7A41F37A8084EEA77A8DEDFD
:10EF58000E7AFDF74ABA00BFDC5303088067002029
:10EF6800F2510308D4650020CC6500201858002011
:10EF7800E5750020883E002000000000B042002017
:10EF8800B84F0020EC650020D4550020DC7100202B
:10EF9800E855002074670020000000808C510308A9
:10EFA800C54D0D9B9DED0E5A95ED006A002B00F0A6
:10EFB800198725EE866AC148A5EE076AB0EE675A3A
:10EFC800A6EE265ABDEEC56A16EE10EA16EE107ABF
:10EFD800E645A8BF67467145C8BF0F4606EE107ADA
:10EFE800B8EEC66A012A80ED006A3DF461AB95ED82
:10EFF800046A9DED0F5A25EE866AA5EE076AB0EE03
:10F00800675AA6EE265ABDEEC56A16EE10EA16EE47
:10F01800107AE645A8BF67467145C8BF0F4606EE99
:10F02800107AB8EEC66A022A80ED016A3DF440AB58
:10F0380095ED086A9DED105A25EE866AA5EE076AD9
:10F04800B0EE675AA6EE265ABDEEC56A16EE10EA6D
:10F0580016EE107AE645A8BF67467145C8BF0F4649
:10F0680006EE107AB8EEC66A032A80ED026A3DF40D
:10F078001FAB95ED0C6A9DED115A25EE866AA5EE3B
:10F08800076AB0EE675AA6EE265ABDEEC56A16EEB6
:10F0980010EA16EE107AE645A8BF67467145C8BF64
:10F0A8000F4606EE107AB8EEC66A042A80ED036AA7
:10F0B8003DF4FEAA95ED106A9DED125A25EE866A7A
:10F0C800A5EE076AB0EE675AA6EE265ABDEEC56AE7
:10F0D80016EE10EA16EE107AE645A8BF67467145A7
:10F0E800C8BF0F4606EE107AB8EEC66A052A80ED4C
:10F0F800046A3DF4DDAA95ED146A9DED135A25EED8
:10F10800866AA5EE076AB0EE675AA6EE265ABDEEE5
:10F11800C56A16EE10EA16EE107AE645A8BF6746ED
:10F128007145C8BF0F4606EE107AB8EEC66A062AC1
:10F1380080ED056A3DF4BCAA95ED186A9DED145A58
:10F1480025EE866AA5EE076AB0EE675AA6EE265A3D
:10F15800BDEEC56A16EE10EA16EE107AE645A8BFAF
:10F1680067467145C8BF0F4606EE107AB8EEC66A04
:10F17800072A80ED066A3DF49BAA95ED1C6A9DED71
:10F18800155A65EE865AE5EE075AE6EEA57AFDEEC3
:10F19800E77A17EE902A9445A8BF94469142D8BFC3
:10F1A800614607EE901AF8EEE77AC0ED077AFDF7A8
:10F1B8007FBABEF1010F40F3348707EE103AB8EE7C
:10F1C800C77AC7EE876AB1EEE68A032D13D04CB131
:10F1D80007EE904AF8EEE77AF4EEC87AF1EE10FA04
:10F1E80001F19680DBF8602002EB560292FBF6F202
:10F1F800CBF8202045E4B0EE480A24F08DFC00B29C
:10F20800E5E7BEF1010F7FF772AC07EE103AB8EEF2
:10F21800C77AC7EE876AB1EEE68A6AE4BEF1010FE3
:10F2280040F3038707EE103AB8EEC77AC7EE876A4D
:10F23800B1EEE68A032D13D04CB107EE904AF8EEF2
:10F24800E77AF4EEC87AF1EE10FA01F16180DBF8A2
:10F25800642002EB560292FBF6F2CBF824202BE452
:10F26800B0EE480A24F058FC00B2E5E7F7EE006A71
:10F27800FDF76EBCF7EE006AFDF7F0BB76EEC65AF6
:10F28800F0EE466AE1E58222FDF74EBFDFED0C7A2B
:10F29800FDF716BF0B4BD3F800E0BEF93270FEF74E
:10F2A8003ABAB6EE007AF4EEC75AF1EE10FA3FF722
:10F2B800FFADFDF7A5B800BF50550020044300205E
:10F2C80000000243B84F002095ED006A9DED0E4AFC
:10F2D800EE4825EE866AFDEEE43AA4EE076AB0EE43
:10F2E800674AA6EE264A13EE901AB4EEC45AF1EE17
:10F2F80010FAB0EE446A88BFB0EE646ABDEEC66A22
:10F3080016EE10EA16EE107AE645A8BF6746714574
:10F31800C8BF0F4606EE107AB8EEC66A012A80ED1D
:10F32800006A3DF4C1A995ED046A9DED0F4A25EEEA
:10F33800866AA4EE076AB0EE674AA6EE264AB4EEDD
:10F34800C45AF1EE10FAB0EE446A88BFB0EE646AAF
:10F35800BDEEC66A16EE10EA16EE107AE645A8BFAC
:10F3680067468E45B8BF0F4606EE107AB8EEC66AF5
:10F37800022A80ED016A3DF497A995ED086A9DED92
:10F38800104A25EE866AA4EE076AB0EE674AA6EE32
:10F39800264AB4EEC45AF1EE10FAB0EE446A88BFB9
:10F3A800B0EE646ABDEEC66A16EE10EA16EE107A82
:10F3B800E645A8BF67468E45B8BF0F4606EE107AE9
:10F3C800B8EEC66A032A80ED026A3DF46DA995ED90
:10F3D8000C6A9DED114A25EE866AA4EE076AB0EE26
:10F3E800674AA6EE264AB4EEC45AF1EE10FAB0EE19
:10F3F800446A88BFB0EE646ABDEEC66A16EE10EACB
:10F4080016EE107AE645A8BF67468E45B8BF0F4688
:10F4180006EE107AB8EEC66A042A80ED036A3DF457
:10F4280043A995ED106A9DED124A25EE866AA4EE71
:10F43800076AB0EE674AA6EE264AB4EEC45AF1EE61
:10F4480010FAB0EE446A88BFB0EE646ABDEEC66AD0
:10F4580016EE10EA16EE107AE645A8BF67468E4506
:10F46800B8BF0F4606EE107AB8EEC66A052A80EDD8
:10F47800046A3DF419A995ED146A9DED134A25EE29
:10F48800866AA4EE076AB0EE674AA6EE264AB4EE8C
:10F49800C45AF1EE10FAB0EE446A88BFB0EE646A5E
:10F4A800BDEEC66A16EE10EA16EE107AE645A8BF5B
:10F4B80067468E45B8BF0F4606EE107AB8EEC66AA4
:10F4C800062A80ED056A3DF4EFA895ED186A9DEDD2
:10F4D800144A25EE866AA4EE076AB0EE674AA6EEDD
:10F4E800264AB4EEC45AF1EE10FAB0EE446A88BF68
:10F4F800B0EE646ABDEEC66A16EE10EA16EE107A31
:10F50800E645A8BF67468E45B8BF0F4606EE107A97
:10F51800B8EEC66A072A80ED066A3DF4C5A895EDDF
:10F528001C6A9DED154A65EE865AE7EE045AE6EE2A
:10F53800A57AB4EEE75AF1EE10FAC8BFF0EE647A95
:10F54800FDF7A2B8D4F824614A003EB1551800EB83
:10F55800850576786D78B542BCF428AA0A4400EB94
:10F5680082000022C4F82401A4F81022C4F814224E
:10F57800FCF71CBA77EEC76AF0EE477ABAE4BEF831
:10F5880034309FED437A07EE903AF8EEE77A414B34
:10F5980067EE877AC3ED007AFDF7DDB83E4A4FEA99
:10F5A800890702EBCC199A083844274436D001322F
:10F5B8004FEA021C09EB0C0809F1100200F11006D1
:10F5C80007F1100112ED024A12ED035A12ED016A19
:10F5D80012ED047A56ED024A56ED035A56ED016AC9
:10F5E80056ED047A64EE244A65EE255A66EE266ADC
:10F5F80067EE277A1032904541ED024A41ED035AF1
:10F6080041ED016A41ED047A06F1100601F110019D
:10F61800D8D1ACF1100291441044174413F0030CF4
:10F628003EF440AFB9EC017AF0EC017A67EE277A44
:10F63800BCF1010CE7EC017AF4D1FEF733BFB7EE69
:10F64800007A77EE677AF4EEE75AF1EE10FA88BF9F
:10F65800F0EE675A39E407EE905ADFED106AF8EEDB
:10F66800E77A66EEA65A9FED0E5A9FED0E6A9FED59
:10F678000E7AA5EE856A26EEA55AA5EE867AE5EEFF
:10F68800076A26EEA70AFFF73BB900BF044300202C
:10F698006F12833A04000020B03F002084F9223F13
:10F6A80092E741B99730083C15A82ABE95ED006A43
:10F6B8009DED0E4ACC4825EE866AFDEEE43AA4EEAE
:10F6C800076AB0EE674AA6EE264A13EE907AB4EEC1
:10F6D800C45AF1EE10FAB0EE446A88BFB0EE646A1C
:10F6E800BDEEC66A16EE10EA16EE101AE645A8BF79
:10F6F80061467745C8BF394606EE101AB8EEC66AA5
:10F70800012A80ED006A3DF4E2AE95ED046A9DEDB4
:10F718000F4A25EE866AA4EE076AB0EE674AA6EE9F
:10F72800264AB4EEC45AF1EE10FAB0EE446A88BF25
:10F73800B0EE646ABDEEC66A16EE10EA16EE101A4E
:10F74800E645A8BF6146BE45B8BF394606EE101A61
:10F75800B8EEC66A022A80ED016A3DF4B8AE95EDAE
:10F76800086A9DED104A25EE866AA4EE076AB0EE97
:10F77800674AA6EE264AB4EEC45AF1EE10FAB0EE85
:10F78800446A88BFB0EE646ABDEEC66A16EE10EA37
:10F7980016EE101AE645A8BF6146BE45B8BF394601
:10F7A80006EE101AB8EEC66A032A80ED026A3DF426
:10F7B8008EAE95ED0C6A9DED114A25EE866AA4EE93
:10F7C800076AB0EE674AA6EE264AB4EEC45AF1EECE
:10F7D80010FAB0EE446A88BFB0EE646ABDEEC66A3D
:10F7E80016EE10EA16EE101AE645A8BF6146BE45A9
:10F7F800B8BF394606EE101AB8EEC66A042A80ED7C
:10F80800036A3DF464AE95ED106A9DED124A25EE4B
:10F81800866AA4EE076AB0EE674AA6EE264AB4EEF8
:10F82800C45AF1EE10FAB0EE446A88BFB0EE646ACA
:10F83800BDEEC66A16EE10EA16EE101AE645A8BF27
:10F848006146BE45B8BF394606EE101AB8EEC66A1C
:10F85800052A80ED046A3DF43AAE95ED146A9DEDF3
:10F86800134A25EE866AA4EE076AB0EE674AA6EE4A
:10F87800264AB4EEC45AF1EE10FAB0EE446A88BFD4
:10F88800B0EE646ABDEEC66A16EE10EA16EE101AFD
:10F89800E645A8BF6146BE45B8BF394606EE101A10
:10F8A800B8EEC66A062A80ED056A3DF410AE95EDFD
:10F8B800186A9DED144A25EE866AA4EE076AB0EE32
:10F8C800674AA6EE264AB4EEC45AF1EE10FAB0EE34
:10F8D800446A88BFB0EE646ABDEEC66A16EE10EAE6
:10F8E80016EE101AE645A8BF6146BE45B8BF3946B0
:10F8F80006EE101AB8EEC66A072A80ED066A3DF4CD
:10F90800E6AD95ED1C6A9DED154A65EE865AE7EE63
:10F91800045AE6EEA57AB4EEE75AF1EE10FAC8BF3B
:10F92800F0EE647AFDEEE77A17EE901A8C45A8BFE0
:10F938008C468F42D8BF674607EE907AF8EEE77A92
:10F94800C0ED077AFDF7C0BD28494A69002A3CF492
:10F95800FBA90A6813604B74FCF7F6B9D4F89C51FC
:10F96800079B5D1BFFF77EBA214DFCF76DBF214B4E
:10F978001B78DA0704D413F0FDFB002840F02E852D
:10F988001D4DD4F80C222B689A423EF66EAA3B789D
:10F99800012B3DF409A9194C2278002A3DF404A949
:10F9A8000B2B19D801229A4040F6030112EA0108EC
:10F9B8007EF4C1AF12F4C06F0ED0093B012B0BD8F7
:10F9C800452019F03BFFFF2019F038FF0C4819F0CB
:10F9D800ABFE404619F032FF0A4B2A685A600B23E7
:10F9E8003B70FEF7A8BF00BF04430020F857002073
:10F9F8008C4D0020E575002018580020BD650020BA
:10FA0800707E0308806700200D9B002B00F0708338
:10FA1800E34D9DED0E4A95ED006A089B25EE866A3A
:10FA2800A4EE076AB0EE674AA6EE264AB0EE446A2C
:10FA380033B1B4EE445AF1EE10FAC8BFB0EE646ABE
:10FA4800FDEEE44ABDEEC66A14EE907A16EE101A80
:10FA58008F4214EE90EA00F3CA846145A8BF61465C
:10FA680006EE101ACF48B8EEC66A012A80ED006A81
:10FA78003CF41EAE95ED046ADDED0F4A089B25EEB9
:10FA8800866AA4EE876AF0EE674AE6EE264AB0EE8A
:10FA9800646A002B00F09884B4EEE45AF1EE10FA90
:10FAA80040F3928439466145A8BF614606EE101AB4
:10FAB800B8EEC66A022A80ED016A3CF4F9AD95ED0C
:10FAC800086ADDED104A089B25EE866AA4EE876A6F
:10FAD800F0EE674AE6EE264AB0EE646A002B00F0C4
:10FAE8006984B4EEE45AF1EE10FA40F363843946BF
:10FAF8006145A8BF614606EE101AB8EEC66A032A29
:10FB080080ED026A3CF4D4AD95ED0C6ADDED114A46
:10FB1800089B25EE866AA4EE876AF0EE674AE6EE51
:10FB2800264AB0EE646A002B00F03A84B4EEE45A38
:10FB3800F1EE10FA40F3348439466145A8BF6146B6
:10FB480006EE101AB8EEC66A042A80ED036A3CF481
:10FB5800AFAD95ED106ADDED124A089B25EE866A79
:10FB6800A4EE876AF0EE674AE6EE264AB0EE646ACB
:10FB7800002B00F00B84B4EEE45AF1EE10FA40F3D7
:10FB8800058439466145A8BF614606EE101AB8EEED
:10FB9800C66A052A80ED046A3CF48AAD95ED146ABC
:10FBA800DDED134A089B25EE866AA4EE876AF0EE1F
:10FBB800674AE6EE264AB0EE646A002B00F0DD8361
:10FBC800B4EEE45AF1EE10FA40F3D78339466145B2
:10FBD800A8BF614606EE101AB8EEC66A062A80ED7E
:10FBE800056A3CF465AD95ED186ADDED144A089B8D
:10FBF80025EE866AA4EE876AF0EE674AE6EE264AA4
:10FC0800B0EE646A002B00F0AF83B4EEE45AF1EE74
:10FC180010FA40F3A98339466145A8BF614606EE4C
:10FC2800101AB8EEC66A072A80ED066A3CF440ADA1
:10FC380095ED1C6ADDED154A089B65EE865AE4EEE3
:10FC4800875AE5EEA67A002B00F08683F4EEC57A93
:10FC5800F1EE10FA40F180833A466245A8BF624649
:10FC6800964607EE90EAF8EEE77AC0ED077AFCF7D9
:10FC78001FBDD4F89C51079B5D1BFFF748B995ED54
:10FC8800000A0893069223F047FF4749DFF84CE142
:10FC9800D1F8EC10DFF848C1069AACF800008EFBEA
:10FCA800013EC917C1EBAE1107EE901AF8EEE77ADC
:10FCB800089BFDEEE77A17EE901AACF80210FCF7F5
:10FCC800C8BD07EE905ADFED396A9FED397A84F89E
:10FCD8000452F8EEE77A67EEA67A77EE876ABDEE09
:10FCE800E66A16EE103A2033402B40F27382DFEDBD
:10FCF800316A314BBDEEE77AC3ED016A17EE103A6F
:10FD08002033402B00F23D829FED2C7AF4EEC77A27
:10FD1800F1EE10FA40F37D83DFED295A9FED296A51
:10FD280001E0F0EE477AF4EEC67AF1EE10FA37EE1B
:10FD3800E57AF6DCDFED247AB4EEE77AF1EE10FA34
:10FD480040F17183DFED1E5A9FED206A01E0B0EEAD
:10FD5800677AB4EEC67AF1EE10FA77EE257AF6D421
:10FD68009FED137AF4EEC77AF1EE10FA40F3C482ED
:10FD78009FED127A77EE677A67EEA75A9FED145ACD
:10FD88009FED146A9FED147AA5EE856A27EEA55AB1
:10FD9800A5EE867AE5EE077AC4ED827AFDF711BD05
:10FDA8005055002004430020F41B002035FA8E3CF7
:10FDB800DB0FC93F0000000004000020DB0F4940B2
:10FDC800DB0FC940E4CB1641DB0F49C0E4CB16C1B9
:10FDD80092E741B99730083C15A82ABED34D621066
:10FDE800084C002025EE866AA5EE076AB0EE675A31
:10FDF800A6EE265ABDEEC56A16EE100A814200F339
:10FE080075816045A8BF604606EE100A0A9BB8EEE9
:10FE1800C66A002B00F03C83DB48012A80ED006AAB
:10FE28003CF446AC95ED046A9DED0F5A25EE866AC2
:10FE3800A5EE076AB0EE675AA6EE265ABDEEC56A69
:10FE480016EE107AB94200F34F816745A8BF67469E
:10FE580006EE107A0A9BB8EEC66A002B00F0F6820E
:10FE6800022A80ED016A3CF423AC95ED086A9DED09
:10FE7800105A25EE866AA5EE076AB0EE675AA6EE16
:10FE8800265ABDEEC56A16EE107AB94200F32A81E9
:10FE98006745A8BF674606EE107A0A9BB8EEC66AA1
:10FEA800002B00F0C982032A80ED026A3CF400AC02
:10FEB80095ED0C6A9DED115A25EE866AA5EE076A46
:10FEC800B0EE675AA6EE265ABDEEC56A16EE107A4F
:10FED800B94200F305816745A8BF674606EE107A68
:10FEE8000A9BB8EEC66A002B00F0C482042A80ED93
:10FEF800036A3CF4DDAB95ED106A9DED125A25EED0
:10FF0800866AA5EE076AB0EE675AA6EE265ABDEED7
:10FF1800C56A16EE107AB94200F3E0806745A8BFBB
:10FF2800674606EE107A0A9BB8EEC66A002B00F008
:10FF38009782052A80ED046A3CF4BAAB95ED146A01
:10FF48009DED135A25EE866AA5EE076AB0EE675A4C
:10FF5800A6EE265ABDEEC56A16EE107AB94200F32F
:10FF6800BB806745A8BF674606EE107A0A9BB8EEC5
:10FF7800C66A002B00F09682062A80ED056A3CF4DA
:10FF880097AB95ED186A9DED145A25EE866AA5EE95
:10FF9800076AB0EE675AA6EE265ABDEEC56A16EE97
:10FFA800107AB9426CDC6745A8BF674606EE107A3E
:10FFB8000A9BB8EEC66A002B00F07E82072A80ED05
:10FFC800066A3CF475AB95ED1C6A9DED155A65EE15
:10FFD800865AE7EE055AE6EEA57AFDEEE77A17EEC1
:10FFE800902A8A4203DB6245A8BF6246114607EEA3
:08FFF800901A0A9BF8EEE77A6B
:020000040801F1
:10000000002B7FF436AE0C9B002B7FF432AE0B9BA3
:100010009E45B8BFF0EE647A2BE65E4A1278032A5A
:1000200000F0ED810022FEF795BD9FED5B8AFFF7A2
:10003000D0B89FED598AFFF701B9D4F89C51079BBE
:100040005D1BFDF77FBF5549096811F080530A9386
:100050007EF432AFFEF727BF9FED510ADFF85081E3
:1000600025EE800A23F05CFDD4F81451A8F80600B0
:10007000FDF771B84B484C498046FEF707BA079820
:1000800019F080FDFDF7E8BE0F4693E7F5F768FB32
:10009000059BDFF81C8193F800E0069BC01AA8F8C6
:1000A0000200FEF7A5BBF5F75BFB059BDFF80081BF
:1000B00093F800E0069BC01AA8F80200FEF713BAF6
:1000C000F5F74EFB059BDFF8E88093F800E0069B10
:1000D0003178D4F81451C01AA8F80400FEF746BBD2
:1000E0000F4645E70F4620E70F46FBE60F46D6E6EC
:1000F0000F46B1E608468BE60EA9BDEEE46A01EBB9
:10010000820290462948089A214D0A9B089416EECF
:10011000107A05E04145A5EC016A00F1100031D0EC
:1001200090ED006AB1EC014A25EE866AA7EE046AFA
:10013000B0EE674AA6EE864AB0EE446A32B1B4EE3B
:10014000445AF1EE10FAC8BFB0EE646ABDEEC64A7A
:1001500006EE107A14EE104AA74206DC14EE104A9E
:100160006445A8BF644606EE104AB8EEC66A002B86
:10017000D0D10C9C002CCDD10B9CA645B8BFB0EEC5
:10018000646AC7E7089CFCF797BADFED037A07E6D5
:10019000044300203C77002000000000746700202A
:1001A0000000C84230410020F024002050550020BB
:1001B000084C002092E741B99730083C15A82ABEA8
:1001C000E4CB1641DB0FC940E4CB16C1DB0FC93FBE
:1001D000DB0F4940DB0FC9BFDB0F49C0F4EEC77A24
:1001E000F1EE10FA40F30F815FED0A5A1FED0C6A31
:1001F00001E0F0EE476AF4EEC66AF1EE10FA36EE70
:10020000E57AF6DC5FED0C6AB4EEE67AF1EE10FA10
:1002100040F110815FED155A1FED156A01E0B0EE57
:10022000667AB4EEC67AF1EE10FA77EE256AF6D465
:100230001FED1A7AF4EEC76AF1EE10FA40F38480EB
:100240001FED1D7A77EE666A66EEA65A1FED275AF5
:100250001FED276A1FED277AA5EE856A26EEA55ABF
:10026000A5EE867AE5EE076A47E51FED277AF4EEFC
:10027000C76AF1EE10FA40F3E0805FED2E5A1FEDF1
:10028000306A01E0F0EE476AF4EEC66AF1EE10FA69
:1002900036EEE57AF6DC5FED306AB4EEE67AF1EE42
:1002A00010FA40F117815FED395A1FED396A01E00C
:1002B000B0EE667AB4EEC67AF1EE10FA77EE256A01
:1002C000F6D41FED3E7AF4EEC76AF1EE10FA05DDC2
:1002D0001FED417A77EE666AFFF7C7B91FED437AE3
:1002E000F4EEC76AF1EE10FA44BF1FED457A77EEDF
:1002F000666AFFF7BAB9BF4F07F18002FEF71DBA71
:100300009FEDBD7AF4EEC77AF1EE10FA44BF9FED8F
:10031000BB7A77EE677A33E5A8F80600ABF8A860F9
:10032000B44CFBF74EBBF1F7C3FE00283EF44BACD8
:10033000FEF744BC802018F0DBFD08B107F080FF19
:100340000AF080FDFEF74CBD9FEDAB7AF4EEC76A74
:10035000F1EE10FA44BF9FEDA97A77EE666A73E773
:10036000FDEEE77A17EE902ABA42FFF67EAC78E40B
:10037000BDEEC66A16EE101AB942BFF651AC394648
:1003800051E4BDEEC66A16EE101AB942BFF623ACB0
:10039000394623E4BDEEC66A16EE101AB942BFF61E
:1003A000F5AB3946FFF7F5BBBDEEC66A16EE101A7F
:1003B000B942BFF6C6AB3946FFF7C6BBBDEEC66A4B
:1003C00016EE101AB942BFF697AB3946FFF797BB46
:1003D000BDEEC66A16EE101AB942BFF668AB3946D2
:1003E000FFF768BB864B1B6803F59C530833C4F8C2
:1003F0000C32FDF73EBD14EE901AFFF735BB08F046
:100400008BFBFBF7D7BAB0EE667AFBE61AF803303F
:10041000002B7EF4D8ABFEF7D2BCB0EE677A8DE449
:1004200094F87831002B7BF461ADFBF74CBDF0EE16
:10043000477A99E4F0EE476AFAE6B0EE667A2AE780
:100440000C9B002B7FF433AD0B9B9E45B8BFB0EEE9
:10045000646A2CE50C9B002B7FF406AD0B9B9E453C
:10046000B8BFB0EE646AFFE40C9B002B7FF465AD6F
:100470000B9B9E45B8BFB0EE646A5EE50C9B002BFB
:100480007FF438AD0B9B9E45B8BFB0EE646A31E592
:1004900008F09CFAFEF7C3BB0C9B002B7FF4C0ACAA
:1004A0000B9B9E45B8BFB0EE646AB9E40C9B002B71
:1004B0007FF466AD0B9B9E45B8BFB0EE646A5FE506
:1004C0000C9B002B7FF47EAD0B9B9E45B8BFB0EE1E
:1004D000646A77E5F0EE476AF3E6132B05D1B0EED8
:1004E000480A23F01DFB099B1880B0EE480ADBF890
:1004F000083244489847059B1B78132BB0EE408A7E
:100500007DF42EA823F00CFB099B5880FDF728B83A
:10051000DFED3D7AB4EEE7EAF1EE10FA66DCDFEDEE
:100520003B7AB4EEE7EAF1EE10FA5FD4384BD3ED44
:10053000007AB1EE677AF4EEC7DAF1EE10FA52D42F
:10054000F4EEE7DAF1EE10FA88BFF0EE67DA314B3D
:1005500087ED00CA1B689342BBF620ABFBF784BB58
:100560002D4A2E4B10681B6898472D4BD7ED006A1B
:1005700093ED007A2B4BD3ED007A2B4B83ED020ADF
:100580002A4B67EE277A2B4427EEAC7AD3ED007A1C
:10059000274B67EE277AF0EE665AEDEEA75A93EDF9
:1005A000006AB1EE467AB4EEE57AF1EE10FA08DCB4
:1005B000F4EEC65AF1EE10FA8CBFB0EE467AB0EE09
:1005C000657A1C4B1B78012B02D0192B7BF4F8ABFE
:1005D000DFED197AF4EEE7DAF1EE10FACCBF012381
:1005E0000023FBF7F8BBF0EE47DAB0E7DFED13DAF4
:1005F000ADE700BFF0240020DB0FC9BFDB0F49C00F
:1006000018580020106F002000C0F84400C0F8C443
:100610004455002028550020BC540020D054002010
:100620000400002010540020A4420020E0540020C8
:10063000485500207453002000009642000000003E
:100640002DE9F04F2DED028B93B005461EF0C8FE4C
:10065000B84B1E7826B113B0BDEC028BBDE8F08F0D
:10066000B54B1B685805F6D5B44F3A68002A00F020
:100670002781B34CD4F8283103F5F43348339D4235
:10068000C0F01E81DFF8148394F82C11D8F80030E4
:10069000C4F82851013184F82C11990701F1228105
:1006A00013F0140F41F0978013F0080F94F82C31D9
:1006B00040F07C8113F0070901F04581282BA14B04
:1006C000029301F04A825E2090479F4B1B78002BDB
:1006D0006BD09B4C9D4AD4F83031EB1A934201F217
:1006E0000380DFF8BCA29AF80080B8F1000F33D184
:1006F000DFF86892D9F80000F5F7B6FAC0B2012821
:100700000ED90228924F41F027833B78002B41F00D
:10071000E284D4F83831EB1AB3F57A6F81F06D8545
:100720008C480768002F40D09AF80030BBB98A4B3C
:10073000D9F800001B689B781E3B012B4FF002018B
:1007400041F2D58404300FF06FFD012200238AF8B6
:10075000002084F8443126E07E4807682FB3D4F89F
:10076000403140F6B732EB1A93421ED994F83C312F
:10077000002B01F0E882013BDBB284F83C31002B16
:1007800001F0D08117F8011B94F84421076094F818
:10079000453172480A440133006884F8442184F8E2
:1007A0004531F5F765FAC4F840516D4A029B12785D
:1007B0001B68012A03F101030A9300F0E686694BE6
:1007C0001B786BB1684F3B6853B1029B5C4CD3F80C
:1007D00000B0D4F85831ABEB0303632B00F28A86E8
:1007E000DFF8C08198F800A0BAF1020F01F076811D
:1007F000574F97F87430032B00F0D7875B4B1B786B
:1008000073B15B4E33685BB14D4CF4F7A9FFD4F87C
:10081000643144F61F62C31A9342834600F2068194
:10082000544B1B78002B4ED1534B1B7843B1444C97
:10083000D4F8B43203F50043E8339D4280F01B87BF
:100840004E4B1B78002B3FF406AF3D4E4C4C4D4DAC
:1008500006F2BD272068F5F707FA00283FF4FBAE43
:100860002068F5F7F9F92B7880465A1E33B12068D5
:100870002A70F5F7F9F90028F2D1ECE6032239469F
:10088000781E24F0F0F896F8BC3296F8BD2286F86F
:10089000BF8283F47F4383F0FF039B1A1FFA88F81B
:1008A0009BB2B8EB132FD5D196F8BE22DBB29A4299
:1008B000D0D1781E0EF0CAFF2B7818442870C9E7F3
:1008C000204B029301E7304C2278002A40F05486F6
:1008D000DFF8D49099F80040002C40F094802B4E23
:1008E0003078002841F08283154C294ED4F8AC2290
:1008F0003178284B93FBF1F313449D4294D3264A5D
:1009000094F8B032C4F8AC52D75CF90701F1938483
:10091000BA0701F103857B0701F1ED8394F8B0324A
:100920003178013393FBF1F201FB123384F8B032DA
:100930007AE700BF685200208C6F0020D44F00205F
:100940000C270020185800208E7700203F0D030050
:100950000C000020CC4F0020C84F0020C44F0020C6
:100960008F7700209C770020585B0020A477002020
:10097000A8770020E8770020F9770020AE770020E4
:10098000B4770020B877002080770020F07700202F
:10099000F8770020A0860100F4770020584F00204F
:1009A000D04F0020E2680020F177002013F0030A06
:1009B0007FF480AE5E2090473B6814209847174B29
:1009C000174AB3F9043082FB03124FEAE379C9EB0B
:1009D000A2090FFA89F95FFA89F00FF0B5FCC9F3A3
:1009E00007200FF0B1FC3B685E2098473B681C2055
:1009F000984750460FF0A8FC50460FF0A5FC94F81D
:100A00002C313A6856E6074E376E002F41F0DD80F4
:100A1000054B89F80070C3F8AC5205E7644F00201D
:100A200067666666007800200C27002094F86A311B
:100A3000002B41F08480E04B1B6803F00802002A81
:100A400048F603414AF60B404BF60F4249F607477A
:100A500004BF02460F4613F0040F4FF0190118BFF0
:100A600017469A0684F86A1103D547F4804747F081
:100A7000200702F045FBC7F30909002841F04F8524
:100A8000CE4B9B79002B41F09F85984664204FF018
:100A9000FF3A4FF0000C0A970B97ADF834C0CDF831
:100AA0003AC0CDF83EC0CDF842C0CDF83090ADF898
:100AB0003680ADF838A08DF846000AAF0FCFDFF8CA
:100AC0000CE384F805C0AEE80F0097E80F00AEE82D
:100AD00007002EF8023B71464FF0010C1B0CFE275D
:100AE0001F20C82201F81E39A770A27184F807C020
:100AF000E07094F87A01207180F0F10383EA031327
:100B0000DAB2130983F0E70343EA022383EAC2035C
:100B10001BB283EA0312D2B2C3F3072383EA121390
:100B200043EA022383EAC2031BB283F0C80282EACB
:100B30000212D2B2C3F3072383EA121343EA022359
:100B400083EAC2031BB283EA0C0787EA0717FFB2E6
:100B5000C3F3072282EA171242EA072200EB0C03D2
:100B600082EAC7070EEB0C0084F87A31278011F86F
:100B7000013B7B4083EA0313DBB21A0982EA1722A6
:100B800042EA032282EAC3031BB29FB2814227805A
:100B9000EDD183F07C0383EA0313DBB24FEA131E2B
:100BA0008EEA172E8EEA032E8EEAC30E0FFA8EFE01
:100BB0001FFA8EF9DFF818C2A4F800905FFA8EFED3
:100BC0004FEA192984F8289084F827E00CF5D178A9
:100BD00004F1220ADCF80000DCF80410DCF808203C
:100BE000DCF80C3047460FC70CF1100CD445B84662
:100BF000F0D1DCF800003860714F9CF8043088F8C0
:100C0000043007F1270884F8C9E184F8CA9117F87D
:100C1000011F3068F5F72CF8B845F8D194F86B212E
:100C2000002A40F087876749029B08781B680A21E1
:100C300084F86B11002801F03D81DFF898E101286C
:100C4000BEF80010059141F2C6840228BEF8028069
:100C500001F07F84BEF804100491032801F074852C
:100C60000428BEF806A001F06A85BEF808100391BA
:100C7000052801F060850628BEF80AC001F05885F5
:100C80000728BEF80C1001D0BEF80E2094F87A01A7
:100C90000A93074687F0300383EA0313DBB24FEA77
:100CA000131E494806978EF07A0E4EEA032E0088EE
:100CB00027718EEAC303DFF820E1C0EB00208EFB32
:100CC000007E8644C017C0EB6E270797059F4FF044
:100CD000000967F30F09049F68F31F494FF00008EC
:100CE00067F30F08039FCDF82C901BB24FF0000E56
:100CF00083EA031067F30F0E0027C0B261F30F07FA
:100D0000C3F307236CF31F4E62F31F474FF0000C31
:100D10009DF81C20CDF834E083EA10136AF31F48D5
:100D2000CDF830800E978DF83CC08DF83D2043EA19
:100D300000230DF1280883EAC007B8E80F003FB28E
:100D400087F0C80989EA0919DFF880E084F805C04E
:100D50005FFA89F9C7F30727AEE80F0087EA19178A
:100D600047EA092398E8030083EAC9031BB283F02A
:100D700023074EF8040B87EA0717FFB2C3F30722D5
:100D800082EA1712069B704642EA072203F1010825
:100D900082EAC70720F814194FF0230CFE2116220F
:100DA000C82384F87A8127800EF1020E84F807C0E8
:100DB000A170E270A37111E0584F0020484F00204D
:100DC000AF280020B85200202477002014270020EC
:100DD0000E270020EE5B00200308208010F8013B66
:100DE0007B4083EA0313DBB21A0982EA172242EA44
:100DF000032282EAC3031BB29FB270452780EDD164
:100E000083F0F40383EA0313DBB24FEA131E8EEA86
:100E1000172E8EEA032E8EEAC30E0FFA8EFE1FFAED
:100E20008EFCD54FA4F800C04FEA1C295FFA8EFE55
:100E300084F81EE084F81F907968BA683868FB6807
:100E400007F5D17CACE80F0038697969BA6904F21A
:100E5000C118ACE8070004F2A31784F8C19184F824
:100E6000C0E117F8011F3068F4F702FFB845F8D168
:100E700094F87271002F40F06B86C04B94F87AC1E1
:100E8000B3F90010B3F90220B3F904309FEDBC6A46
:100E9000677107EE103A029B1B680A938CF06A0395
:100EA00083EA031306EE901AD9B20B0983F0D50337
:100EB00043EA012383EAC1031BB283EA03115242CE
:100EC000C9B207EE902AC3F3072383EA111343EA5A
:100ED0000123F8EEE77AF8EEE66AB8EEC77A83EA1D
:100EE000C1031BB267EE867A66EE866A27EE067A43
:100EF000002083F0C80ECDED0C7ACDED0B6A8DEDA0
:100F00000D7A0E900F9010908EEA0E180DF12809B0
:100F10005FFA88F8C3F3072EB9E80F008EEA181EAF
:100F20004EEA082E8EEAC80EDFF870820FFA8EFEA7
:100F3000A8E80F008EF01E0799E8070087EA071A55
:100F40005FFA8AFACEF3072787EA1A1747EA0A27D1
:100F500088E8070087EACA071C214FF0050A4FF00E
:100F60001E094FF0FE0EC8220CF10103E17084F857
:100F700072A184F8079084F802E0A8F11001A27130
:100F800008F10C0084F804C0278084F87A3111F845
:100F9000013B7B4083EA0313DBB21A0982EA172282
:100FA00042EA032282EAC3031BB29FB28142278036
:100FB000EDD183F0270383EA0313DBB21A0982EA37
:100FC000172282EA032282EAC3031BB21FFA83FCC0
:100FD000DFF8A481A4F800C05FFA83FE4FEA1C2C5E
:100FE00084F825C084F824E008F5D17904F1220AB8
:100FF000D8F80000D8F80410D8F80820D8F80C3039
:101000004F460FC708F11008D045B946F0D15D4FE3
:10101000B8F80030A9F8003007F1240884F8C6E1D8
:1010200084F8C7C117F8011F3068F4F721FEB845EE
:10103000F8D194F873310293002B40F08585524B20
:101040001B68052213F0140F84F8732140F08A8680
:10105000DFED4E7A94F87AC1484B4D4AB3F904104B
:10106000B2F906204B4F4C48CDED0C7A8CF02203A0
:1010700083EA03135FFA83FE4FEA1E1383F05903DA
:1010800043EA0E23B2F5FA6F83EACE031BB2A8BF80
:101090004FF4FA6283EA031EB2F57A7F5FFA8EFE9E
:1010A000B8BF4FF47A72C3F307234FF0640883EAA2
:1010B0001E13A2F57A7208FB02F243EA0E2387FBA5
:1010C000028783EACE0ED2174FF0000980FB018021
:1010D000C2EBA712C9170FFA8EF7CDF82890CDF8FA
:1010E0002C90CDF83490C1EBA00387F0C8090DF126
:1010F0002808ADF83A20ADF83830C64689EA091913
:10110000BEE80F005FFA89F9C7F3072787EA1917C6
:1011100047EA092787EAC909204FDEF800E084F88A
:1011200004C00FC70FFA89F989F04A0383EA031054
:10113000C0B2C9F3072383EA10133A460CF1010148
:1011400043EA002383EAC00342F810E900204FF08D
:101150004A094FF0FE0C4FF0140E84F87A11C821A2
:1011600060712380043784F8079084F802C084F803
:1011700003E0A171184613E00E270020644F002001
:1011800088C3E43AAF280020584F00200000000038
:10119000EE5B0020D34D6210676666661427002060
:1011A00012F8011B414081EA0111C9B20B0983EA1F
:1011B000102343EA012383EAC10109B288B2BA428B
:1011C0002080EDD181F0140181EA0111C9B24FEA0A
:1011D000111E8EEA102E8EEA012E8EEAC10E0FFA33
:1011E0008EFE1FFA8EF94FEA192CBC4BBB4884F8CF
:1011F0001DC05FFA8EFE84F81CE0B84F59689A68EB
:101200000068DB68A4F8009007F5D179A9E80F0021
:1012100038697969B7F818A0A9E8030004F2A317A0
:10122000A9F800A0BA4684F8BFC184F8BEE104F270
:10123000BF191AF8011F3068F4F71AFDD145F8D12B
:10124000A74BA84A1B781278013B12F00100DBB2D1
:1012500014BFC0214021172B03D8A34A13441B7B82
:101260000293A24B1A8893071ABF002341F0100182
:10127000012312F4027F18BF022312F0100F18BFCF
:10128000062312F0200F18BF1023002840F0A68775
:101290004FF0030994F87AC10A938CF0460383EA6D
:1012A0000313DAB2130983F0920343EA022383EAB9
:1012B000C2031BB283EA0310C0B2C3F3072282EA5F
:1012C000101242EA002282EAC00212B282F0C80E74
:1012D0008EEA0E1E00235FFA8EFE9DF808A08DF8A0
:1012E0002CA00320C2F307228DF82F9082EA1E1251
:1012F0008DF82D308DF82E108DF8300042EA0E2931
:1013000098E8070089EACE0E0FFA8EF8DFF8E0E1E0
:10131000E37188EA0819AEE803005FFA89F9C8F3B7
:10132000072888EA191848EA092181EAC90994F8C6
:1013300008808EF800200FFA89F988EA090282EA0B
:1013400002185FFA88F8C9F3072282EA181242EA03
:101350000822607AA17A94F80B90637182EAC8023D
:1013600012B2504080EA0010C0B2C2F3072282EAF3
:10137000101242EA002282EAC00212B2514081EA0F
:101380000111C9B2C2F3072282EA111242EA012214
:1013900082EAC10212B289EA020989EA09195FFAEE
:1013A00089F9C2F3072282EA191242EA092294F863
:1013B0000C80607BA17B84F804C082EAC90212B26F
:1013C00088EA020888EA08185FFA88F8C2F3072258
:1013D00082EA181242EA082282EAC80212B2504097
:1013E00080EA0010C0B2C2F3072282EA101242EA79
:1013F000002282EAC00212B2514081EA0111C9B250
:10140000C2F3072282EA111242EA012282EAC102F1
:10141000E17B94F8109013B281EA030282EA02128F
:10142000D2B2C3F3072383EA121343EA022383EA07
:10143000C2031BB289EA030282EA0212D2B2C3F3E8
:10144000072383EA121343EA022383EAC2031BB28F
:1014500083F0320282EA0212D2B2C3F3072383EA94
:10146000121343EA022383EAC2031BB29AB24FF07B
:10147000FE08DBB222800920C8210CF1010C84F89F
:1014800002804FEA1228AEF10E02E070A17184F8DA
:101490007AC184F812800293637451685EF80E0C6E
:1014A00092683EF8023C0EF5CA7CACE80700ACF846
:1014B00000309DF808308CF802900EF5D27A84F84E
:1014C000B48184F8B33117F8011F3068F4F7D0FB0A
:1014D000BA45F8D1C4F864B1FFF7A2B90E270020CD
:1014E00044430020E5750020FC530308B44F00205E
:1014F00014270020DFF8D8A3DFF8D883DFF8D893CB
:1015000041200EF0E9FBBAF9023088FB0320DB171B
:10151000C3EBA00080B20EF0C5FBBAF9003088FB27
:101520000320DB17C3EBA00080B20EF0BBFBBAF9BF
:10153000043088FB0320DB17C3EBA00080B20EF061
:10154000B1FB99F800103868F4F792FB94F85C311D
:1015500013F0010800F01184CB4AC4F858B10133EC
:10156000DBB2A2FB0312D20802EB8202A3EB42031E
:1015700084F85C31FFF734B9C44BC5491868F4F7F7
:1015800043FB00232370FFF7A3B9C24F386800283C
:101590003FF415A94FF0000ADFF84083BE4CAB467C
:1015A0005546F4F761FBF8B1F5B94FF00109AA46C9
:1015B0003868F4F751FB83B27E2B00F0A48298F8D0
:1015C0000120002A49D194F84811B1B11B2B84F8AD
:1015D000482100F072820D2B45D0386888F80190C0
:1015E000F4F742FB0028E3D1AA4650460AAAAB49C9
:1015F0005D460EF089FBFFF7E2B87D2B00F06484B6
:1016000094F84C2122B180F02003DBB284F84C1115
:1016100094F84721062A10D8B4F84A1138681944BA
:10162000A4F84A11A118013281F8503184F84721F9
:10163000F4F71AFB0028BBD1D6E7B4F84A2188F8A2
:10164000019013449BB21A0A52FA83F3FF2BA4F8B9
:101650004A31386802D1924DA3E73868F4F704FBA9
:101660000028A5D1C0E73868A4F84A21F4F7FCFAAD
:1016700000289DD1B8E794F8B832C4F8B452012BD1
:1016800040F2658394F8B9228649981801EB8001ED
:10169000013202F001024E6A84F8B922BEB1824FD3
:1016A0000B970DF14808123FA52348F8207D8022B2
:1016B00084F8103115232946404684F8112184F816
:1016C0001231B047002840F0C78294F8B832774A08
:1016D000013382FB0312A2EBE37202EB42029B1A7C
:1016E00084F8B832FFF7ACB8714A724B92F80BE04D
:1016F000029AD4F8341110681B886F4A401A4FF4CC
:101700007A71DFB201FB0EF11B0A977717758842D9
:101710004FF00007D37753759770177180F00483EB
:10172000664B6749DFF8A4E11B68DFF898C10F68D2
:101730008868DCF80010C4F830518EFB038CDB178E
:10174000C3EB6C13DFF88CC18EFB018E8CFB07980A
:101750008CFB009CC017C0EBAC0003F5FA734FEA9A
:10176000E17C9BB2CCEB6E1CFF1701F5EA4EC7EB98
:10177000A8070EF1300E93761B0A0CF1780C4FEA95
:101780002E2E3031D3764FEA27280312177782F8AE
:101790001D8082F8200082F8213082F824C082F86F
:1017A00023E082F82210FEF79CBFDFF83491D9F8CD
:1017B0000000F4F74DFA00283FF420A8D9F8000003
:1017C0000121F4F741FA0222002387F8742088F8F7
:1017D0000030FFF713B85E2090473B6830209847F1
:1017E000384BD3F800905FFA89F00EF0ADFDC9F3E5
:1017F00007200EF0A9FD94F82C3113F003097FF4B3
:1018000000A93149D4F828212C4B8A42186840F2AB
:10181000AF8480EAE073A3EBE0732C4A1BB282FB37
:1018200003124FEAE37BCBEB621B4FF0640909FB29
:101830001B390FFA89F90FFA8BFB5FFA89FA5FFA05
:101840008BF2C9F30729CBF3072B3B6802925E208A
:1018500098473B6810209847029A10460EF074FD96
:1018600058460EF071FD3B685E2098473B6821208A
:10187000984750460EF068FD48460EF065FDD8F8D2
:1018800000303A68FEF710BFCDCCCCCCEC7700200E
:1018900040770020C04F00200C2700205228002055
:1018A0005C280020FC53030831280020565555556C
:1018B0007C4D0020244D0020BC7700205C4F002090
:1018C000104D0020604F00203F4B4C001F85EB5116
:1018D000644F002067666666346500200C000020B7
:1018E000006A0020DFF858939FEDCA8A4FF0240A5F
:1018F0005E20904750463B689847C74BF9EC016A19
:101900009B8A07EE103AF8EEE66AB8EEC77A0AF15B
:10191000010AC6EE877A5FFA8AFA67EE887AFDEEE8
:10192000E77ACDED027ABDF908B05FFA8BF00EF0E0
:101930000BFDCBF307200EF007FDBAF1270F00F0E7
:10194000B7803A68D4E75E2090473B68022098470A
:10195000FF200DF001FF0378FF2B00F0C68390F904
:1019600001304FEAE3795FFA89F9D8B20EF0ECFC66
:1019700048460EF0E9FC3B685E2098473B68032030
:101980009847FF200DF0E8FE0378FF2B00F0A983B5
:10199000B0F90830D8B2C3F307290EF0D5FC484699
:1019A0000EF0D2FC9D4B1B78042B77D0DFF894B25D
:1019B000B4F82E119BF80020DFF88CA291FBF2F313
:1019C00002FB13139BB2BAF80010A4F82E314FEAB1
:1019D00003191FFA89F9642303FB01235200B3FBA7
:1019E000F2F349EA0329C3F303225E203B681FFA9E
:1019F00089F949EA020998473B68062098475FFA47
:101A000089F00EF0A1FC4FEA19200EF09DFC8449EC
:101A1000B4F82E214B7ABAF800A00132012BA4F8B9
:101A20002E2100F0A9854A7B0AEB8A031FFA83FA6C
:101A3000002A40F0DD833B685E2098473B683A20EF
:101A40009847784BA3FB0A394FEA59191FFA89FBCB
:101A50005FFA8BF00EF078FC4FEA1B200EF074FC5E
:101A60003B685E2098473B683B209847642303FB14
:101A700019A39BB26C48053380FB0320DB17C3EB33
:101A8000A000C0B20EF060FC00200EF05DFCDFF89C
:101A9000BC9199F80630002B40F06F83D8F80030E5
:101AA0001B0700F1228294F82C313A68FEF706BE3B
:101AB000D8F800303A68FEF7F3BD3868F4F7D4F888
:101AC00000287FF48AAD386884F8469188F8019040
:101AD000F4F7CAF800287FF46BAD85E5F3F740FE14
:101AE000524B1B68A0EB030B40F6B8339B4500F24A
:101AF000D6814F4B1A793A2A00F05484002388F893
:101B00000030FEF77BBE386884F846A184F847A110
:101B100084F8489188F801A0F4F7A6F800287FF42B
:101B200047AD61E594F8441194F8453141484A1CA9
:101B3000FEF731BE013A84F86B21FFF799B9013BFA
:101B400084F86A31FFF76AB8013B84F87331C1E465
:101B5000013F84F87271FFF76CBA4FF0000A5E2003
:101B6000D3F8008084F82CA190473B68DFF8E09020
:101B70001720984750460EF0E7FB2F4BA3FB082396
:101B80009B0BA9FB03125209C2EB0212A3EB8203C7
:101B9000D8B20EF0D9FB3B685E2098473B6818200E
:101BA0009847264BA3FB08239B09A9FB0312520964
:101BB000C2EB0212A3EB8203D8B20EF0C5FB504673
:101BC0000EF0C2FB3A68FEF77EBD0024DFF8848089
:101BD00027464FF0500A02E0DBB283F3118816F873
:101BE00004B0601C594630440DF05AFF002840F004
:101BF00075810BF101031C44EFF311838AF3128802
